:1000000000000320A55C0100895C0100415C010047
:10001000415C0100415C0100415C0100415C010068
:10002000415C0100415C0100415C0100895C010010
:10003000895C0100415C01005D510100D553010064
:10004000895C0100895C0100895C0100895C010018
:10005000895C0100895C0100895C0100895C010008
:10006000895C0100895C0100895C0100895C0100F8
:10007000895C0100895C0100895C0100895C0100E8
:10008000895C0100895C0100895C0100895C0100D8
:10009000895C0100895C0100895C0100895C0100C8
:1000A00059120100B5130100895C0100895C01004F
:1000B000895C0100895C0100895C0100F96E010026
:1000C000895C010021910100895C01007D920100A1
:1000D000895C0100AD930100895C0100895C01002D
:1000E000895C0100895C0100895C0100895C010078
:1000F000895C0100895C0100895C0100895C010068
:10010000895C0100895C0100895C0100895C010057
:10011000895C0100E5710100895C0100895C0100D6
:10012000895C0100895C0100895C0100895C010037
:10013000895C0100895C0100895C0100895C010027
:10014000A94E0100895C0100DD940100895C010079
:10015000895C0100895C0100895C0100895C010007
:10016000895C0100895C010011150100895C0100B6
:10017000895C0100895C0100895C0100895C0100E7
:10018000895C010069F80000895C0100895C01005C
:10019000895C0100895C01000D960100895C010009
:1001A000895C0100895C0100895C0100895C0100B7
:1001B000895C0100895C0100895C0100895C0100A7
:1001C000895C0100895C0100895C0100895C010097
:1001D000FFFFFFFFFFFFFFFFFFFFFFFFFFFFFFFF2F
:10040000FFFFFFFFFFFFFFFFFFFFFFFFDEF9FFFF23
:1004100010B5054C237833B9044B13B10448AFF33E
:1004200000800123237010BD00B0FF1F00000000FA
:100430006C050F00084B10B51BB108490848AFF315
:1004400000800848036803B910BD074B002BFBD0A0
:10045000BDE81040184700BF0000000004B0FF1FB7
:100460006C050F0050A2FF1F0000000049F2F823A6
:10047000C1F6FF731B7C022B9DBF41F24C52C0F2B0
:10048000020252F823000020704700BF49F2F8230F
:10049000C1F6FF735B7C032B9DBF41F26852C0F233
:1004A000020252F823000020704700BF49F2F823EF
:1004B000C1F6FF7349F2A422987C49F2B023C1F639
:1004C000FF72C1F6FF7300280CBF10461846704734
:1004D00049F2F823C1F6FF7393F822306BB149F269
:1004E0002C33C1F6FF7346F64F62C0F2200249F288
:1004F0002C301A60C1F6FF70704749F22C33C1F6F8
:10050000FF7346F24F62C0F2660249F22C301A6065
:10051000C1F6FF70704700BF704700BF704700BF53
:10052000704700BF704700BF08B549F2F823C1F615
:10053000FF73DA7C72B14FF6E07149F22030C0F2FD
:100540000101C1F6FF701CF00BFB49F22030C1F62F
:10055000FF7008BD4FF6D47149F22030C0F201019E
:10056000C1F6FF701CF0FCFA49F22030C1F6FF70B2
:1005700008BD00BF10B549F2F823C1F6FF73B2EE13
:10058000047A1B7D07EE903AF8EE677A49F2BC24B4
:10059000C7EE876AC1F6FF7416EE900A1BF008F8E2
:1005A0000B464FF6EC710246C0F2010120461CF0EA
:1005B000D7FA204610BD00BF10B549F2F823C1F6A6
:1005C000FF73B2EE047A5B7D07EE903AF8EE677A3D
:1005D00049F23834C7EE876AC1F6FF7416EE900A06
:1005E0001AF0E6FF0B464FF6EC710246C0F201012D
:1005F00020461CF0B5FA204610BD00BF10B549F2E8
:10060000F823C1F6FF7349F24434C1F6FF744FF684
:10061000F87193F90A202046C0F201011CF0A0FAFB
:10062000204610BD10B5044614F0C0FB204610BD96
:1006300008B549F2F823C1F6FF7393F8212072B18F
:1006400040F20C0149F2C420C0F20201C1F6FF7071
:100650001CF086FA49F2C420C1F6FF7008BD40F2D2
:100660000403C0F2020393E8030049F2C423C1F675
:10067000FF731860197149F2C420C1F6FF7008BDFC
:10068000006803681B68184700F0F703F52B06D0D5
:10069000F92804D0EF2803D800F0F00070470020BC
:1006A000704700BF38B549F2E464C1F6FF740146F3
:1006B00000230A22204614F095FF0546204614F038
:1006C0007FFF284438BD00BF10B504461CF078FAFF
:1006D00001462046BDE8104018F026BB10B5044680
:1006E0001CF06EFA0146204618F01EFB044649F243
:1006F000E460C1F6FF7014F063FF204410BD00BF3A
:1007000040F2140070B5C0F20200FFF7E7FF40F2BC
:100710003800C0F202004DF23044FFF7DFFFC2F2B2
:1007200000044CF6E031C2F20001204611F0F6FE62
:1007300040F23C00C0F202004DF21806FFF7CEFF77
:10074000C1F6FF764CF2A433C2F2000340F240003F
:1007500049F2F8257268DA70C1F6FF75C0F202003E
:10076000FFF7BCFF40F244006B7E7360C0F20200F2
:10077000FFF7B4FF44F2C013C2F2000300211420BB
:100780006A7E986383F83C10596372B68242A8BFB0
:1007900002469200DA6262B640F24800C0F20200FD
:1007A000FFF79CFF204611F005FF40F24C00C0F21D
:1007B0000200BDE87040FFF791BF00BF40F250005B
:1007C00010B51621C0F2020018F0AEFA49F2E4604A
:1007D000C1F6FF704DF2304414F0F2FEC2F2000494
:1007E0004CF2E0712046C2F2000111F097FE4DF28A
:1007F0001802C1F6FF724CF2A433C2F20003526831
:100800001A702046BDE8104011F0D4BE38B5044639
:1008100040F268000D46C0F202000D2118F084FA83
:1008200049F2F823C1F6FF7393F822300BB32B047F
:1008300003F4FE03013C43F44043240243F00C0361
:1008400004F470641C434DF6A0602146C2F200001F
:1008500013F054FD40F27800C0F20200FFF734FFBD
:10086000204617F0D7FB40F29000C0F20200FFF7DD
:100870002BFF49F2E460C1F6FF70BDE8384014F088
:100880009FBE00BF38B5044640F2A0000D46C0F23E
:1008900002000D2118F048FA49F2F823C1F6FF735F
:1008A00093F822300BB32B0403F4FE03013C43F412
:1008B0005043240243F00D0304F470641C434DF6CE
:1008C000A0602146C2F2000013F018FD40F278004B
:1008D000C0F20200FFF7F8FE204617F09BFB40F243
:1008E0009000C0F20200FFF7EFFE49F2E460C1F6AB
:1008F000FF70BDE8384014F063BE00BF70B5064617
:1009000040F2B0000C46C0F202001221154618F069
:100910000BFA49F2F823C1F6FF7393F822303BB982
:1009200049F2E460C1F6FF70BDE8704014F048BEC3
:100930006B1E1B02240404F4FE0403F470632343BF
:1009400043F45043340143F00D03E4B21C434DF62D
:10095000A060C2F20000214613F0D0FC40F2780003
:10096000C0F20200FFF7B0FE6EB140F29000C0F29C
:100970000200FFF7A9FE49F2E460C1F6FF70BDE88E
:10098000704014F01DBE204617F044FBEDE700BF99
:1009900038B5044640F2C400C0F202001A2118F033
:1009A000C3F949F2F823C1F6FF7393F822301BB361
:1009B0004DF6E445C1F6FF75F321A86C03681B688A
:1009C0009847A86C036804F07F01DB6C984740F2FD
:1009D000E000C0F20200FFF777FE200400F4FE0002
:1009E00040F4734040F0020017F014FB40F2900016
:1009F000C0F20200FFF768FE49F2E460C1F6FF7042
:100A0000BDE8384014F0DCBD38B5044640F2F000D3
:100A1000C0F20200242118F087F949F2F823C1F648
:100A2000FF7393F822301BB34DF6E445C1F6FF7512
:100A3000F121A86C03681B689847A86C03682146DD
:100A40001B68984740F2E000C0F20200FFF73CFE4E
:100A500004F00F044FF202102404C0F210002043EF
:100A600017F0D8FA40F29000C0F20200FFF72CFE17
:100A700049F2E460C1F6FF70BDE8384014F0A0BD53
:100A800038B5044640F21810C0F20200152118F0E3
:100A90004BF949F2F823C1F6FF7393F822303BB3C8
:100AA0004DF6E445C1F6FF75F321A86C03681B6899
:100AB0009847A86C036804F07F01DB6C984740F20C
:100AC000E000C0F20200FFF7FFFD210401F4FE0187
:100AD00041F473414DF6A060C2F2000041F0020102
:100AE00013F00CFC40F27800C0F20200FFF7ECFDBE
:100AF00049F2E460C1F6FF70BDE8384014F060BD13
:100B000038B5054640F230100C46C0F202000D2107
:100B100018F00AF949F2F823C1F6FF7393F822306E
:100B20004BB304F30D0404F500536C1E1A042402A5
:100B300002F4FE0204F47064144344F460445B0461
:100B400003F0FE4344F00E041C434DF6A060214622
:100B5000C2F2000013F0D2FB40F27800C0F20200B3
:100B6000FFF7B2FD204617F055FA40F29000C0F2B0
:100B70000200FFF7A9FD49F2E460C1F6FF70BDE88D
:100B8000384014F01DBD00BF38B5044640F2401097
:100B9000C0F202001F2118F0C7F849F2F823C1F68D
:100BA000FF7393F822303BB34DF6E445C1F6FF7571
:100BB000F121A86C03681B689847A86C036821465C
:100BC0001B68984740F2E000C0F20200FFF77CFD8E
:100BD00004F00F044FF202112404C0F210014DF68C
:100BE000A060C2F20000214313F088FB40F27800BD
:100BF000C0F20200FFF768FD49F2E460C1F6FF7041
:100C0000BDE8384014F0DCBC10B540F260104CF286
:100C1000A434C2F200042A21C0F2020018F084F8C1
:100C200049F2E46094F90310C1F6FF7014F06AFC15
:100C300049F2E460C1F6FF7014F0C2FC4EF2B871E4
:100C40004DF23040C2F20001C2F2000011F066FC29
:100C50004DF230400221C2F2000011F087FC4DF24B
:100C60001801C1F6FF7194F903204B682370002A24
:100C700044F2C013C2F2000315DB12240020A2428A
:100C80004A609C6383F83C005863D4BF92004822BA
:100C900072B6DA6262B64DF23040C2F20000BDE8D0
:100CA000104011F087BC00221220986383F83C208A
:100CB0005A63E2704A6072B6DA6262B64DF2304050
:100CC000C2F20000012111F04BFCE4E738B5054603
:100CD00049F2E46440F28C10C1F6FF741E21C0F2A8
:100CE000020018F021F8294600230A22204614F0B9
:100CF00079FC40F2AC100E21C0F2020018F014F89A
:100D000049F2F823C1F6FF730A2293F82110204616
:100D1000002314F067FC40F2BC100121C0F2020075
:100D200018F002F8204614F04BFC002038BD00BF3C
:100D3000F8B549F2F824C1F6FF740F4694F8213053
:100D40001646054623B1984202D0FFF7BFFF50B1C7
:100D50004BF21C23C2F2000394F9091018683944BD
:100D600000220BF0B7FD40F2C010C0F202001221C9
:100D700017F0DAFF94F822302BB3330603F0FE436A
:100D800043F400433F04013D43F0080307F4FE072A
:100D90002D023B4305F470651D434DF6A0602946C6
:100DA000C2F2000013F0AAFA40F27800C0F202008A
:100DB000FFF78AFC284617F02DF940F29000C0F2A8
:100DC0000200FFF781FC49F2E460C1F6FF70BDE864
:100DD000F84014F0F5BB00BFF8B549F2F824C1F6AD
:100DE000FF740F4694F821301646054623B1984209
:100DF00002D0FFF76BFF50B14BF21C23C2F200038D
:100E000094F909101868394432460BF063FD40F23A
:100E1000D410C0F20200112117F086FF94F822309E
:100E20002BB3360606F0FE4646F410463F04013D5D
:100E300046F0090607F4FE072D023E4305F47065EF
:100E400035434DF6A0602946C2F2000013F056FA71
:100E500040F27800C0F20200FFF736FC284617F097
:100E6000D9F840F29000C0F20200FFF72DFC49F2E1
:100E7000E460C1F6FF70BDE8F84014F0A1BB00BF0C
:100E8000F8B549F2F826C1F6FF760F4696F82130FC
:100E90001546044623B1984202D0FFF717FF48B128
:100EA0004BF21C23C2F200032A4618680368394635
:100EB0005B68984740F2E810C0F202000D2117F07D
:100EC00033FF96F822302BB32D0605F0FE4545F48E
:100ED00030453F04013C45F00B0507F4FE072402B2
:100EE0003D4304F470642C434DF6A0602146C2F2E9
:100EF000000013F003FA40F27800C0F20200FFF79E
:100F0000E3FB204617F086F840F29000C0F20200A2
:100F1000FFF7DAFB49F2E460C1F6FF70BDE8F84084
:100F200014F04EBB40F2F81038B51A21C0F202009E
:100F300017F0FAFE49F2E460C1F6FF704DF230445A
:100F400014F03EFBC2F200044DF25C712046C2F286
:100F5000000111F0E3FA4DF21801C1F6FF7149F2F8
:100F6000F8224CF2A430C2F20000C1F6FF7244F243
:100F7000C013C2F200034D68457192F820204A6008
:100F8000002063259D6383F83C00586372B6AA4233
:100F9000A8BF2A469200DA6262B62046BDE8384011
:100FA00011F008BB40F2142070B51C21C0F2020001
:100FB00017F0BAFE49F2E460C1F6FF7014F000FBCE
:100FC0004BF63C314DF23040C2F20001C2F200005B
:100FD00011F0A4FA49F24032C1F6FF724DF2180145
:100FE000C1F6FF7112784E684A604CF2A43044F2A8
:100FF000C013C2F200036321C2F2000000250124E5
:101000008A42067083F83C505C6399630EDC5AB1E7
:10101000920072B6DA6262B64DF23040C2F200005F
:10102000BDE8704011F0C6BA0422F2E74FF4C67270
:10103000EFE700BF40F2342070B51A21C0F2020081
:1010400017F072FE49F2E460C1F6FF7014F0B8FACE
:101050004DF2F0314DF23040C2F20001C2F2000018
:1010600011F05CFA49F2F822C1F6FF724DF2180154
:10107000C1F6FF7192F823204E684A604CF2A4300A
:1010800044F2C013C2F200033021C2F20000002576
:1010900001248A42467183F83C505C6399630EDCFC
:1010A0005AB1920072B6DA6262B64DF23040C2F2C4
:1010B0000000BDE8704011F07DBA0422F2E7C022C2
:1010C000F0E700BF40F2502038B51E21C0F2020008
:1010D00017F02AFE49F2E460C1F6FF704DF2304489
:1010E00014F06EFAC2F200044DF2B0312046C2F2A2
:1010F000000111F013FA4DF21801C1F6FF7149F227
:10110000F8224CF2A430C2F20000C1F6FF7244F2A1
:10111000C013C2F200034D68457192F821204A6065
:10112000002010259D6383F83C00586372B6AA42E4
:10113000A8BF2A469200DA6262B62046BDE838406F
:1011400011F038BA40F2702038B51D21C0F202000B
:1011500017F0EAFD49F2E460C1F6FF704DF2304449
:1011600014F02EFAC2F200044AF618412046C2F2E8
:10117000000111F0D3F94DF21801C1F6FF7149F2E7
:10118000F8224CF2A430C2F20000C1F6FF7244F221
:10119000C013C2F200034D68C570127D4A60002082
:1011A00063259D6383F83C00586372B6AA42A8BFCA
:1011B0002A469200DA6262B62046BDE8384011F055
:1011C000F9B900BF40F29020F8B51B21C0F202002F
:1011D00017F0AAFD49F2E460C1F6FF704DF2304409
:1011E00014F0EEF9C2F200044AF6D8312046C2F2F9
:1011F000000111F093F949F2F823C1F6FF734DF2A3
:101200001801C1F6FF7193F91F304F684B604CF223
:10121000A43044F2C012C2F200026FF03101C2F2F7
:101220000000002632258B42C770B8BF0B465163C1
:1012300082F83C60956372B6AB42A8BF2B469B0018
:10124000D36262B62046BDE8F84011F0B3B900BFE2
:1012500040F2AC2038B51E21C0F2020017F064FD48
:1012600049F2E460C1F6FF704DF2304414F0A8F981
:10127000C2F200044CF264312046C2F2000111F0C7
:101280004DF94DF21801C1F6FF7149F2F8224CF206
:10129000A430C2F20000C1F6FF7244F2C013C2F2E1
:1012A00000034D68C570127E4A60002063259D636F
:1012B00083F83C00586372B6AA42A8BF2A4692003F
:1012C000DA6262B62046BDE8384011F073B900BF5B
:1012D00040F2CC2038B52021C0F2020017F024FDE6
:1012E00049F2E460C1F6FF704DF2304414F068F941
:1012F000C2F200044DF688112046C1F6FF7111F0CC
:101300000DF94DF21801C1F6FF7149F2F8224CF2C5
:10131000A430C2F20000C1F6FF7244F2C013C2F260
:1013200000034D68C570D27C4A60002060259D6333
:1013300083F83C00586372B6AA42A8BF2A469200BE
:10134000DA6262B62046BDE8384011F033B900BF1A
:1013500040F2F02038B51E21C0F2020017F0E4FC84
:1013600049F2E460C1F6FF704DF2304414F028F900
:10137000C2F200044CF620012046C2F2000111F036
:10138000CDF84DF21801C1F6FF7149F2F8224CF286
:10139000A430C2F20000C1F6FF7244F2C013C2F2E0
:1013A00000034D68C570D27E4A60002063259D63AE
:1013B00083F83C00586372B6AA42A8BF2A4692003E
:1013C000DA6262B62046BDE8384011F0F3B800BFDB
:1013D00040F2103038B52021C0F2020017F0A4FC12
:1013E00049F2E460C1F6FF704DF2304414F0E8F8C1
:1013F000C2F200044DF25C012046C2F2000111F07D
:101400008DF84DF21801C1F6FF7149F2F8224CF245
:10141000A430C2F20000C1F6FF7244F2C013C2F25F
:1014200000034D68C570927B4A60002063259D6370
:1014300083F83C00586372B6AA42A8BF2A469200BD
:10144000DA6262B62046BDE8384011F0B3B800BF9A
:1014500040F23430F8B51921C0F2020017F064FCF4
:1014600049F2E460C1F6FF704DF2304414F0A8F880
:10147000C2F200044DF6D0512046C1F6FF7111F0C2
:101480004DF849F2F823C1F6FF734DF21801C1F689
:10149000FF7193F91E304F684B604CF2A43044F258
:1014A000C012C2F200026FF03101C2F20000002649
:1014B00032258B42C770B8BF0B46516382F83C603F
:1014C000956372B6AB42A8BF2B469B00D36262B64F
:1014D0002046BDE8F84011F06DB800BF40F2503032
:1014E00038B51C21C0F2020017F01EFC49F2E4607E
:1014F000C1F6FF704DF2304414F062F8C2F20004FD
:101500004BF694212046C1F6FF7111F007F84DF219
:101510001801C1F6FF7149F2F8224CF2A430C2F270
:101520000000C1F6FF7244F2C013C2F200034D681E
:10153000C570927C4A60002001259D6383F83C00C1
:10154000586372B69200DA6262B62046BDE838404F
:1015500011F030B840F2703038B51E21C0F20200F0
:1015600017F0E2FB49F2E460C1F6FF704DF230443F
:1015700014F026F8C2F200044DF6E8312046C1F618
:10158000FF7110F0CBFF4DF21801C1F6FF7149F267
:10159000F8224CF2A430C2F20000C1F6FF7244F20D
:1015A000C013C2F200034D68C570927E4A600020ED
:1015B00014259D6383F83C00586372B6AA42A8BF05
:1015C0002A469200DA6262B62046BDE8384010F042
:1015D000F1BF00BF40F2903038B52021C0F20200C8
:1015E00017F0A2FB49F2E460C1F6FF704DF23044FF
:1015F00013F0E6FFC2F200044DF628112046C2F2B5
:10160000000110F08BFF4DF21801C1F6FF7149F295
:10161000F8224CF2A430C2F20000C1F6FF7244F28C
:10162000C013C2F200034D688570127B4A6000202F
:1016300063259D6383F83C00586372B6AA42A8BF35
:101640002A469200DA6262B62046BDE8384010F0C1
:10165000B1BF00BF40F2B43038B51F21C0F2020064
:1016600017F062FB49F2E460C1F6FF704DF23044BE
:1016700013F0A6FFC2F200044EF6B4012046C2F2F7
:10168000000110F04BFF4DF21801C1F6FF7149F255
:10169000F8224CF2A430C2F20000C1F6FF7244F20C
:1016A000C013C2F200034D68C570127F4A6000206B
:1016B00063259D6383F83C00586372B6AA42A8BFB5
:1016C0002A469200DA6262B62046BDE8384010F041
:1016D00071BF00BF40F2D430F8B51621C0F202004D
:1016E00017F022FB49F2E460C1F6FF704DF230447E
:1016F00013F066FFC2F200044BF23C412046C1F6F3
:10170000FF7110F00BFF49F2F823C1F6FF734DF2A1
:101710001801C1F6FF7193F90A304F684B604CF223
:10172000A43044F2C012C2F200026FF03101C2F2E2
:101730000000002632258B428770B8BF0B465163EC
:1017400082F83C60956372B6AB42A8BF2B469B0003
:10175000D36262B62046BDE8F84010F02BBF00BF50
:1017600040F2EC3038B52121C0F2020017F0DCFA6B
:1017700049F2E460C1F6FF704DF2304413F020FFEF
:10178000C2F200044CF6A4612046C2F2000110F03F
:10179000C5FE4DF21801C1F6FF7149F2F8224CF274
:1017A000A430C2F20000C1F6FF7244F2C013C2F2CC
:1017B00000034D68C570527F4A60002063259D6319
:1017C00083F83C00586372B6AA42A8BF2A4692002A
:1017D000DA6262B62046BDE8384010F0EBBE00BFCA
:1017E00040F2104070B51821C0F2020017F09CFAC8
:1017F00049F2E460C1F6FF704DF2304413F0E0FEB0
:10180000C2F200044CF2D0312046C2F2000110F0C6
:1018100085FE49F2F823C1F6FF734DF21801C1F6B7
:10182000FF714CF2A43044F2C012C2F2000293F9EC
:1018300008304E684B60C2F200000021632523EAA5
:10184000E3738670956382F83C10516372B6AB42C5
:10185000A8BF2B469B00D36262B62046BDE870400D
:1018600010F0A8BE40F22C40F8B51B21C0F20200D7
:1018700017F05AFA49F2E460C1F6FF704DF23044B5
:1018800013F09EFEC2F200044DF660012046C2F243
:10189000000110F043FE49F2F823C1F6FF734DF248
:1018A0001801C1F6FF7193F909304F684B604CF293
:1018B000A43044F2C012C2F200026FF01701C2F26B
:1018C0000000002618258B428770B8BF0B46516375
:1018D00082F83C60956372B6AB42A8BF2B469B0072
:1018E000D36262B62046BDE8F84010F063BE00BF88
:1018F00040F2484038B51B21C0F2020017F014FA3C
:1019000049F2E460C1F6FF704DF2304413F058FE26
:10191000C2F200044CF270412046C2F2000110F005
:10192000FDFD4DF21801C1F6FF7149F2F8224CF2AB
:10193000A430C2F20000C1F6FF7244F2C013C2F23A
:1019400000034D68C570127C4A60002002259D632B
:1019500083F83C00586372B6AA42A8BF2A46AA4040
:10196000DA6262B62046BDE8384010F023BE00BF00
:1019700040F2644038B52021C0F2020017F0D4F9DB
:1019800049F2E460C1F6FF704DF2304413F018FEE6
:10199000C2F200044DF29C012046C2F2000110F098
:1019A000BDFD4DF21801C1F6FF7149F2F8224CF26B
:1019B000A430C2F20000C1F6FF7244F2C013C2F2BA
:1019C00000034D68C570D27D4A60002063259D6389
:1019D00083F83C00586372B6AA42A8BF2A46920018
:1019E000DA6262B62046BDE8384010F0E3BD00BFC1
:1019F00040F2884038B52121C0F2020017F094F976
:101A000049F2E460C1F6FF704DF2304413F0D8FDA6
:101A1000C2F200044DF67C212046C2F2000110F013
:101A20007DFD4DF21801C1F6FF7149F2F8224CF22A
:101A3000A430C2F20000C1F6FF7244F2C013C2F239
:101A400000034D68C570927D4A60002063259D6348
:101A500083F83C00586372B6AA42A8BF2A46920097
:101A6000DA6262B62046BDE8384010F0A3BD00BF80
:101A700040F2AC4038B51C21C0F2020017F054F916
:101A800049F2E460C1F6FF704DF2304413F098FD66
:101A9000C2F200044BF200112046C1F6FF7110F0B3
:101AA0003DFD4DF21801C1F6FF7149F2F8224CF2EA
:101AB000A430C2F20000C1F6FF7244F2C013C2F2B9
:101AC00000034D68C570527D4A60002063259D6308
:101AD00083F83C00586372B6AA42A8BF2A46920017
:101AE000DA6262B62046BDE8384010F063BD00BF40
:101AF00040F2CC4038B52021C0F2020017F014F9B2
:101B000049F2E460C1F6FF704DF2304413F058FD25
:101B1000C2F200044BF2C0012046C1F6FF7110F082
:101B2000FDFC4DF21801C1F6FF7149F2F8224CF2AA
:101B3000A430C2F20000C1F6FF7244F2C013C2F238
:101B400000034D68457192F822204A60002001256B
:101B50009D6383F83C00586372B69200DA6262B605
:101B60002046BDE8384010F025BD00BF40F2F040EF
:101B700038B51821C0F2020017F0D6F849F2E46037
:101B8000C1F6FF704DF2304413F01AFDC2F20004AA
:101B90004BF2CC312046C2F2000110F0BFFC4DF2F6
:101BA0001801C1F6FF7149F2F8224CF2A430C2F2DA
:101BB0000000C1F6FF7244F2C013C2F200034D6888
:101BC0008570D2794A60002063259D6383F83C00CC
:101BD000586372B6AA42A8BF2A469200DA6262B679
:101BE0002046BDE8384010F0E5BC00BF40F20C5084
:101BF00038B52421C0F2020017F096F849F2E460EB
:101C0000C1F6FF704DF2304413F0DAFCC2F200046A
:101C10004BF220412046C2F2000110F07FFC4DF251
:101C20001801C1F6FF7149F2F8224CF2A430C2F259
:101C30000000C1F6FF7244F2C013C2F200034D6807
:101C4000C570527B4A60002063259D6383F83C0089
:101C5000586372B6AA42A8BF2A469200DA6262B6F8
:101C60002046BDE8384010F0A5BC00BF40F234501B
:101C700038B51F21C0F2020017F056F849F2E460AF
:101C8000C1F6FF704DF2304413F09AFCC2F200042A
:101C90004DF69C212046C1F6FF7110F03FFC4DF23D
:101CA0001801C1F6FF7149F2F8224CF2A430C2F2D9
:101CB0000000C1F6FF7244F2C013C2F200034D6887
:101CC000C570527C4A60002003259D6383F83C0068
:101CD000586372B6AA42A8BF2A469200DA6262B678
:101CE0002046BDE8384010F065BC00BF40F25450BB
:101CF00038B51921C0F2020017F016F849F2E46075
:101D0000C1F6FF704DF2304413F05AFCC2F20004E9
:101D10004CF60C112046C1F6FF7110F0FFFB4DF29E
:101D20001801C1F6FF7149F2F8224CF2A430C2F258
:101D30000000C1F6FF7244F2C013C2F200034D6806
:101D4000857052794A60002063259D6383F83C00CA
:101D5000586372B6AA42A8BF2A469200DA6262B6F7
:101D60002046BDE8384010F025BC00BF40F270505E
:101D700038B51821C0F2020016F0D6FF49F2E4602F
:101D8000C1F6FF704DF2304413F01AFCC2F20004A9
:101D90004DF2CC712046C1F6FF7110F0BFFB4DF241
:101DA0001801C1F6FF7149F2F8224CF2A430C2F2D8
:101DB0000000C1F6FF7244F2C013C2F200034D6886
:101DC0008570D27A4A60002063259D6383F83C00C9
:101DD000586372B6AA42A8BF2A469200DA6262B677
:101DE0002046BDE8384010F0E5BB00BF40F28C5003
:101DF00038B51A21C0F2020016F096FF49F2E460ED
:101E0000C1F6FF704DF2304413F0DAFBC2F2000469
:101E10004DF624612046C1F6FF7110F07FFB4DF2B4
:101E20001801C1F6FF7149F2F8224CF2A430C2F257
:101E30000000C1F6FF7244F2C013C2F200034D6805
:101E4000857092794A60002063259D6383F83C0089
:101E5000586372B6AA42A8BF2A469200DA6262B6F6
:101E60002046BDE8384010F0A5BB00BF40F2A850A6
:101E700038B51B21C0F2020016F056FF49F2E460AB
:101E8000C1F6FF704DF2304413F09AFBC2F2000429
:101E90004CF228612046C2F2000110F03FFB4DF2E7
:101EA0001801C1F6FF7149F2F8224CF2A430C2F2D7
:101EB0000000C1F6FF7244F2C013C2F200034D6885
:101EC000C570D27B4A60002063259D6383F83C0087
:101ED000586372B6AA42A8BF2A469200DA6262B676
:101EE0002046BDE8384010F065BB00BF40F2C4504A
:101EF00038B51721C0F2020016F016FF49F2E4606F
:101F0000C1F6FF704DF2304413F05AFBC2F20004E8
:101F10004BF6F4412046C2F2000110F0FFFA4DF2F8
:101F20001801C1F6FF7149F2F8224CF2A430C2F256
:101F30000000C1F6FF7244F2C013C2F200034D6804
:101F4000857012794A60002063259D6383F83C0008
:101F5000586372B6AA42A8BF2A469200DA6262B6F5
:101F60002046BDE8384010F025BB00BF40F2DC50F1
:101F700070B51C21C0F2020016F0D6FE49F2E460F2
:101F8000C1F6FF7013F01CFB4AF6DC214DF2304025
:101F9000C2F20001C2F2000010F0C0FA49F2403271
:101FA000C1F6FF724DF21801C1F6FF7112784E684A
:101FB0004A604CF2A43044F2C013C2F20003632121
:101FC000C2F20000002501248A42067083F83C50CA
:101FD0005C6399630EDC5AB1920072B6DA6262B643
:101FE0004DF23040C2F20000BDE8704010F0E2BA9D
:101FF0000422F2E74FF4C672EFE700BF40F2FC5054
:1020000008B5C0F20200142116F08EFE49F2F82342
:10201000C1F6FF7393F82230D3B14DF6E443C1F615
:10202000FF73FC21986C03681B68984740F2E0003E
:102030000F21C0F2020016F077FE4FF60F4015F0A8
:10204000E9FF40F29000C0F202000F2116F06CFE92
:1020500049F2E460C1F6FF70BDE8084013F0B0BA81
:1020600040F2146008B5C0F20200162116F05CFEC2
:1020700049F2F823C1F6FF7393F82230CBB14DF645
:10208000A060C2F200004FF20F6112F037F940F287
:1020900078001421C0F2020016F046FE4FF20F60E5
:1020A00015F0B8FF40F29000C0F202000F2116F0C8
:1020B0003BFE49F2E460C1F6FF70BDE8084013F052
:1020C0007FBA00BF40F22C6008B5C0F202001B21AD
:1020D00016F02AFE49F2F823C1F6FF7393F8223076
:1020E000D3B14DF6E443C1F6FF73FF21986C03684A
:1020F0001B68984740F2E0000F21C0F2020016F082
:1021000013FE4FF60F7015F085FF40F29000C0F2FD
:1021100002000F2116F008FE49F2E460C1F6FF70DC
:10212000BDE8084013F04CBA40F2486008B5C0F270
:102130000200152116F0F8FD49F2F823C1F6FF73ED
:1021400093F82230D3B14DF6E443C1F6FF73FA2180
:10215000986C03681B68984740F2E0000F21C0F2BA
:10216000020016F0E1FD4FF60F2015F053FF40F28C
:102170009000C0F202000F2116F0D6FD49F2E46093
:10218000C1F6FF70BDE8084013F01ABA40F2606073
:1021900008B5C0F202001D2116F0C6FD49F2F82371
:1021A000C1F6FF7393F82230D3B14DF6E443C1F684
:1021B000FF73FE21986C03681B68984740F2E000AB
:1021C0000F21C0F2020016F0AFFD4FF60F6015F0C0
:1021D00021FF40F29000C0F202000F2116F0A4FD92
:1021E00049F2E460C1F6FF70BDE8084013F0E8B9B9
:1021F00040F2806008B5C0F20200182116F094FD8C
:1022000049F2F823C1F6FF7393F82230D3B14DF6AB
:10221000E443C1F6FF73FB21986C03681B68984781
:1022200040F2E0000F21C0F2020016F07DFD4FF6F3
:102230000F3015F0EFFE40F29000C0F202000F21C7
:1022400016F072FD49F2E460C1F6FF70BDE8084087
:1022500013F0B6B940F29C6008B5C0F20200152137
:1022600016F062FD49F2F823C1F6FF7393F82230AD
:10227000D3B14DF6E443C1F6FF73F821986C0368BF
:102280001B68984740F2E0000F21C0F2020016F0F0
:102290004BFD4FF60F0015F0BDFE40F29000C0F26E
:1022A00002000F2116F040FD49F2E460C1F6FF7014
:1022B000BDE8084013F084B910B5044640F2B4609C
:1022C000C0F20200152116F02FFD49F2F823C1F6E5
:1022D000FF7393F82230F3B1240404F4FE0444F4B1
:1022E000734444F002044DF6A0602146C2F200009F
:1022F00012F004F840F278001421C0F2020016F047
:1023000013FD204615F086FE40F29000C0F2020058
:102310000F2116F009FD49F2E460C1F6FF70BDE837
:10232000104013F04DB900BF2DE9F041804640F256
:10233000CC600F46C0F20200152116F0F5FC49F200
:10234000F823C1F6FF7393F822303BB949F2E460F9
:10235000C1F6FF70BDE8F04113F032B94DF6E44527
:10236000C1F6FF75F021A86C0368DB6C984757B184
:10237000444608EB0706A86C14F8011B03681B68A9
:102380009847A642F7D1A86C0368F721DB6C984701
:1023900040F2E0000F21C0F2020016F0C5FC394601
:1023A0004046002215F08AFE40F29000C0F2020082
:1023B0000F2116F0B9FC49F2E460C1F6FF70BDE8E8
:1023C000F04113F0FDB800BF40F2E46008B5C0F280
:1023D0000200182116F0A8FC49F2F823C1F6FF7399
:1023E00093F82230CBB14DF6A060C2F200004FF658
:1023F0000F6111F083FF40F278001421C0F2020057
:1024000016F092FC4FF60F6015F004FE40F29000BB
:10241000C0F202000F2116F087FC49F2E460C1F619
:10242000FF70BDE8084013F0CBB800BF40F2007069
:1024300008B5C0F20200132116F076FC49F2F82329
:10244000C1F6FF7393F82230CBB14DF6A060C2F213
:1024500000004FF60F3111F051FF40F278001421C7
:10246000C0F2020016F060FC4FF60F3015F0D2FDFE
:1024700040F29000C0F202000F2116F055FC49F224
:10248000E460C1F6FF70BDE8084013F099B800BFE2
:1024900040F2147008B5C0F20200162116F044FC98
:1024A00049F2F823C1F6FF7393F82230CBB14DF611
:1024B000A060C2F200004FF60F7111F01FFF40F252
:1024C00078001421C0F2020016F02EFC4FF60F70B7
:1024D00015F0A0FD40F29000C0F202000F2116F0AE
:1024E00023FC49F2E460C1F6FF70BDE8084013F038
:1024F00067B800BF38B5044640F22C700D46C0F2F4
:102500000200102116F010FC49F2F823C1F6FF7307
:1025100093F82230DBB14DF6A06000232A46C2F2C8
:102520000000214611F028FF40F278001421C0F28B
:10253000020016F0F9FB29462046002215F0BEFDE8
:1025400040F29000C0F202000F2116F0EDFB49F2BC
:10255000E460C1F6FF70BDE8384013F031B800BF49
:1025600040F2407008B5C0F20200102116F0DCFB0A
:1025700049F2F823C1F6FF7393F82230CBB14DF640
:10258000A060C2F200004FF60F2111F0B7FE40F23A
:1025900078001421C0F2020016F0C6FB4FF60F209F
:1025A00015F038FD40F29000C0F202000F2116F045
:1025B000BBFB49F2E460C1F6FF70BDE8084012F0D1
:1025C000FFBF00BF40F2547008B5C0F202000F21F7
:1025D00016F0AAFB49F2F823C1F6FF7393F82230F4
:1025E000CBB14DF6A060C2F200004FF60F4111F0E2
:1025F00085FE40F278001421C0F2020016F094FB30
:102600004FF60F4015F006FD40F29000C0F20200B8
:102610000F2116F089FB49F2E460C1F6FF70BDE8B6
:10262000084012F0CDBF00BF40F2647008B5C0F2A0
:102630000200102116F078FB49F2F823C1F6FF736F
:1026400093F82230CBB14DF6A060C2F200004FF6F5
:102650000F0111F053FE40F278001421C0F2020085
:1026600016F062FB4FF60F0015F0D4FC40F290001C
:10267000C0F202000F2116F057FB49F2E460C1F6E8
:10268000FF70BDE8084012F09BBF00BF2DE9F0418C
:10269000804640F278700F46C0F20200102116F01A
:1026A00043FB49F2F823C1F6FF7393F822303BB99C
:1026B00049F2E460C1F6FF70BDE8F04112F080BF5E
:1026C0004DF6E445C1F6FF75F021A86C0368DB6C9C
:1026D000984757B1444608EB0706A86C14F8011B4D
:1026E00003681B689847A642F7D1A86C0368F721D6
:1026F000DB6C984740F2E0000F21C0F2020016F0B8
:1027000013FB4DF6A0603A464146C2F2000000239A
:1027100011F032FE40F27800C0F20200142116F0EF
:1027200003FB49F2E460C1F6FF70BDE8F04112F02E
:1027300047BF00BF40F28C7008B5C0F20200102104
:1027400016F0F2FA49F2F823C1F6FF7393F822303B
:10275000F3B14DF6E443C1F6FF73FA21986C0368B8
:102760001B68984740F2E0000F21C0F2020016F00B
:10277000DBFA4DF6A060C2F200004FF60F2111F017
:10278000BDFD40F27800C0F20200142116F0CCFA30
:1027900049F2E460C1F6FF70BDE8084012F010BFD6
:1027A00040F2A07008B5C0F202000F2116F0BCFA8A
:1027B00049F2F823C1F6FF7393F82230F3B14DF6D6
:1027C000E443C1F6FF73FC21986C03681B689847CB
:1027D00040F2E0000F21C0F2020016F0A5FA4DF61B
:1027E000A060C2F200004FF60F4111F087FD40F2E9
:1027F0007800C0F20200142116F096FA49F2E46063
:10280000C1F6FF70BDE8084012F0DABE40F2B070C9
:1028100008B5C0F20200162116F086FA49F2F82334
:10282000C1F6FF7393F82230F3B14DF6E443C1F6DD
:10283000FF73FF21986C03681B68984740F2E00023
:102840000F21C0F2020016F06FFA4DF6A060C2F23E
:1028500000004FF60F7111F051FD40F27800C0F208
:102860000200142116F060FA49F2E460C1F6FF702C
:10287000BDE8084012F0A4BE40F2C87008B5C0F22E
:102880000200182116F050FA49F2F823C1F6FF733E
:1028900093F82230F3B14DF6E443C1F6FF73FE2105
:1028A000986C03681B68984740F2E0000F21C0F263
:1028B000020016F039FA4DF6A060C2F200004FF6A1
:1028C0000F6111F01BFD40F27800C0F202001421EC
:1028D00016F02AFA49F2E460C1F6FF70BDE808403C
:1028E00012F06EBE40F2E47008B5C0F202001B2187
:1028F00016F01AFA49F2F823C1F6FF7393F8223062
:10290000D3B14DF6E443C1F6FF73F621986C03682A
:10291000DB6C984740F2E0000F21C0F2020016F095
:1029200003FA4FF20F6015F075FB40F29000C0F211
:1029300002000F2116F0F8F949F2E460C1F6FF70C9
:10294000BDE8084012F03CBE40F6000008B5C0F2F9
:102950000200102116F0E8F949F2F823C1F6FF73DE
:1029600093F82230F3B14DF6E443C1F6FF73F8213A
:10297000986C03681B68984740F2E0000F21C0F292
:10298000020016F0D1F94DF6A060C2F200004FF639
:102990000F0111F0B3FC40F27800C0F202001421E4
:1029A00016F0C2F949F2E460C1F6FF70BDE80840D4
:1029B00012F006BE40F6140008B5C0F20200132162
:1029C00016F0B2F949F2F823C1F6FF7393F82230FA
:1029D000F3B14DF6E443C1F6FF73FB21986C036835
:1029E0001B68984740F2E0000F21C0F2020016F089
:1029F0009BF94DF6A060C2F200004FF60F3111F0C6
:102A00007DFC40F27800C0F20200142116F08CF92F
:102A100049F2E460C1F6FF70BDE8084012F0D0BD95
:102A200038B5044640F62800C0F202001F2116F017
:102A30007BF949F2F823C1F6FF7393F82230FBB11A
:102A400004F00F044FF202152404C0F210052543D0
:102A50004DF6A0602946C2F2000011F04FFC40F292
:102A600078001421C0F2020016F05EF9284615F035
:102A7000D1FA40F29000C0F202000F2116F054F992
:102A800049F2E460C1F6FF70BDE8384012F098BD2D
:102A900040F6480010B51821C0F2020016F044F9C3
:102AA00049F2E460C1F6FF7012F08AFD4BF69061C6
:102AB0004DF23040C2F20001C2F200000FF02EFDD4
:102AC0004DF230400221C2F200000FF04FFD4CF2F7
:102AD000A433C2F200034DF21801C1F6FF7193F95D
:102AE000052048681870002A19DB44F2C013C2F2AE
:102AF000000303240020A2424A609C6383F83C0048
:102B00005863D4BF92000C2272B6DA6262B64DF2FC
:102B10003040C2F20000BDE810400FF04BBD44F25F
:102B2000C012C2F2000200200324946382F83C0029
:102B300050635871486072B6D06262B64DF2304050
:102B4000C2F2000001210FF00BFDE0E740F6640047
:102B500010B51C21C0F2020016F0E6F849F2E4605C
:102B6000C1F6FF7012F02CFD4CF2A4514DF2304032
:102B7000C1F6FF71C2F200000FF0D0FC4DF2304000
:102B80000221C2F200000FF0F1FC4CF2A433C2F2B9
:102B900000034DF21801C1F6FF7193F90220486855
:102BA0001870002A19DB44F2C013C2F20003082493
:102BB0000020A2424A609C6383F83C005863D4BF63
:102BC0009200202272B6DA6262B64DF23040C2F252
:102BD0000000BDE810400FF0EDBC44F2C012C2F29C
:102BE000000200200824946382F83C00506398702F
:102BF000486072B6D06262B64DF23040C2F2000058
:102C000001210FF0ADFCE0E740F6840008B5C0F20A
:102C10000200162116F088F849F2F823C1F6FF7376
:102C200093F82230F3B14DF6E443C1F6FF73F62179
:102C3000986C0368DB6C984740F2E0000F21C0F20B
:102C4000020016F071F84DF6A060C2F200004FF2DB
:102C50000F6111F053FB40F27800C0F20200142122
:102C600016F062F849F2E460C1F6FF70BDE8084072
:102C700012F0A6BC38B5054612F044FC04462846BE
:102C800012F09EFC204438BD10B44FF6DC640023E3
:102C9000C0F201044172026104600372C36041B179
:102CA000194600E0026942F82310427A01339A4241
:102CB000F8DC4FF28853C2F200031A680AB90CE03C
:102CC0001A465369002BFBD1506100234361838076
:102CD000C38083725DF8044B70471860F5E700BF4E
:102CE00010B4036841681A780C78417A037A0C4270
:102CF00002EA03021AD0837A03F003030AB143F015
:102D0000040343F008039A10082B82722AD8072B79
:102D100022D2032B2ED011D9042B13D0062B14D181
:102D2000C3685DF8044B023BC3607047837A03F0CD
:102D30000303002AE7D043F00403E4E7012B0BD0A0
:102D4000022B02D1C368013BC3605DF8044B70479E
:102D50000D2BF7D00E2BF8D1C3685DF8044B01336F
:102D6000C36070470C2B05D0F2D8092BD8D00B2BA1
:102D7000E8D0EAE7C3685DF8044B0233C3607047EC
:102D800008B54EF66443C2F20003D3F8EC00FFF737
:102D9000A7FF08BD08B54EF66443C2F20003D3F89E
:102DA000E800FFF79DFF08BD08B54EF66443C2F288
:102DB0000003D3F8E400FFF793FF08BD08B54EF613
:102DC0006443C2F20003D3F8E000FFF789FF08BDB7
:102DD00008B54EF66443C2F20003D3F8DC00FFF7F7
:102DE0007FFF08BD08B54EF66443C2F20003D3F876
:102DF000D800FFF775FF08BD08B54EF66443C2F270
:102E00000003D3F8D400FFF76BFF08BD08B54EF6FA
:102E10006443C2F20003D3F8D000FFF761FF08BD9E
:102E200008B54EF66443C2F20003D3F8CC00FFF7B6
:102E300057FF08BD08B54EF66443C2F20003D3F84D
:102E4000C800FFF74DFF08BD08B54EF66443C2F257
:102E50000003D3F8C400FFF743FF08BD08B54EF6E2
:102E60006443C2F20003D3F8C000FFF739FF08BD86
:102E700008B54EF66443C2F20003D3F8BC00FFF776
:102E80002FFF08BD08B54EF66443C2F20003D3F825
:102E9000B800FFF725FF08BD08B54EF66443C2F23F
:102EA0000003D3F8B400FFF71BFF08BD08B54EF6CA
:102EB0006443C2F20003D3F8B000FFF711FF08BD6E
:102EC00008B54EF66443C2F20003D3F8AC00FFF736
:102ED00007FF08BD08B54EF66443C2F20003D3F8FD
:102EE000A800FFF7FDFE08BD08B54EF66443C2F228
:102EF0000003D3F8A400FFF7F3FE08BD08B54EF6B3
:102F00006443C2F20003D3F8A000FFF7E9FE08BD56
:102F100008B54EF66443C2F20003D3F89C00FFF7F5
:102F2000DFFE08BD08B54EF66443C2F20003D3F8D5
:102F30009800FFF7D5FE08BD08B54EF66443C2F20F
:102F40000003D3F89400FFF7CBFE08BD08B54EF69A
:102F50006443C2F20003D3F89000FFF7C1FE08BD3E
:102F600008B54EF66443C2F20003D3F88C00FFF7B5
:102F7000B7FE08BD08B54EF66443C2F20003D3F8AD
:102F80008800FFF7ADFE08BD08B54EF66443C2F2F7
:102F90000003D3F88400FFF7A3FE08BD08B54EF682
:102FA0006443C2F20003D3F88000FFF799FE08BD26
:102FB00008B54EF66443C2F20003D86FFFF790FEE7
:102FC00008BD00BF08B54EF66443C2F20003986F17
:102FD000FFF786FE08BD00BF08B54EF66443C2F297
:102FE0000003586FFFF77CFE08BD00BF08B54EF622
:102FF0006443C2F20003186FFFF772FE08BD00BF02
:1030000008B54EF66443C2F20003D86EFFF768FEBF
:1030100008BD00BF08B54EF66443C2F20003986EC7
:10302000FFF75EFE08BD00BF08B54EF66443C2F26E
:103030000003586EFFF754FE08BD00BF08B54EF6FA
:103040006443C2F20003186EFFF74AFE08BD00BFDA
:1030500008B54EF66443C2F20003D86DFFF740FE98
:1030600008BD00BF08B54EF66443C2F20003986D78
:10307000FFF736FE08BD00BF08B54EF66443C2F246
:103080000003586DFFF72CFE08BD00BF08B54EF6D3
:103090006443C2F20003186DFFF722FE08BD00BFB3
:1030A00008B54EF66443C2F20003D86CFFF718FE71
:1030B00008BD00BF08B54EF66443C2F20003986C29
:1030C000FFF70EFE08BD00BF08B54EF66443C2F21E
:1030D0000003586CFFF704FE08BD00BF08B54EF6AC
:1030E0006443C2F20003186CFFF7FAFD08BD00BF8D
:1030F00008B54EF66443C2F20003D86BFFF7F0FD4B
:1031000008BD00BF08B54EF66443C2F20003986BD9
:10311000FFF7E6FD08BD00BF08B54EF66443C2F2F6
:103120000003586BFFF7DCFD08BD00BF08B54EF685
:103130006443C2F20003186BFFF7D2FD08BD00BF65
:1031400008B54EF66443C2F20003D86AFFF7C8FD23
:1031500008BD00BF08B54EF66443C2F20003986A8A
:10316000FFF7BEFD08BD00BF08B54EF66443C2F2CE
:103170000003586AFFF7B4FD08BD00BF08B54EF65E
:103180006443C2F20003186AFFF7AAFD08BD00BF3E
:1031900008B54EF66443C2F20003D869FFF7A0FDFC
:1031A00008BD00BF08B54EF66443C2F2000398693B
:1031B000FFF796FD08BD00BF08B54EF66443C2F2A6
:1031C00000035869FFF78CFD08BD00BF08B54EF637
:1031D0006443C2F200031869FFF782FD08BD00BF17
:1031E00008B54EF66443C2F20003D868FFF778FDD5
:1031F00008BD00BF08B54EF66443C2F200039868EC
:10320000FFF76EFD08BD00BF08B54EF66443C2F27D
:1032100000035868FFF764FD08BD00BF08B54EF60F
:103220006443C2F200031868FFF75AFD08BD00BFEF
:103230001D2810B50B4600F0E983024622D92C2840
:1032400000F064813FD8242800F0EE8340F2A8808B
:10325000282800F0748300F2D680262800F0F5813B
:1032600040F2D5824EF66444C2F2000442F6117177
:10327000C0F2000104222720C4F89C3012F008FF9D
:10328000012010BD0E2800F097833AD8062800F0E0
:10329000A1836CD90A2800F0058300F20781082871
:1032A00000F07E8140F275824EF66444C2F2000462
:1032B00043F26911C0F2000104220920636212F096
:1032C000E7FE012010BD342800F0BD8336D8302839
:1032D00000F0638300F2D6802E2800F0528140F285
:1032E00001824EF66444C2F2000442F67161C0F2FB
:1032F000000104222F20C4F8BC3012F0C9FE0120C6
:1033000010BD152800F0748364D9192800F0FA81E3
:1033100000F2A580172800F08A8140F2D1824EF693
:103320006444C2F2000443F23D01C0F200010422F1
:103330001820236612F0ACFE012010BD382800F0E2
:10334000CE8275D8362800F0398140F27F824EF661
:103350006444C2F2000442F6D151C0F200010422DA
:103360003720C4F8DC3012F093FE012010BD022893
:1033700000F0018240F27881042800F04B8140F295
:10338000BD824EF66444C2F2000443F2B911C0F2A9
:10339000000104220520636112F07AFE012010BDB5
:1033A000202800F0448240F28981222800F0238105
:1033B00040F2D4824EF66444C2F2000442F66171D7
:1033C000C0F2000104222320C4F88C3012F060FE09
:1033D000012010BD112800F0B18140F25A8113285C
:1033E00000F0FB8040F2B8814EF66444C2F2000463
:1033F00043F28D01C0F2000104221420236512F073
:1034000047FE012010BD2A2800F0AC8040F2E08188
:103410004EF66444C2F2000442F6C161C0F20001FB
:1034200004222B20C4F8AC3012F032FE012010BD73
:103430003A2800F08880C0F072823B2840F06D820C
:103440004EF66444C2F2000442F68151C0F200011B
:103450000422C4F8EC3012F01BFE012010BD1B2822
:1034600063D040F28B824EF66444C2F2000442F60E
:10347000ED71C0F2000104221C20236712F008FE47
:10348000012010BD322824D040F292814EF66444CF
:10349000C2F2000442F62161C0F20001042233208E
:1034A000C4F8CC3012F0F4FD012010BD0C281FD060
:1034B00040F29E814EF66444C2F2000443F21911B8
:1034C000C0F2000104220D20636312F0E1FD01202F
:1034D00010BD4EF66444C2F2000442F63561C0F2FB
:1034E00000010422C4F8C83012F0D2FD012010BD42
:1034F0004EF66444C2F2000443F22D11C0F2000102
:103500000422236312F0C4FD012010BD4EF6644472
:10351000C2F2000442F6AD61C0F200010422C4F818
:10352000B03012F0B5FD012010BD4EF66444C2F279
:10353000000443F20101C0F200010422E36612F02C
:10354000A7FD012010BD4EF66444C2F2000442F60D
:103550009551C0F200010422C4F8E83012F098FD41
:10356000012010BD4EF66444C2F2000442F6D5615B
:10357000C0F200010422C4F8A83012F089FD012035
:1035800010BD4EF66444C2F2000442F68561C0F2FA
:1035900000010422C4F8B83012F07AFD012010BDF9
:1035A0004EF66444C2F2000443F27D11C0F2000101
:1035B0000422236212F06CFD012010BD4EF664441B
:1035C000C2F2000442F6E551C0F200010422C4F840
:1035D000D83012F05DFD012010BD4EF66444C2F2F9
:1035E000000443F2A101C0F200010422E36412F0DE
:1035F0004FFD012010BD4EF66444C2F2000442F6B5
:103600007571C0F200010422C4F8883012F040FD48
:10361000012010BD4EF66444C2F2000443F2CD1105
:10362000C0F20001236112F033FD012010BD4EF6FF
:103630006444C2F2000443F25101C0F200010422CA
:10364000E36512F025FD012010BD4EF66444C2F280
:10365000000442F62571C0F200010422C4F898303B
:1036600012F016FD012010BD002800F0FF80012897
:1036700040F053814EF66444C2F2000443F2092143
:10368000C0F2000104220120636012F001FD01205C
:1036900010BD0F2800F0F880102840F03E814EF653
:1036A0006444C2F2000443F2DD01C0F200010422CE
:1036B0001020236412F0ECFC012010BD1E282FD036
:1036C0001F2840F02A814EF66444C2F2000442F6FC
:1036D000B171C0F2000104221F20E36712F0D8FC90
:1036E000012010BD4EF66444C2F2000442F6996116
:1036F000C0F2000104222D20C4F8B43012F0C8FC3E
:10370000012010BD4EF66444C2F2000443F22901C8
:10371000C0F200010422636612F0BAFC012010BD61
:103720004EF66444C2F2000442F6C571C0F20001D4
:103730000422A36712F0ACFC012010BD4EF66444D5
:10374000C2F2000443F2C901C0F200010422636422
:1037500012F09EFC012010BD4EF66444C2F200043B
:1037600043F2B501C0F2000104221220A36412F05A
:103770008FFC012010BD4EF66444C2F2000443F2F7
:10378000F511C0F200010422A36012F081FC0120B7
:1037900010BD4EF66444C2F2000443F29111C0F22F
:1037A000000104220720E36112F072FC012010BD29
:1037B0004EF66444C2F2000442F64961C0F20001D0
:1037C00004223120C4F8C43012F062FC012010BD84
:1037D0004EF66444C2F2000442F6E961C0F2000110
:1037E00004222920C4F8A43012F052FC012010BD9C
:1037F0004EF66444C2F2000443F24111C0F20001EB
:1038000004220B20E36212F043FC012010BD4EF6AF
:103810006444C2F2000442F63971C0F2000104228D
:103820002520C4F8943012F033FC012010BD4EF670
:103830006444C2F2000442F69D71C0F20001042209
:10384000C4F8803012F024FC012010BD4EF6644410
:10385000C2F2000442F6F951C0F200010422352000
:10386000C4F8D43012F014FC012010BD4EF66444AC
:10387000C2F2000443F21D21C0F2000104222360C1
:1038800012F006FC012010BD4EF66444C2F20004A2
:1038900043F2F101C0F200010422E36312F0F8FBED
:1038A000012010BD4EF66444C2F2000443F25511EB
:1038B000C0F200010422A36212F0EAFB012010BD55
:1038C0004EF66444C2F2000443F26501C0F2000106
:1038D00004221620A36512F0DBFB012010BD4EF67A
:1038E0006444C2F2000442F6BD51C0F20001042259
:1038F000C4F8E03012F0CCFB012010BD4EF6644459
:10390000C2F2000443F2E111C0F2000104220320DC
:10391000E36012F0BDFB012010BD002010BD4EF68B
:103920006444C2F2000442F6A951C0F2000104222C
:103930003920C4F8E43012F0ABFB012010BD4EF684
:103940006444C2F2000442F6FD61C0F200010422A8
:10395000C4F8A03012F09CFB012010BD4EF6644468
:10396000C2F2000442F68971C0F200010422212053
:10397000C4F8843012F08CFB012010BD4EF6644474
:10398000C2F2000443F21501C0F2000104221A2021
:10399000A36612F07DFB012010BD4EF66444C2F216
:1039A000000442F65D61C0F200010422C4F8C03098
:1039B00012F06EFB012010BD4EF66444C2F200040A
:1039C00043F20511C0F200010422A36312F060FB70
:1039D000012010BD4EF66444C2F2000443F2A5116A
:1039E000C0F200010422A36112F052FB012010BDBD
:1039F0004EF66444C2F2000443F27901C0F20001C1
:103A00000422636512F044FB012010BD4EF66444AD
:103A1000C2F2000442F6D971C0F2000104226367C9
:103A200012F036FB012010BD4EF66444C2F20004D1
:103A300042F64D71C0F200010422C4F8903012F039
:103A400027FB012010BD4EF66444C2F2000442F68A
:103A50000D61C0F200010422C4F8D03012F018FB4E
:103A6000012010BDF8B5044615460E460846022151
:103A700012F086FD2846022112F082FD4FF6CC732B
:103A8000C0F20E03012253F83600227200F50071D5
:103A9000216053F8351062724DF2C04301F5007792
:103AA00062F31F4300226760E260013BFDD190F8A2
:103AB000003291F8002203F00103D20744BF43F023
:103AC0000203DBB2A37221463046FFF7B1FB214669
:103AD00020742846FFF7ACFB237C18442074204652
:103AE000F8BD00BF10B5037C012B04462CD972B67B
:103AF000E36862B6002BB8BF033362699B10934240
:103B00000DDBA1698B4217DC237C012B20D972B617
:103B1000E06862B60028B8BF0330801010BD237F74
:103B200023B972B69200E26062B6EDE7A3699B002A
:103B300072B6E36062B6E7E7237F002BF1D172B67D
:103B40008900E16062B6DFE772B6FFF7C9F8CFE738
:103B500072B62046FFF7C4F8DAE700BF091A49B287
:103B600038B581EAE175A5EBE175D5B100294FF0D3
:103B700000040BDB4DF230400134C2F200000021A2
:103B8000E4B20EF0EDFCAC42F4DB38BD4DF2304057
:103B90000134C2F200000121E4B20EF0E1FCAC42BB
:103BA000F4DB38BDF8B544F2C014C2F20004074695
:103BB00004F12000FFF796FF4CF2A435C2F2000595
:103BC0004DF23046C2F200064BF6FC21E855C2F237
:103BD000000130460EF0A2FC304602210EF0C6FC79
:103BE0004DF2180295F90030C1F6FF720021052050
:103BF0005360A06323EAE37384F83C10616372B6F8
:103C00008342A8BF03469B00E36262B6F8BD00BFD3
:103C1000F8B544F2C014C2F20004074604F12000D3
:103C2000FFF760FF4CF2A435C2F200054DF23046BA
:103C3000C2F200064CF2A451E855C1F6FF713046BD
:103C40000EF06CFC304602210EF090FC4DF2180292
:103C500095F90230C1F6FF72002108205360A0637D
:103C600023EAE37384F83C10616372B68342A8BF11
:103C700003469B00E36262B6F8BD00BFF8B544F2AC
:103C8000C014C2F20004074604F12000FFF72AFF27
:103C90004CF2A435C2F200054DF23046C2F20006E5
:103CA0004EF2B871E855C2F2000130460EF036FC13
:103CB000304602210EF05AFC4DF2180295F90330FD
:103CC000C1F6FF72002112205360A06323EAE37360
:103CD00084F83C10616372B68342A8BF03469B0020
:103CE000E36262B6F8BD00BFF8B544F2C014C2F298
:103CF0000004074604F12000FFF7F4FE4CF2A4355F
:103D0000C2F200054DF23046C2F200064BF6906159
:103D1000E855C2F2000130460EF000FC30460221A8
:103D20000EF024FC4DF2180295F90530C1F6FF7231
:103D3000002103205360A06323EAE37384F83C105E
:103D4000616372B68342A8BF03469B00E36262B61A
:103D5000F8BD00BF38B549F240330546C1F6FF73E0
:103D600040F69C0049F2E464C1F6FF740B21C0F2F6
:103D700002001D7014F0D8FF2946204600230A22B5
:103D800011F030FC2046BDE8384011F019BC00BFEE
:103D900038B5054649F2E46440F6A8000B21C1F6A7
:103DA000FF74C0F2020014F0BFFF002329460A226C
:103DB000204611F017FC204611F002FC4BF684134C
:103DC000C1F6FF731D7038BD38B5054649F2E4648D
:103DD00040F6B4000A21C1F6FF74C0F2020014F0EC
:103DE000A3FF294600230A22204611F0FBFB2046B0
:103DF00011F0E6FB07EE905A0023C4F2C623F8EE5A
:103E0000676A07EE103A86EE870A002307EE903ABB
:103E10004BF21C23C2F2000330EE270A186807F0A9
:103E200033FB49F2F823C1F6FF731D7138BD00BFA3
:103E300038B5054649F2E46440F6C0000C21C1F6ED
:103E4000FF74C0F2020014F06FFF294600230A221B
:103E5000204611F0C7FB204611F0B2FB07EE905A46
:103E60000023C4F2C623F8EE676A07EE103A86EE26
:103E7000870A002307EE903A4BF21C23C2F200039C
:103E800030EE270A186807F0EBFB49F2F823C1F679
:103E9000FF735D7138BD00BF38B5054649F2E46473
:103EA00040F6D0000D21C1F6FF74C0F2020014F0FC
:103EB0003BFF294600230A22204611F093FB2046AF
:103EC00011F07EFB07EE905A0023C4F2C623F8EEF1
:103ED000676A07EE103A86EE870A002307EE903AEB
:103EE0004BF21C23C2F2000330EE270A186807F0D9
:103EF000A3FC49F2F823C1F6FF739D7138BD00BFE2
:103F000038B5054649F2E46440F6E0000B21C1F6FD
:103F1000FF74C0F2020014F007FF294600230A22B2
:103F2000204611F05FFB204611F04AFB07EE905A45
:103F30000023C4F2C623F8EE676A07EE103A86EE55
:103F4000870A002307EE903A4BF21C23C2F20003CB
:103F500030EE270A186807F059FD49F2F823C1F638
:103F6000FF73DD7138BD00BF38B5054649F2E46422
:103F700040F6EC000B21C1F6FF74C0F2020014F011
:103F8000D3FE2946204611F0BDFA204611F018FB59
:103F900007EE905A0023C4F2C623F8EEE76A07EE54
:103FA000103A86EE870A002307EE903A4BF21C2364
:103FB000C2F2000330EE270A186808F0D5F849F27B
:103FC000F823C1F6FF731D7238BD00BF38B5054632
:103FD00049F2E46440F6F8000E21C1F6FF74C0F225
:103FE000020014F0A1FE2946204611F08BFA20466B
:103FF00011F0E6FA49F2F823C1F6FF735D7238BD9D
:1040000038B5054649F2E46440F608100921C1F6C6
:10401000FF74C0F2020014F087FE2946204611F01A
:1040200071FA204611F0CCFA07EE905A0023C4F240
:10403000482306EE103AF8EEE77A0023C4F2C823CC
:1040400006EE903A77EE867A002387EEA60A07EE10
:10405000103A4BF21C23C2F2000330EE070A186834
:1040600008F070F949F2F823C1F6FF739D7238BD6C
:1040700038B5054649F2E46440F614100B21C1F648
:10408000FF74C0F2020014F04FFE294600230A22FA
:10409000204611F0A7FA204611F092FA07EE905A46
:1040A0000023C4F2C623F8EE676A07EE103A86EEE4
:1040B000870A002307EE903A4BF21C23C2F200035A
:1040C00030EE270A186808F029FA49F2F823C1F6F9
:1040D000FF73DD7238BD00BF38B5054649F2E464B0
:1040E00040F620101321C1F6FF74C0F2020014F054
:1040F0001BFE294600230A22204611F073FA2046AF
:1041000011F05EFA07EE905A0023C4F2C623F8EECF
:10411000676A07EE103A86EE870A002307EE903AA8
:104120004BF21C23C2F2000330EE270A186807F096
:104130002FFF49F2F823C1F6FF731D7338BD00BF8E
:1041400038B5054649F2E46440F634101621C1F64C
:10415000FF74C0F2020014F0E7FD294600230A2292
:10416000204611F03FFA204611F02AFA07EE905A45
:104170000023C4F2C623F8EE676A07EE103A86EE13
:10418000870A002307EE903A4BF21C23C2F2000389
:1041900030EE270A186807F00FFE49F2F823C1F63F
:1041A000FF735D7338BD00BF38B5054649F2E4645E
:1041B00040F64C101321C1F6FF74C0F2020014F057
:1041C000B3FD294600230A22204611F00BFA2046AF
:1041D00011F0F6F907EE905A0023C4F2C623F8EE68
:1041E000676A07EE103A86EE870A002307EE903AD8
:1041F0004BF21C23C2F2000330EE270A186807F0C6
:10420000EFFC49F2F823C1F6FF739D7338BD00BF80
:1042100038B5054649F2E46440F660100E21C1F657
:10422000FF74C0F2020014F07FFD294600230A2229
:10423000204611F0D7F9204611F0C2F907EE905A46
:104240000023C4F2C623F8EE676A07EE103A86EE42
:10425000870A002307EE903A4BF21C23C2F20003B8
:1042600030EE270A186808F045FA49F2F823C1F63B
:10427000FF73DD7338BD00BF30B5054649F2E46415
:1042800040F6701083B0C1F6FF740E21C0F2020038
:1042900014F04AFD294600230A22204611F0A2F913
:1042A000204611F08DF949F2F82407EE905AC1F634
:1042B000FF740023F8EE676A07EE903AB6EE007AD4
:1042C000637D627CE6EE877A44F20020C2F2000051
:1042D00001EE103A237D00EE903AFCEEE77AB8EE5C
:1042E000411AF8EE600ACDED017AF2EE047A81EE21
:1042F000271AE37C9DF80410C0EEA70A00EE103ADE
:10430000A37CB8EE400A09F057FD257403B030BD18
:1043100030B5054649F2E46440F6801083B0C1F63A
:10432000FF741221C0F2020014F0FEFC29460023A3
:104330000A22204611F056F9204611F041F907EE05
:10434000905AF8EE676AB0EE087AC6EE877A49F2BC
:10435000F824C1F6FF740022637D217C44F2002022
:10436000C2F2000007EE102A01EE103A237D77EE2C
:10437000877A00EE903AFCEEE77AB8EE411AF8EE52
:10438000600ACDED017AF2EE047A81EE271AE37C21
:104390009DF80420C0EEA70A00EE103AA37CB8EE08
:1043A000400A09F009FD657403B030BD30B505461B
:1043B00049F2E46440F6941083B0C1F6FF740F2113
:1043C000C0F2020014F0B0FC294600230A22204665
:1043D00011F008F9204649F2F824C1F6FF7411F0F3
:1043E000EFF807EE905A002307EE103A637D627CE7
:1043F000217CF8EE677A01EE103A237D77EE877A1A
:1044000000EE903AFCEEE77AB8EE411AF8EE600A58
:10441000CDED017AF2EE047A81EE271AE37C44F2C4
:104420000020C2F20000C0EEA70A00EE103A9DF88C
:104430000430B8EE400A09F0BFFC003518BF012572
:10444000A57403B030BD00BF70B5064649F2E465FF
:1044500040F6A4101321C1F6FF75C0F2020049F224
:10446000F82414F061FCC1F6FF74314600230A22DF
:10447000284611F0B7F8284611F0A2F8637D627C57
:10448000217C01EE103A237D00EE903AB8EE411AFD
:10449000F8EE600AF2EE047A81EE271A44F2002068
:1044A000A37CC2F20000C0EEA70A07EE906AB8EE45
:1044B000670A09F081FCE67470BD00BF70B506465E
:1044C00049F2E46540F6B8101021C1F6FF75C0F25C
:1044D000020049F2F82414F027FCC1F6FF743146BB
:1044E00000230A22284611F07DF8284611F068F8CA
:1044F000637D627C217C01EE103A07EE906AE37CDA
:10450000F8EE670A00EE103AB8EE411AF2EE047ABD
:1045100044F20020A37C81EE271AC2F20000C0EE14
:10452000A70AB8EE400A09F047FC267570BD00BF27
:1045300070B5064649F2E46540F6CC100F21C1F68D
:10454000FF75C0F2020049F2F82414F0EDFBC1F649
:10455000FF74314600230A22284611F043F828460A
:1045600011F02EF8237D627C217C00EE903A07EE5C
:10457000906AE37CB8EE671A00EE103AF8EE600A33
:10458000F2EE047A44F20020A37CC0EEA70AC2F245
:10459000000081EE271AB8EE400A09F00DFC66759E
:1045A00070BD00BF10B5044640F6DC101421C0F207
:1045B000020014F0B9FB49F2E460002321460A220C
:1045C000C1F6FF7011F00EF849F2E460C1F6FF7019
:1045D00010F0F6FF07EE904A0023C4F2C62307EE60
:1045E000103AB8EE676A0023C6EE077A06EE903AF4
:1045F00077EEA67AB7EE007AF4EEC77AF1EE10FA0B
:1046000015DD44F20C22C2F2000245F2606147F669
:104610007053535249F2F8224DF62071C1F6FF72E1
:10462000C1F6FF7145F2606094750B5210BDF4EE57
:10463000E67AF1EE10FA33D445F62943C4F20F635B
:1046400007EE103A27EE877ABDEEC77A17EE103ADA
:1046500003F5B34319331BB244F20C22B7EE007AD0
:10466000C2F2000245F26061F4EEC77AF1EE10FA90
:1046700053521BDCF5EEC07AF1EE10FA13D445F676
:104680002943C4F20F6307EE103A67EE877AFDEE16
:10469000E77A17EE903A03F5B34319331BB2B9E743
:1046A00045F69913D8E745F69913B3E747F67053E3
:1046B000B0E700BF38B5044640F6F4101321C0F24D
:1046C000020014F031FB49F2E460002321460A2283
:1046D000C1F6FF7010F086FF49F2E460C1F6FF708A
:1046E00010F06EFF07EE904A0023C4F2C62307EED7
:1046F000103AB8EE676A0023C6EE077A06EE903AE3
:1047000077EEA67AB7EE007AF4EEC77AF1EE10FAF9
:1047100042DD44F6CD4143F2333272B644F20C230B
:10472000C2F2000345F25C6545F25E605A531952CD
:1047300062B6B7EE007AF4EEC77AF1EE10FA15DD44
:1047400044F6CD4143F2333372B64DF62072C1F6D2
:10475000FF7245F25C6545F25E605353115262B6DA
:1047600049F2F823C1F6FF73DC7538BDF5EEC07A67
:10477000F1EE10FA2CD44CF6CD43C4F24C6307EEA4
:10478000103A67EE877AFDEEE77A17EE903AC3F5B6
:10479000004109B21BB2D7E7F4EEE67AF1EE10FA67
:1047A00010D44CF6CD43C4F24C6307EE103A27EE1A
:1047B000877ABDEEC77A17EE102AC2F5004109B21A
:1047C00012B2AAE74FF40041CFF6FF710022A4E72E
:1047D0004FF40041CFF6FF710023B5E710B5044652
:1047E00040F608201121C0F2020014F09DFA49F2AF
:1047F000E460214600230A22C1F6FF7010F0F2FEA9
:1048000049F2E460C1F6FF7010F0DAFE07EE904A5C
:104810000023C4F2C62306EE103AF8EE675A0023CE
:10482000C5EE867A4DF668124DF6A001C2F200027E
:10483000C2F2000106EE903A4FF47E43C4F2FF63E9
:1048400007EE103A77EEA67A4FF48033F4EEC77A8B
:10485000F1EE10FA93618B612BDC4FF47E43CCF2C6
:10486000FF6307EE103AF4EEC77AF1EE10FA2BD49C
:10487000B0EE677ABEEEC87A17EE103A4FF47E407B
:10488000C4F2FF6007EE100AF4EEC77AF1EE10FAF8
:10489000D36124DC4FF47E43CCF2FF6307EE103A81
:1048A000F4EEC77AF1EE10FA12D50023C8F2010334
:1048B00003E00023C7F6FF73D36149F2F822C1F683
:1048C000FF72CB61147610BD0023C8F20103D5E757
:1048D000B0EE677ABEEEC87A17EE103AEDE7002325
:1048E000C7F6FF73E9E700BF38B5054649F2E4644F
:1048F00040F61C201521C1F6FF74C0F2020014F02E
:1049000013FA002329460A22204610F06BFE2046A7
:1049100010F056FE49F2F823C1F6FF735D7638BDFC
:1049200038B5054649F2E46440F634201121C1F659
:10493000FF74C0F2020014F0F7F9002329460A229E
:10494000204610F04FFE204610F03AFE49F2F823C0
:10495000C1F6FF739D7638BD38B5054649F2E4646B
:1049600040F648201121C1F6FF74C0F2020014F095
:10497000DBF9002329460A22204610F033FE2046A8
:1049800010F01EFE49F2F823C1F6FF73DD7638BD44
:1049900070B5064649F2E46540F65C201221C1F686
:1049A000FF75C0F2020049F2F82414F0BDF9C1F617
:1049B000FF74314600230A22284610F013FE2846D1
:1049C00010F0FEFD637F06EE106A07EE903A0023BA
:1049D000C4F2C62306EE903AF8EE677AB8EE466A5D
:1049E000C7EEA60A002344F20020C2F2000086EEC1
:1049F000260A07EE103A70EE870A30EE070A08F032
:104A00004FFD267770BD00BF70B5064649F2E465DC
:104A100040F670201421C1F6FF75C0F2020049F281
:104A2000F82414F081F9C1F6FF74314600230A22FC
:104A3000284610F0D7FD284610F0C2FD237F06EE71
:104A4000106A07EE903A0023C4F2C62306EE903AAD
:104A5000F8EE677AB8EE466A87EEA60A002344F2BB
:104A60000020C2F20000C6EE260A07EE103A30EE31
:104A7000070A70EE870A08F013FD667770BD00BF65
:104A800070B5064649F2E46540F688200C21C1F66F
:104A9000FF75C0F2020049F2F82414F045F9C1F69E
:104AA000FF74314600230A22284610F09BFD284659
:104AB00010F086FD94F91F3007EE106A07EE903A69
:104AC0000023C4F2482306EE103AF8EEE77AB8EE77
:104AD000477A77EE867A37EE067A0023C4F2C82347
:104AE00006EE903A77EEA77A37EE077AC7EEA60A77
:104AF00044F20020C2F2000087EE260AF7EE007AA8
:104B000070EEE70A30EE670A08F0FEFDA67770BD8A
:104B100070B5064649F2E46540F698200E21C1F6CC
:104B2000FF75C0F2020049F2F82414F0FDF8C1F656
:104B3000FF74314600230A22284610F053FD284610
:104B400010F03EFD94F91E3007EE106A07EE903A21
:104B50000023C4F2482306EE103AF8EEE77AB8EEE6
:104B6000477A77EE867A37EE067A0023C4F2C823B6
:104B700006EE903A77EEA77A37EE077A87EEA60A26
:104B800044F20020C2F20000C7EE260AF7EE007AD7
:104B900030EE670A70EEE70A08F0B6FDE67770BD02
:104BA00038B5054649F2E46440F6A8200D21C1F667
:104BB000FF74C0F2020014F0B7F800230A2229465D
:104BC000204610F00FFD204610F0FAFC07EE905A38
:104BD0000023C4F2C62306EE903AB8EE676A0023BB
:104BE000C6EE267A49F2F822C1F6FF7282F820500A
:104BF00007EE103A4BF2BC0377EE877AC1F6FF73EB
:104C0000C3ED007A38BD00BF38B5054649F2E4640B
:104C100040F6B8201121C1F6FF74C0F2020014F072
:104C200083F8002329460A22204610F0DBFC2046A8
:104C300010F0C6FC49F2F823C1F6FF7383F8215047
:104C400038BD00BF38B5044649F2E46540F6CC20D3
:104C50001321C1F6FF75C0F2020014F065F8214679
:104C600000230A22284610F0BDFC284610F0A8FCBC
:104C700049F2F8230034C1F6FF7318BF012483F80A
:104C8000224038BD70B5064649F2E46540F6E020A2
:104C9000C1F6FF750D21C0F202004BF21C2414F086
:104CA00043F8C2F20004314600230A22284610F0DD
:104CB00099FC284610F084FC2068314607F040FB40
:104CC00049F2F823C1F6FF73206883F82360BDE83A
:104CD000704006F0E7B800BF2DE9F04149F2F82432
:104CE000C1F6FF74002394F80480C4F2C62340F692
:104CF000B4002DED028BC0F2020008EE903A0023C2
:104D000008EE103AFBF7E0FC4046FBF7CBFC07EE61
:104D1000908AF8EE677A4BF21C2587EEA80AC2F259
:104D2000000549F2E4662868C1F6FF7630EE080A0D
:104D300006F0AAFB677984F8048040F6C000C0F250
:104D40000200FBF7C1FC3846FBF7ACFC07EE907A9B
:104D5000F8EE677A286887EEA80A30EE080A06F0AF
:104D60007FFC94F80680677140F6D000C0F2020024
:104D7000FBF7AAFC4046FBF795FC07EE908AF8EE9D
:104D8000677A286887EEA80A30EE080A06F054FD14
:104D9000E77984F8068040F6E000C0F20200FBF7F5
:104DA00093FC3846FBF77EFC07EE907AF8EE677AC4
:104DB000286887EEA80A30EE080A06F027FE94F964
:104DC0000880E77140F6EC000B21C0F2020013F0FE
:104DD000ABFF4146304610F095FB304610F0F0FB3B
:104DE00007EE908AF8EEE77A286887EEA80A30EE98
:104DF000080A07F0B9F994F90A7084F8088040F6B7
:104E000008100921C0F2020013F08EFF3946304627
:104E100010F078FB304610F0D3FB07EE907A0023B9
:104E2000C4F2482306EE903AF8EEE77A0023C4F283
:104E3000C82377EEA67A07EE103A87EE870A28682D
:104E400030EE080A07F07EFAE67AA77240F61410F0
:104E5000C0F20200FBF738FC3046FBF723FC07EEFC
:104E6000906AF8EE677A286887EEA80A30EE080A9A
:104E700007F054FB277BE67240F62010C0F20200D8
:104E8000FBF722FC3846FBF70DFC07EE907AF8EEB4
:104E9000677A286887EEA80A30EE080A07F078F8E3
:104EA000667B277340F63410C0F20200FBF70CFC5F
:104EB0003046FBF7F7FB07EE906AF8EE677A286852
:104EC00087EEA80A30EE080A06F076FFA77B667325
:104ED00040F64C10C0F20200FBF7F6FB3846FBF739
:104EE000E1FB07EE907AF8EE677A286887EEA80A69
:104EF00030EE080A06F074FEE67BA77340F66010F9
:104F0000C0F20200FBF7E0FB3046FBF7CBFB07EEFD
:104F1000906AF8EE677A286887EEA80A30EE080AE9
:104F200007F0E8FB207CE673FFF7A6F9607CFFF74B
:104F3000EFF9A07CFFF73AFAE07CFFF785FA207DD5
:104F4000FFF7BCFA607DFFF7F3FAA07DFFF72AFBBD
:104F5000E07DFFF7AFFB207EFFF740FC667E40F66A
:104F60001C20C0F20200FBF7AFFB3046FBF79AFBB8
:104F7000A77E667640F63420C0F20200FBF7A4FB61
:104F80003846FBF78FFBE67EA77640F64820C0F256
:104F90000200FBF799FB3046FBF784FB207FE676A7
:104FA000FFF7F6FC607FFFF72FFDA07FFFF768FD9E
:104FB000E07FFFF7ADFD94F8206040F6A820C0F236
:104FC0000200FBF781FB3046FBF76CFB07EE906AB3
:104FD000B8EE677A94F8218084F82060C7EE287ACA
:104FE0004BF2BC0340F6B820C1F6FF73C0F20200DA
:104FF00037EE888A83ED008AFBF766FB4046FBF7B5
:1050000051FB94F8227084F8218040F6CC20C0F245
:105010000200FBF759FB3846FBF744FB94F823608A
:1050200084F8227040F6E020C0F20200FBF74CFB4F
:105030003046FBF737FB2868314607F081F9BDECB5
:10504000028B286884F82360BDE8F04105F02ABF90
:10505000F8B54DF6E444C1F6FF7447F61221A06C92
:105060000368DB69984740F6D95540F6315140F660
:1050700081620326C0F20005C0F20001C0F2000206
:1050800040F6850084F8646065602160E260C0F2EB
:10509000000040F6013340F60D0742F2F54642F6B5
:1050A000212540F6FD0142F2B9226061C0F2000301
:1050B000C0F20007C0F20006C0F20005C0F2000115
:1050C000C0F2000242F26100A3612761E66125623D
:1050D000A160A262C0F2000042F2296342F261576D
:1050E00042F22D4642F2C55542F2C93142F2914296
:1050F000C0F20001C0F20002E062C0F20003C0F2A0
:105100000007C0F20006C0F2000540F6F02021645E
:1051100062642363676300234FF6FF77A663E5634A
:10512000C0F2020084F84C3084F84E3084F84D30E0
:10513000A365636584F8E93084F8663084F86530E7
:1051400084F8673084F86830E7652766FBF7C6FAAD
:105150000DF0A4FA4DF6A063C2F2000346F66D749A
:1051600047F2D50147F23D22C0F20004C0F200012F
:10517000C0F2000247F29D30C3F86841C3F86411E1
:10518000C3F87021C0F2000047F2A54747F2DD5690
:1051900042F2293540F6092447F2E56140F69112C2
:1051A000C3F87801C0F20007C0F20006C0F20005A3
:1051B000C0F20004C0F20001C0F2000242F6E500B5
:1051C000C3F87C71C3F87461C3F88451C3F8884193
:1051D000C3F86C11C3F89021C0F2000042F25527C9
:1051E00042F2291642F2F11541F6FD7442F28D1198
:1051F00042F2C502C0F20001C0F20002C3F89401FD
:10520000C0F20007C0F20006C0F20005C0F20004C0
:1052100040F60830C3F89871C3F89C61C3F8A051F8
:10522000C3F8A441C3F8A811C3F8AC21C0F202002E
:10523000FBF754FA4FF65803C2F2000347F21D0E73
:10524000C0F2000E4FF65007C3F800E0C2F20007AC
:1052500047F2851EC0F2000E4FF65404C7F800E076
:10526000C2F2000447F2E92EC0F2000E4FF6280603
:10527000C4F800E0C2F2000647F21D4EC0F2000E74
:105280004FF61802C6F800E0C2F2000247F23D5E97
:10529000C0F2000E4FF61400C2F800E0C2F20000A7
:1052A00047F25D6EC0F2000E4FF63805C0F800E020
:1052B000C2F2000542F28D6EC0F2000E4FF63001D0
:1052C000C5F800E0C2F2000140F6893EC0F2000ECF
:1052D0004FF62403C1F800E0C2F2000347F26D7EEE
:1052E000C0F2000E4FF64C07C3F800E0C2F2000710
:1052F00040F6812EC0F2000E4FF63404C2F20004D4
:10530000C7F800E042F60947C0F200074FF2FC760A
:10531000C2F2000627604FF62C0242F64917C2F28D
:105320000002C0F200074FF60C0042F23574C2F2E0
:105330000000C0F2000437604FF644054FF6040148
:105340004FF6000342F6B517C2F20005C2F20003A1
:10535000C0F200071460C2F2000142F2A17642F6E8
:10536000790442F60D02C0F20006C0F200040760A4
:10537000C0F2000240F628302E600C601A60C0F2C5
:105380000200BDE8F840FBF7A9B900BFFFFFFFFF2F
:1053900070B54BF20352C0EB8023CAF27E5282FBFF
:1053A00003122DED048B1A44DB17C3EBA21349F251
:1053B000F8249A1C0546C1F6FF7440F6443082B0CA
:1053C00003FB02F300261421C0F2020008EE103A9B
:1053D00084F8246013F0A8FC49F2E4600A22334602
:1053E0002946C1F6FF7010F0FDF8BAEEC68A40F605
:1053F0005C300121C0F2020013F096FC18EE100A96
:1054000016F0D6F841EC100B49F2E4600321C1F626
:10541000FF7010F027F940F660300621C0F202005C
:1054200013F082FC49F2E46094F92410C1F6FF7095
:1054300010F068F840F65C300121C0F2020013F071
:1054400073FC49F2E4609FED560B0321C1F6FF7037
:1054500010F008F940F668300221C0F2020013F0A3
:1054600063FC40F2F343C3F6357307EE903A28EE3F
:10547000278A18EE100A16F09BF841EC190B49F236
:10548000E460B0EE490AF0EE690A0321C1F6FF704C
:1054900010F0E8F840F66C300121C0F2020013F081
:1054A00043FCB0EE490AF0EE690A49F2E4600321D8
:1054B000C1F6FF7010F0D6F849F2E460C1F6FF7053
:1054C00010F07EF84FF47E43C4F2FF6307EE903A8B
:1054D000B4EEE78AF1EE10FA2FDC4FF47E43CCF203
:1054E000FF6307EE903AB4EEE78AF1EE10FA47D484
:1054F000F0EE487AFEEEC87A17EE902A4FF47E411D
:10550000C4F2FF6107EE901A4DF66813C2F2000371
:10551000B4EEE78AF1EE10FA9A613CDC4FF47E4378
:10552000CCF2FF6307EE903AB4EEE78AF1EE10FAA0
:105530002AD50023C8F2010307E04DF66812C2F233
:1055400000020023C7F6FF7393614FF23462C2F288
:1055500000024EF6F40012680192C2F200004DF60D
:10556000A0014DF29C72C2F20001C2F20002019C45
:10557000046001208B61107002B0BDEC048B70BD23
:105580000022C8F20102B9E7F0EE487AFEEEC87ACE
:1055900017EE903AD9E70023C7F6FF73D5E700BFAF
:1055A000000000000000E03F2DE9F0414FF23466BA
:1055B000C2F2000682B04DF6982533680093C1F61A
:1055C000FF75009B2A689B1AB3F5487F00F243825F
:1055D0004DF21804C1F6FF744EF28050C2F2000082
:1055E0000DF014F844F2C010C2F20000FEF77AFA8F
:1055F00023684DF2180898420746C1F6FF7800F379
:10560000A784C0F27D849F4227D049F2EF28FBB2E5
:10561000C1F6FF78184688F80030FFF7B9FE40F66B
:105620001C40C0F20200FBF74FF898F80000FBF7AF
:1056300039F84CF69C314DF23040C2F20001C2F212
:1056400000000CF06BFF4DF23040C2F200000CF095
:10565000B1FF33680193019B2B604EF28050C2F280
:10566000000027600DF010F8002840F04A824DF647
:10567000D805C2F200054EF29050C2F200000CF0C4
:10568000C5FF44F2E010C2F20000FEF72BFA064616
:105690004DF23040C2F200000CF05CFF854200F099
:1056A00023824DF23040C2F200000CF053FF4BF663
:1056B0004423C1F6FF73834200F0E6844DF230408C
:1056C000C2F200000CF046FF4CF22C23C1F6FF732F
:1056D000834200F0E7844DF23040C2F200000CF04B
:1056E00039FF4BF2CC13C2F20003834200F0228454
:1056F0004DF23040C2F200000CF02CFF4CF670135B
:10570000C2F20003834200F00A854DF23040C2F23B
:1057100000000CF01FFF4DF6BC23C2F200038342D1
:1057200000F00F854DF23040C2F200000CF012FF85
:105730004CF25453C1F6FF73834200F04C854DF296
:105740003040C2F200000CF005FF4CF6CC33C1F63D
:10575000FF73834200F0CA844DF23040C2F2000071
:105760000CF0F8FE4BF67803C1F6FF73834200F0AD
:105770006C854DF23040C2F200000CF0EBFE4CF2B2
:10578000C013C2F20003834200F088854DF230401E
:10579000C2F200000CF0DEFE4EF2A053C2F2000393
:1057A000834200F0A0854DF23040C2F200000CF0C0
:1057B000D1FE4BF27C33C2F20003834200F0B88585
:1057C0004DF23040C2F200000CF0C4FE4CF60C2347
:1057D000C1F6FF73834200F0D0854DF23040C2F233
:1057E00000000CF0B7FE4BF63453C2F200038342C4
:1057F00000F0E8854DF23040C2F200000CF0AAFE45
:105800004CF64C33C2F20003834200F016864DF290
:105810003040C2F200000CF09DFE4BF27C13C2F24D
:105820000003834200F02E864DF23040C2F20000A9
:105830000CF090FE4DF20C73C2F20003834200F0B4
:1058400046864DF23040C2F200000CF083FE4DF26D
:10585000DC03C2F20003834200F08B864DF230403D
:10586000C2F200000CF076FE4EF6F803C2F200031E
:10587000834200F06F864DF23040C2F200000CF01F
:1058800069FE4CF66003C2F20003834200F05386C7
:105890004DF23040C2F200000CF05CFE4CF2883356
:1058A000C1F6FF73834200F037864DF23040C2F2FA
:1058B00000000CF04FFE4BF64063C2F2000383423F
:1058C00000F0A8864DF23040C2F200000CF042FE1B
:1058D0004DF26033C2F20003834200F009874DF2BB
:1058E0003040C2F200000CF035FE4BF21C03C1F652
:1058F000FF73834200F0ED864DF23040C2F20000AB
:105900000CF028FE4CF65063C1F6FF73834200F0A2
:10591000D1864DF23040C2F200000CF01BFE4BF27B
:105920006C73C1F6FF73834200F0B5864DF23040D0
:10593000C2F200000CF00EFE4DF60C33C2F2000372
:10594000834200F04C874DF23040C2F200000CF070
:1059500001FE4CF21043C2F20003834200F0308794
:105960004DF23040C2F200000CF0F4FD4DF69053C1
:10597000C2F20003834200F014874DF23040C2F2BD
:1059800000000CF0E7FD4CF21023C2F2000383424A
:1059900000F0F8864DF23040C2F200000CF0DAFD63
:1059A0004DF21433C1F6FF73834200F0DC864DF2F2
:1059B0003040C2F200000CF0CDFD4DF6DC23C1F604
:1059C000FF73834200F0C0864DF23040C2F2000007
:1059D0000CF0C0FD4BF26C03C1F6FF73834200F084
:1059E000A4864DF23040C2F200000CF0B3FD4AF242
:1059F0002463C2F200038342636800F088864DF29C
:105A000018079E42C1F6FF7700F3138616DA40F6B8
:105A10008030C0F20200FAF757FE49F2E4603146E6
:105A2000C1F6FF70FDF726F9F0B23979FEF796F866
:105A30004DF23040C2F200000CF0C2FD4EF2905028
:105A4000C2F2000066600CF01FFE002840F0858264
:105A500002B0BDE8F0814DF23040C2F200000CF01F
:105A600079FD4CF27C23C1F6FF7383427FF4B0AD25
:105A700041F2640044F2C017C2F20007C0F2020013
:105A8000FAF72CFE07F12000FEF72CF84CF2A438B0
:105A9000C2F200084BF6FC2188F827004DF2304096
:105AA000C2F20001C2F200000CF038FD4DF23040AD
:105AB0000221C2F200004DF218040CF057FDC1F6AD
:105AC000FF7498F90030636000220521B96323EA6E
:105AD000E37387F83C207A6372B68B42A8BF0B460B
:105AE0009B00FB6262B677E563689E42A6D0F0B287
:105AF000FEF730F94DF23040C2F200000CF05AFDD2
:105B00009CE740F62C40C0F20200FAF7DDFD4DF2B2
:105B10003040C2F200000CF01DFD4DF6D805C2F277
:105B20000005854200F030834DF23040C2F20000A3
:105B30000CF010FD4BF22C33C2F20003834200F054
:105B40002E834DF23040C2F200000CF003FD4BF604
:105B50004423C1F6FF73834200F04B834DF2304083
:105B6000C2F200000CF0F6FC4CF22C23C1F6FF73DD
:105B7000834200F049834DF23040C2F200000CF045
:105B8000E9FC4BF2CC13C2F20003834200F04783DE
:105B90004DF23040C2F200000CF0DCFC4CF6701309
:105BA000C2F20003834200F045834DF23040C2F25E
:105BB00000000CF0CFFC4DF6BC23C2F20003834280
:105BC00000F052834DF23040C2F200000CF0C2FCF3
:105BD0004CF25453C1F6FF73834200F054834DF2EC
:105BE0003040C2F200000CF0B5FC4CF6CC33C1F6EC
:105BF000FF73834200F088824DF23040C2F2000011
:105C00000CF0A8FC4BF67803C1F6FF73834200F05A
:105C100054834DF23040C2F200000CF09BFC4CF279
:105C2000C013C2F20003834200F052834DF23040B1
:105C3000C2F200000CF08EFC4BF24013C1F6FF7371
:105C4000834200F05F834DF23040C2F200000CF05E
:105C500081FC4EF2A053C2F20003834200F05D8348
:105C60004DF23040C2F200000CF074FC4BF27C3379
:105C7000C2F20003834200F06A834DF23040C2F268
:105C800000000CF067FC4CF60C23C1F6FF73834256
:105C900000F068834DF23040C2F200000CF05AFC74
:105CA0004BF63453C2F20003834200F075834DF289
:105CB0003040C2F200000CF04DFC4CF64C33C2F206
:105CC0000003834200F073834DF23040C2F20000C3
:105CD0000CF040FC4BF27C13C2F20003834200F054
:105CE00080834DF23040C2F200000CF033FC4DF2E4
:105CF0000C73C2F20003834200F07E834DF2304009
:105D0000C2F200000CF026FC4DF2DC03C2F20003EC
:105D1000834200F087834DF23040C2F200000CF065
:105D200019FC4EF6F803C2F20003834200F06F83C1
:105D30004DF23040C2F200000CF00CFC4CF6600357
:105D4000C2F20003834200F092834DF23040C2F26F
:105D500000000CF0FFFB4CF28833C1F6FF73834266
:105D600000F07A834DF23040C2F200000CF0F2FBFA
:105D70004BF64063C2F20003834200F09D834DF274
:105D80003040C2F200000CF0E5FB4DF26033C2F28D
:105D90000003834200F085834DF23040C2F20000E0
:105DA0000CF0D8FB4BF21C03C1F6FF73834200F0EA
:105DB0009D834DF23040C2F200000CF0CBFB4CF65C
:105DC0005063C1F6FF73834200F09B834DF2304075
:105DD000C2F200000CF0BEFB4BF26C73C1F6FF7315
:105DE000834200F0E0834DF23040C2F200000CF03C
:105DF000B1FB4DF60C33C2F20003834200F0C883BE
:105E00004DF23040C2F200000CF0A4FB4CF2104303
:105E1000C2F20003834200F0F2834DF23040C2F23E
:105E200000000CF097FB4DF69053C2F20003834242
:105E300000F0DA834DF23040C2F200000CF08AFB31
:105E40004CF21023C2F20003834200F0C2834DF2F1
:105E50003040C2F200000CF07DFB4BF2DC23C2F2BA
:105E60000003834200F0AA834DF23040C2F20000EA
:105E70000CF070FB4DF21433C1F6FF73834200F057
:105E8000FF834DF23040C2F200000CF063FB4DF690
:105E9000DC23C1F6FF73834200F0E7834DF230400C
:105EA000C2F200000CF056FB4BF26C03C1F6FF731C
:105EB000834200F0CF834DF23040C2F200000CF07C
:105EC00049FB4AF22463C2F20003834200F0B78325
:105ED0004DF23040C2F200000CF03CFB4CF6546333
:105EE000C2F2000383427FF4C6AB41F25000C0F21D
:105EF0000200FAF7F3FB0620FDF754FEFFF7BBBBE9
:105F000040F61040C0F20200FAF7DEFB49F2E4600E
:105F10003946C1F6FF700FF0F5FA49F2E460C1F6B8
:105F2000FF700FF04DFBD8F800309F427FF46DAB4F
:105F3000FFF793BB63689E423FF480ADF0B2FDF77C
:105F4000ABFF4DF23040C2F200000CF033FB75E5C0
:105F500040F60040C0F20200D6E740F68C30C0F2B6
:105F60000200FAF7BBFB4DF23040C2F200000CF029
:105F7000F1FA854200F0F7804DF23040C2F20000A5
:105F80000CF0E8FA4CF21023C2F20003834200F056
:105F900011814DF23040C2F200000CF0DBFA4BF2FE
:105FA0002C33C2F20003834200F0C7804DF2304030
:105FB000C2F200000CF0CEFA4BF24013C1F6FF73B0
:105FC000834200F0CC804DF23040C2F200000CF071
:105FD000C1FA4BF2DC23C2F20003834200F04F818E
:105FE00000252F462E4640F69830C0F20200FAF700
:105FF0006BFB616849F2E46001312944C1F6FF702E
:106000000FF080FA49F2E460C1F6FF700FF0D8FAA1
:1060100040F6B430C0F20200FAF756FB49F2E460F1
:106020006168C1F6FF700FF06DFA40F6D430C0F22F
:106030000200FAF749FB49F2E460394600230A22DC
:10604000C1F6FF700FF0CEFA49F2E460C1F6FF70BE
:106050000FF0B6FA6168013131444DF230404DF233
:106060001804C9B2C2F20000C1F6FF740CF084FA41
:1060700030B36168013131444DF23040C9B2C2F2EF
:1060800000000CF07FFAE3E463689E423FF4D6AC74
:10609000F0B2FDF799FE4DF23040C2F200000CF074
:1060A00089FACBE463689E423FF4C8ACF0B2FDF7D6
:1060B000BFFE4DF23040C2F200000CF07BFABDE4AE
:1060C00040F6EC30C0F20200FAF7FEFA616849F2DD
:1060D000E46001312944C1F6FF700FF013FA49F270
:1060E000E460C1F6FF700FF06BFAB1E463689E42A2
:1060F0003FF4A4AC70B2FDF783FF4DF23040C2F222
:1061000000000CF057FA99E440F60850C0F2020083
:10611000FAF7E4FA0D20FDF77BFDFFF7ACBA6368F0
:106120009E423FF48BACF0B2FDF7EAFE4DF23040F8
:10613000C2F200000CF03EFA80E406252F462E46FF
:1061400051E763689E423FF479AC70B2FDF70CFFF3
:106150004DF23040C2F200000CF02CFA6EE4102533
:106160002F462E463FE749F24034C1F6FF7440F611
:106170009C00C0F20200FAF7A7FA2078FAF792FA28
:106180002078FDF7E7FD63E440F64440C0F20200EA
:10619000FAF7A4FA0120FDF705FDFFF76CBA40F607
:1061A0004440C0F20200FAF799FA0220FDF7FAFC27
:1061B000FFF761BA49F24034C1F6FF7440F6A80017
:1061C000C0F20200FAF780FA2078FAF76BFA20782A
:1061D000FDF7DEFD3CE463689E423FF42FAC70B2F5
:1061E000FDF7F4FE4DF23040C2F200000CF0E2F98F
:1061F00024E440F65C40C0F20200FAF76FFA072090
:10620000FDF706FDFFF737BA40F67840C0F202000E
:10621000FAF764FA0820FDF7FBFCFFF72CBA40F60A
:106220009440C0F20200FAF759FA0920FDF7F0FC99
:10623000FFF721BA40F6B040C0F20200FAF74EFA7A
:106240000A20FDF7E5FCFFF716BA63689E423FF4AB
:10625000F5ABF0B2FDF70CFF4DF23040C2F200009A
:106260000CF0A8F9FFF7EABB40F6CC40C0F2020000
:10627000FAF734FA0B20FDF7CBFCFFF7FCB9232526
:106280002F462E46AFE640F6E840C0F20200FAF78D
:1062900025FA0C20FDF7BCFCFFF7EDB963689E42C0
:1062A0003FF4CCABF0B2FDF717FF4DF23040C2F235
:1062B00000000CF07FF9FFF7C1BB40F62050C0F2A0
:1062C0000200FAF70BFA0E20FDF7A2FCFFF7D3B994
:1062D00040F63C50C0F20200FAF700FA0F20FDF73A
:1062E00097FCFFF7C8B963689E423FF4A7ABF0B2D2
:1062F000FDF726FF4DF23040C2F200000CF05AF9D3
:10630000FFF79CBB40F66050C0F20200FAF7E6F9D6
:106310000320FDF747FCFFF7AEB940F67450C0F21A
:106320000200FAF7DBF91020FDF7A8FCFFF7A3B98C
:1063300063689E423FF482ABF0B2FDF735FF4DF249
:106340003040C2F200000CF035F9FFF777BB40F6A1
:106350009850C0F20200FAF7C1F91120FDF78EFC47
:10636000FFF789B940F6B850C0F20200FAF7B6F963
:106370001220FDF783FCFFF77EB963689E423FF46D
:106380005DABF0B2FDF744FF4DF23040C2F20000C9
:106390000CF010F9FFF752BB40F6D450C0F20200E7
:1063A000FAF79CF91320FDF769FCFFF764B940F692
:1063B000F050C0F20200FAF791F91420FDF75EFCEC
:1063C000FFF759B963689E423FF438ABF0B2FDF76E
:1063D00053FF4DF23040C2F200000CF0EBF8FFF733
:1063E0002DBB40F61060C0F20200FAF777F91520D5
:1063F000FDF744FCFFF73FB940F62C60C0F2020005
:10640000FAF76CF91620FDF739FCFFF734B940F6BE
:106410006860C0F20200FAF761F91820FDF72EFC5F
:10642000FFF729B940F64C60C0F20200FAF756F9BE
:106430001720FDF723FCFFF71EB963689E423FF467
:10644000FDAAF0B2FDF764FF4DF23040C2F2000049
:106450000CF0B0F8FFF7F2BA40F6A460C0F2020008
:10646000FAF73CF91A20FDF709FCFFF704B940F6EA
:106470008460C0F20200FAF731F91920FDF7FEFB43
:10648000FFF7F9B863689E423FF4D8AAF0B2FDF76F
:106490008DFF4DF23040C2F200000CF08BF8FFF798
:1064A000CDBA40F6E460C0F20200FAF717F91C20FA
:1064B000FDF7E4FBFFF7DFB840F6C460C0F202006E
:1064C000FAF70CF91B20FDF7D9FBFFF7D4B8636886
:1064D0009E423FF4B3AAF0B2FDF7B6FF4DF2304052
:1064E000C2F200000CF066F8FFF7A8BA40F6087098
:1064F000C0F20200FAF7F2F81D20FDF7BFFBFFF72C
:10650000BAB840F62870C0F20200FAF7E7F81E2089
:10651000FDF7B4FBFFF7AFB863689E423FF48EAA65
:10652000F0B2FEF7C7F84DF23040C2F200000CF0B6
:1065300041F8FFF783BA63689E423FF47FAAF0B246
:10654000FEF730F84DF23040C2F200000CF032F8A5
:10655000FFF774BA63689E423FF470AAF0B2FDF789
:10656000E7FF4DF23040C2F200000CF023F8FFF7D5
:1065700065BA63689E423FF461AAF0B2FDF79EFFE0
:106580004DF23040C2F200000CF014F8FFF756BA9A
:1065900040F66870C0F20200FAF7A0F82020FDF77C
:1065A0006DFBFFF768B840F64870C0F20200FAF7DA
:1065B00095F81F20FDF762FBFFF75DB840F6D0703D
:1065C000C0F20200FAF78AF80520FDF7EBFAFFF7B0
:1065D00052B840F6B870C0F20200FAF77FF8042013
:1065E000FDF7E0FAFFF747B840F6A070C0F20200EE
:1065F000FAF774F82220FDF741FBFFF73CB840F6AC
:106600008870C0F20200FAF769F82120FDF736FB26
:10661000FFF731B863689E423FF410AAF0B2FEF76C
:10662000DDF84DF23040C2F200000BF0C3FFFFF77F
:1066300005BA40F67030C0F20200FFF7ECB941F243
:106640003800C0F20200FAF749F82620FDF74CFBAB
:10665000FFF711B841F21800C0F20200FAF73EF855
:106660002520FDF741FBFFF706B840F6FC70C0F2AD
:106670000200FAF733F82420FDF736FBFEF7FBBFE4
:1066800040F6E470C0F20200FAF728F82320FDF784
:106690002BFBFEF7F0BF63689E423FF4CFA9F0B238
:1066A000FEF776F94DF23040C2F200000BF082FFA7
:1066B000FFF7C4B963689E423FF4C0A9F0B2FEF789
:1066C0004BF94DF23040C2F200000BF073FFFFF7C0
:1066D000B5B963689E423FF4B1A9F0B2FEF720F964
:1066E0004DF23040C2F200000BF064FFFFF7A6B994
:1066F00063689E423FF4A2A9F0B2FEF7F5F84DF2AE
:106700003040C2F200000BF055FFFFF797B99E42F0
:106710003FF494A9F0B2FEF7B5FA4DF23040C2F260
:1067200000000BF047FFFFF789B963689E423FF412
:1067300085A9F0B2FEF786FA4DF23040C2F20000B1
:106740000BF038FFFFF77AB963689E423FF476A9F1
:10675000F0B2FEF759FA4DF23040C2F200000BF0F1
:1067600029FFFFF76BB963689E423FF467A9F0B257
:10677000FEF716FA4DF23040C2F200000BF01AFF9D
:10678000FFF75CB963689E423FF458A9F0B2FDF789
:10679000FFFA4DF23040C2F200000BF00BFFFFF7A2
:1067A0004DB963689E423FF449A9F0B2FEF7B0F9D3
:1067B0004DF23040C2F200000BF0FCFEFFF73EB994
:1067C00063689E423FF43AA9F0B2FEF759F94DF2E0
:1067D0003040C2F200000BF0EDFEFFF72FB9636806
:1067E0009E423FF42BA9F0B2FEF70EF94DF2304075
:1067F000C2F200000BF0DEFEFFF720B92DE9F043F6
:106800004FF6FC64C0F201040FCC91B06D460FC589
:106810000FCC0FC50FCC0FC594E80F0085E80F0013
:1068200049F2FC21C1F6FF710D1F05F128074FF059
:10683000FF3411F8013B83EA040210A802F00F02B2
:1068400000EB820249F2F82652F8402C82EA141436
:1068500084EA131303F00F0300EB8303B94253F8E8
:10686000403C83EA1414C1F6FF766FEA0404E0D1D9
:106870004FF6FC6CC0F2010CBCE80F00EE46AEE82F
:106880000F00BCE80F00AEE80F00BCE80F004BF6AD
:106890008418AEE80F009CE80F00C1F6FF7846F8B8
:1068A000044B98F800408EE80F00601E00EB80005B
:1068B000C0004FF0FF3216F8013B83EA020110AC32
:1068C00001F00F0104EB8101BE4251F8401C81EA46
:1068D000121282EA131303F00F0310A901EB8303D2
:1068E00049F2F82453F8403C83EA1212C1F6FF74CF
:1068F0006FEA0202DFD1C5F1010505EB0009227044
:1069000014F8016B04EB090528460FF0ADF8864238
:106910003146284601D00FF0C1F8BC42F0D141F217
:10692000DC002821C0F2020012F0FEF949F2E46016
:1069300000230A2298F80010C1F6FF700EF052FEF4
:1069400041F208100621C0F2020012F0EDF998F8A9
:106950000030013B03EB8303D90049F2E4600231CC
:1069600000231022C1F6FF700EF03CFE49F2E460F5
:10697000C1F6FF700EF024FE002388F8003011B03D
:10698000BDE8F083F0B549F24035C1F6FF759BB024
:106990002E781AAB013E06EB8606C3F16B0303EBC0
:1069A000C6060DF1FF340DF1270730190FF05CF822
:1069B00004F8010FA742F8D14FF6FC64C0F20104BD
:1069C0000FCC0AAE37460FC70FCC0FC70FCC0FC77F
:1069D00094E80F004FF0FF3487E80F0001A911F889
:1069E000013B83EA04021AA802F00F0200EB8202C4
:1069F000B14252F8402C82EA141484EA131303F0D3
:106A00000F0300EB830353F8403C83EA14146FEA4E
:106A10000404E4D141F28000C0F20200F9F754FE10
:106A2000009E49F2E460314600231022C1F6FF7057
:106A30000EF0D8FD41F29400C0F20200F9F744FED6
:106A400049F2E460C1F6FF700023102221460EF0E7
:106A5000C9FDA6423CD041F24C10C0F20200F9F749
:106A60003DFE4BF68413C1F6FF732A781A70FFF7C8
:106A7000C5FE49F2EF24C1F6FF7441F22010C0F2C6
:106A80000200F9F721FE49F2E460217800230A228E
:106A9000C1F6FF700EF0A6FD49F2E460C1F6FF708A
:106AA0000EF08EFD41F23410C0F20200F9F70CFE38
:106AB00049F2E4606321C1F6FF700EF023FD49F254
:106AC000E460C1F6FF701BB0BDE8F0400EF078BD89
:106AD0004EF28050C2F200000BF0D4FD18B32D78B6
:106AE00049F2F724C1F6FF74013D05EB8505C4F1B9
:106AF000020303EBC50504F1280628190EF0B4FFC4
:106B000004F8010FB442F8D100200EF0ADFF49F2B5
:106B1000EF24C1F6FF74207041F21010C0F20200A1
:106B2000F9F7D2FDA9E74EF29050C2F200000BF047
:106B3000A9FD00288FD0D2E72DE9F8434FF20E6966
:106B4000C2F2000941F2A0102DED028BC0F202004A
:106B5000F9F7BAFDB9F8003007EE103A43F23333D3
:106B6000C4F2233308EE903AB8EEC77A43F23333D7
:106B7000C4F2A33308EE103A37EE287A49F2E464FF
:106B8000C7EE087AC1F6FF744FF20867C2F2000739
:106B90004FF20C68C2F200084FF28C56C2F20006A7
:106BA0004CF66C15C2F2000517EE900A14F000FDC9
:106BB00041EC100B0A2120460EF054FD41F2A810C2
:106BC000C0F20200F9F780FD3B8807EE903AF8EE3C
:106BD000E77A77EEA87A87EE887A17EE100A14F033
:106BE000E7FC41EC100B0A2120460EF03BFD41F280
:106BF000B810C0F20200F9F767FDB8F8001020469F
:106C00000EF080FC41F2C010C0F20200F9F75CFD0A
:106C1000318820460EF076FC41F2D010C0F202001E
:106C2000F9F752FD298820460EF06CFC41F2E8107D
:106C3000C0F20200F9F748FD4CF6DC33C2F2000363
:106C40000A221968204600230EF0CCFC41F2F41011
:106C5000C0F20200F9F738FD4CF25053C1F6FF7351
:106C60000A221968204600230EF0BCFC41F20420E1
:106C7000C0F20200F9F728FD4CF27073C1F6FF7301
:106C80000A221968204600230EF0ACFC41F21020C5
:106C9000C0F20200F9F718FD4BF21C23C2F2000308
:106CA000186805F013FE014620460EF02BFC204626
:106CB0000EF086FCBDEC028BB9F80030B8F800206D
:106CC0003B80002332802B80BDE8F883F8B5044672
:106CD000551E4F1E2270A570012200256170227181
:106CE0002946A57184F8B950C4F8A050C4F8A4503E
:106CF000C4F8A850C4F8AC50C4F8B050C4F8B450AC
:106D0000982284F8B850E77004F108001E4615F088
:106D1000D3FC0222627120460BF084F8A579042D81
:106D20000CD805F12803254444F8236030780BF093
:106D300051FC85F8B400A3790133A3712046F8BD56
:106D4000F8B50446551E4F1E2270A570012200257D
:106D5000617022712946A57184F8B950C4F8A05019
:106D6000C4F8A450C4F8A850C4F8AC50C4F8B0504B
:106D7000C4F8B450982284F8B850E77004F10800C1
:106D80001E4615F099FC0222627120460BF04AF86B
:106D9000A579042D0DD805F12803254444F8236076
:106DA00096F900000BF014FC85F8B400A3790133C8
:106DB000A3712046F8BD00BFF8B50446551E4F1E0E
:106DC0002270A57001220025617022712946A571EB
:106DD00084F8B950C4F8A050C4F8A450C4F8A8501E
:106DE000C4F8AC50C4F8B050C4F8B450982284F839
:106DF000B850E77004F108001E4615F05DFC022251
:106E0000627120460BF00EF8A579042D0CD805F11F
:106E10002803304644F823600BF0DEFB254485F858
:106E2000B400A3790133A3712046F8BDF8B5044638
:106E3000551E4F1E2270A57001220025617022711F
:106E40002946A57184F8B950C4F8A050C4F8A450DC
:106E5000C4F8A850C4F8AC50C4F8B050C4F8B4504A
:106E6000982284F8B850E77004F108001E4615F027
:106E700023FC0222627120460AF0D4FFA579042D7A
:106E80000CD805F12803304644F823600BF09EFB34
:106E9000254485F8B400A3790133A3712046F8BDD9
:106EA0002DE9F04193F0010807460E46154610D132
:106EB00069B1013D0024B86C15F8011F0368013465
:106EC0001B689847A642F6D8B8F1000F08D1BDE874
:106ED000F081806C0368F021DB6C9847002EE8D1CC
:106EE000B86C0368F721DB6CBDE8F041184700BFC0
:106EF0002DE9F0479DF82040013CE4B20F2C03D867
:106F00004EB2002E0D4601DBBDE8F087E0290ED918
:106F1000F729F9D90835EDB2012303FA05F515F083
:106F2000DD0FF1D04830BDE8F047F9F7A9BB814645
:106F3000806C1F46036846EA0401C9B21B6890468C
:106F40009847D9F84800036808F07F011B6805F0EE
:106F5000EF059847C02DD7D0D9F84800036807F04F
:106F60007F011B68BDE8F047184700BFF0B549F244
:106F7000F824C1F6FF7483B094F821300E4615460C
:106F8000074623B1984202D0F9F7A0FE50B14BF268
:106F90001C23C2F2000394F90910186831442A46F0
:106FA00005F098FC41F22420C0F20200162111F0F5
:106FB000BBFE94F822303BB34DF6E4402B463246FC
:106FC0009021C1F6FF700097FFF792FF2D0640F267
:106FD000E000C0F2020005F0FE45F9F775FB45F44C
:106FE00010453604781E45F0090506F4FE06000239
:106FF000354300F47060284311F00CF840F2900023
:10700000C0F20200F9F760FB49F2E460C1F6FF70DC
:1070100003B0BDE8F0400EF0D3BA00BFF0B549F2BE
:10702000F824C1F6FF7483B094F821300E4615465B
:10703000074623B1984202D0F9F748FE50B14BF20F
:107040001C23C2F2000394F90910186831442A463F
:1070500005F040FC41F23C20C0F20200112111F089
:1070600063FE94F822305BB34DF6E4402B46324683
:107070009021C1F6FF700097FFF73AFF2D0640F20E
:10708000E000C0F2020005F0FE45F9F71DFB45F4F3
:1070900010453604791E45F0090506F4FE0609027E
:1070A000354301F470614DF6A060C2F2000029433F
:1070B0000DF024F940F27800C0F20200F9F704FB69
:1070C00049F2E460C1F6FF7003B0BDE8F0400EF095
:1070D00077BA00BFF0B549F2F824C1F6FF7483B067
:1070E00094F821300E461546074623B1984202D047
:1070F000F9F7ECFD50B14BF21C23C2F2000394F9F6
:10710000091018683144002205F0E4FB41F25020D8
:10711000C0F20200172111F007FE94F822303BB3B1
:107120004DF6E4402B4632468021C1F6FF700097B1
:10713000FFF7DEFE2D0640F2E000C0F2020005F08F
:10714000FE45F9F7C1FA45F400453604781E45F0CE
:10715000080506F4FE060002354300F4706028437B
:1071600010F058FF40F29000C0F20200F9F7ACFABC
:1071700049F2E460C1F6FF7003B0BDE8F0400EF0E4
:107180001FBA00BFF0B549F2F824C1F6FF7483B00E
:1071900094F821300E461546074623B1984202D096
:1071A000F9F794FD50B14BF21C23C2F2000394F99D
:1071B000091018683144002205F08CFB41F2682068
:1071C000C0F20200122111F0AFFD94F822305BB33F
:1071D0004DF6E4402B4632468021C1F6FF70009701
:1071E000FFF786FE2D0640F2E000C0F2020005F037
:1071F000FE45F9F769FA45F400453604791E45F075
:10720000080506F4FE060902354301F470614DF6E7
:10721000A060C2F2000029430DF070F840F278003F
:10722000C0F20200F9F750FA49F2E460C1F6FF70CB
:1072300003B0BDE8F0400EF0C3B900BFF0B549F2AD
:10724000F825C1F6FF7583B095F821300E46144637
:10725000074623B1984202D0F9F738FD48B14BF206
:107260001C23C2F2000322461868036831465B689B
:10727000984741F27C20C0F20200122111F054FD27
:1072800095F822303BB34DF6E44023463246B02118
:10729000C1F6FF700097FFF72BFE240640F2E000D6
:1072A000C0F2020004F0FE44F9F70EFA44F4304450
:1072B0003604781E44F00B0406F4FE060002344344
:1072C00000F47060204310F0A5FE40F29000C0F280
:1072D0000200F9F7F9F949F2E460C1F6FF7003B072
:1072E000BDE8F0400EF06CB9F0B549F2F825C1F6F2
:1072F000FF7583B095F821300E461446074623B13A
:10730000984202D0F9F7E2FC48B14BF21C23C2F2DA
:10731000000322461868036831465B68984741F2CB
:107320009020C0F202000D2111F0FEFC95F82230F1
:107330005BB34DF6E44023463246B021C1F6FF7000
:107340000097FFF7D5FD240640F2E000C0F20200EE
:1073500004F0FE44F9F7B8F944F430443604791ED9
:1073600044F00B0406F4FE060902344301F4706194
:107370004DF6A060C2F2000021430CF0BFFF40F2C6
:107380007800C0F20200F9F79FF949F2E460C1F613
:10739000FF7003B0BDE8F0400EF012B930B50546FD
:1073A00041F2A02083B00C46C0F20200122111F07D
:1073B000BBFC49F2F823C1F6FF7393F822301BB3EC
:1073C0004DF6E44022460023D021C1F6FF7000951F
:1073D000FFF78EFD40F2E000C0F202002404F9F74E
:1073E00073F904F4FE04681E44F45044000244F0AF
:1073F0000D0400F47060204310F00CFE40F2900089
:10740000C0F20200F9F760F949F2E460C1F6FF70DA
:1074100003B0BDE830400EF0D3B800BF30B505462C
:1074200041F2B42083B00C46C0F202000D2111F0ED
:107430007BFC49F2F823C1F6FF7393F822303BB38B
:107440004DF6E44022460023D021C1F6FF7000959E
:10745000FFF74EFD40F2E000C0F202002404F9F70D
:1074600033F904F4FE04691E44F45044090244F064
:107470000D0401F470614DF6A060C2F200002143DA
:107480000CF03CFF40F27800C0F20200F9F71CF962
:1074900049F2E460C1F6FF7003B0BDE830400EF081
:1074A0008FB800BF30B5054641F2C42083B00C460A
:1074B000C0F20200122111F037FC49F2F823C1F6A4
:1074C000FF7393F822307BB304F500524DF6E4408D
:1074D000C2F3C613E02102F07F020095C1F6FF70EF
:1074E000FFF706FD04F30D0440F2E00004F500543C
:1074F000C0F20200013DF9F7E7F82D02200400F484
:10750000FE0005F47065054345F46040640440F0F6
:107510000E0004F0FE44204310F07CFD40F2900089
:10752000C0F20200F9F7D0F849F2E460C1F6FF704A
:1075300003B0BDE830400EF043B800BF30B505469B
:1075400041F2D82083B00C46C0F202000D2111F0A8
:10755000EBFB49F2F823C1F6FF7393F822309BB39B
:1075600004F500524DF6E440C2F3C613E02102F0E8
:107570007F020095C1F6FF70FFF7BAFC04F30D041B
:1075800040F2E00004F50054C0F20200013DF9F7BA
:107590009BF82D02210401F4FE0105F470650D43F2
:1075A00045F46041640441F00E0104F0FE444DF6E0
:1075B000A060C2F2000021430CF0A0FE40F278006F
:1075C000C0F20200F9F780F849F2E460C1F6FF70FA
:1075D00003B0BDE830400DF0F3BF00BF30B5054645
:1075E00041F2E82083B00C46C0F20200122111F0F3
:1075F0009BFB49F2F823C1F6FF7393F822301BB3CB
:107600004DF6E44022460023C021C1F6FF700095EC
:10761000FFF76EFC40F2E000C0F202002404F9F72C
:1076200053F804F4FE04681E44F44044000244F09D
:107630000C0400F47060204310F0ECFC40F2900069
:10764000C0F20200F9F740F849F2E460C1F6FF70B9
:1076500003B0BDE830400DF0B3BF00BF30B5054604
:1076600041F2FC2083B00C46C0F202000D2111F063
:107670005BFB49F2F823C1F6FF7393F822303BB36A
:107680004DF6E44022460023C021C1F6FF7000956C
:10769000FFF72EFC40F2E000C0F202002404F9F7EC
:1076A00013F804F4FE04691E44F44044090244F053
:1076B0000C0401F470614DF6A060C2F20000214399
:1076C0000CF01CFE40F27800C0F20200F8F7FCFF5C
:1076D00049F2E460C1F6FF7003B0BDE830400DF040
:1076E0006FBF00BF70B5064641F20C3082B00C4649
:1076F000C0F202001721154611F016FB49F2F823DB
:10770000C1F6FF7393F8223043B949F2E460C1F641
:10771000FF7002B0BDE870400DF052BF4DF6E4407E
:10772000C1F6FF7000962B462246A021FFF7E0FB32
:1077300041F22430C0F20200F8F7C6FF36B140F241
:107740009000C0F20200F8F7BFFFDEE7681E0002FB
:10775000240404F4FE0400F47060204340F450401C
:1077600040F00D0010F056FCE9E700BF70B506468A
:1077700041F2303082B00C46C0F2020012211546B0
:1077800011F0D2FA49F2F823C1F6FF7393F82230D0
:1077900053B34DF6E44022462B46A021C1F6FF70BC
:1077A0000096FFF7A5FB41F22430C0F20200F8F783
:1077B0008BFF691E0902240401F4706104F4FE04C5
:1077C0000C4344F45044310144F00D04C9B24DF669
:1077D000A060C2F2000021430CF090FD40F278005E
:1077E000C0F20200F8F770FF49F2E460C1F6FF70E2
:1077F00002B0BDE870400DF0E3BE00BFF8B504462E
:10780000806C03681B69984708B90020F8BDA06C1C
:1078100003685B699847C3B203F0FB01F929F4D010
:10782000A26D7AB994F84D2084F84F30150666D4CD
:1078300040B20028C0F24781002084F84D00A065C6
:107840006065F8BD010633D494F84F10F02904EBBD
:10785000020124D081F84F30616D4B1E9A4224D32F
:1078600094F84F20F02AE7D0130600F1C2800020E0
:1078700094F8503084F86600032984F8650084F891
:10788000673000F0CD80012384F86800A065606552
:1078900084F8E930002384F84D300120F8BD81F8E8
:1078A0006930636D013B9A42C6D20132A265ACE7F2
:1078B000A3F1F7010829C7D8012505FA01F010F452
:1078C000DD7F40F0CD800029BED194F86930F02BE7
:1078D000B2D1561C2244F720370A82F8690084F896
:1078E000676084F8687084F8651084F84D10284645
:1078F00084F8663084F8E950A1656165F8BD02F14D
:107900000C05EEB2012E93D902F0FB0EBEF1F90F79
:107910008ED0EF2A36D802F0F007802F33D140B254
:10792000002886DB012184F84F2084F85030A165BF
:10793000EDB2012D80D9BEF1F90F3FF47DAFEF2AF2
:1079400000F29B8002F0F003F12B4ED000F2978002
:10795000B02B43D03BD9D02B47D043D9E02B3DD0DF
:10796000F02B7FF469AF0021802084F84D1084F85B
:10797000693060657F21A36D8B4211D20133A3650D
:107980000020F8BD174607F0DF06902EC7D007F09D
:10799000BF06A02EC3D007F0EF07C02FBFD047E728
:1079A0001046F8F771FE02F00F020023013294F83E
:1079B000501084F8660084F86520012084F8671070
:1079C00084F86830A365636584F8E900F8BD902BFE
:1079D00004D0A02B02D0802B7FF42EAF032363654D
:1079E0000221C8E7C02B7FF427AF02236365012182
:1079F000C1E7F42A3FF43BAF1046F8F745FE802874
:107A000084F8660064D102F00F03013394F85050FB
:107A100084F86750032984F8653018BF002501D128
:107A200094F8515084F8685000230121B028A365D0
:107A3000636584F8E91007D00AD8902804D0A028FC
:107A400002D080287FF426AF84F84D200120F8BDB5
:107A5000D028F9D0E028F7D0C0287FF41BAFF3E797
:107A6000002284F8672084F8682084F8652084F870
:107A7000663084F8E9502846F8BD134664E7F82BD1
:107A800006D018D8F32BB0D0A8D3F62B7FF4D4AE01
:107A90001046F8F7F9FD0022012384F8652084F8E8
:107AA000672084F8682084F86600A265626584F81F
:107AB000E9301846F8BDFA2BFFF4BEAEFC2BE7D92F
:107AC000FE2BE5D2B8E61A468E4603F10C052FE7E9
:107AD000902898D0B02896D0A02894D0D02892D0C2
:107AE000E02890D0C0288ED000238FE790F8663031
:107AF000F12B7CD00ED9FA2B2BD01FD8F32B38D0FA
:107B0000C0F08180F62B7AD0F82B40F08B80036B8D
:107B1000F3B11847B02B6ED031D9D02B21D03ED93C
:107B2000E02B42D0F02B7ED1C3698BB1B0F8671047
:107B3000802900F1690028BF80211847FC2B0CD058
:107B400051D3FE2B4BD0FF2B6BD1436C002BE0D1DC
:107B50007047436B002BDCD1FAE7C36B002BD8D105
:107B6000F6E74369002BF3D090F8671090F86500B2
:107B70001847836A002BEBD090F867001847902BCA
:107B800029D0A02B23D0802BE2D10368002BDFD09B
:107B900090F8682090F8671090F865001847C02B9F
:107BA00042D10369002BDFD1D2E78269002ACFD00E
:107BB00090F8681090F8673090F86500C90101F4FA
:107BC0007E5103F07F031943A1F5005110478368EC
:107BD000002BDDD1BCE74368002BD9D1B8E7036C9B
:107BE000002B96D1B4E7836B002B92D1B0E7036AE8
:107BF000002BC1D1ACE7C368002BC9D1A8E7C36A89
:107C0000002B86D1A4E7426A002AA1D090F8683000
:107C100090F86700DB0103F47E5300F07F00184307
:107C20001047704770477047704700BF90F8643046
:107C3000DA0725D513F0FE0F22D070B590F8665004
:107C400085F08002602A82B004461AD9F62D66D0EB
:107C50005FD8F12D76D04FD9F22D2DD0F32D1AD13A
:107C6000806C94F86760036829461B689847A06C8D
:107C70000368DB6C06F07F0102B0BDE87040184776
:107C8000704790F865608E4207D031B15B08012BD8
:107C900008D0032B27D002B070BD5B08012B01D0A8
:107CA000022BF8D194F8683094F8672000962946A2
:107CB0002046FFF71DF9EEE7806C94F86730026804
:107CC00094F868601268294643EAC6159047A06C8C
:107CD000036805F07F019B6C9847A06C0368C5F3AF
:107CE000C6119B6CC8E794F8683094F8672000963A
:107CF0002946FFF7FDF8CEE7F02DCCD1B0F867109C
:107D0000802900F1690228BF80210123FFF7C8F80C
:107D1000C1E7FC2D2DD8FA2D01D2F82DBBD105F1EC
:107D20000803DBB2072BB6D8012202FA03F313F0E3
:107D3000DD0FB0D0294604F1480002B0BDE8704024
:107D4000F8F79EBC806C94F8672094F86830066859
:107D50001201294603F00F0302F0700532681D433B
:107D60009047A06C03681B68294602B0BDE87040CC
:107D70001847FE2D8FD3D2E7F0B54CF62C3087B0E4
:107D8000C1F6FF7007F066FC00287FD14FF2346423
:107D9000C2F200044DF6E445C1F6FF7595F84C605B
:107DA000102E1CD9002010F0D7FB0BF0ADFC4DF6C7
:107DB000A0600021C2F200000CF098FB4DF22003FD
:107DC00022680392C1F6FF73039A1868121A4FF2E1
:107DD0003461642AC2F200011ED807B0F0BD284603
:107DE000FFF70CFD0028DDD095F86630902B00F0F1
:107DF000358183F08003602B40F233814DF6E440FF
:107E0000C1F6FF70FFF772FE4DF6E4403146C1F651
:107E1000FF70FFF70BFFC5E70A680492049A1A6027
:107E2000FDF7C2FB4BF68413C1F6FF731B78002BE2
:107E300040F024814DF29C73C2F200031A78002AAC
:107E4000CBD04EF6F40122680592C2F20001059AE9
:107E5000086841F28831121A8A42BED949F2EF22EB
:107E6000C1F6FF720024204615781C700DF0FCFD51
:107E7000854203D0294620460DF010FE41F27C10C9
:107E8000C0F20200F8F72AFC07B0F0BD4CF66C1007
:107E9000C1F6FF7007F0DEFB00283FF477AF4DF628
:107EA0008416C1F6FF760EF0A7FB3368C01A4FF2B6
:107EB0003464B0F5356FC2F200047FF66BAF4DF25B
:107EC000A0750EF099FBC2F20005236801932A68A1
:107ED000019B30609B1A41F28832934200F2DB80B2
:107EE0004CF62C30C1F6FF7007F0C4FB06460028A4
:107EF00000F0D8804CF66C10C1F6FF7007F0BAFBAA
:107F00000746002800F0D5800EF076FB4BF21C23CC
:107F1000C2F200030546186803683A461B683146FA
:107F200098470EF069FB40F65A33401B984206D939
:107F30004CF6DC33C2F200031A6801321A604CF6C8
:107F40006C13C2F200031A88824238BF188072B6DE
:107F50004CF24033C2F200031A7F02F0FF010AB173
:107F600000221A7762B679B372B647F6FF754FF4FE
:107F70000040B3F91E10B3F92020DD83188462B6E7
:107F8000002982EAE273A3EBE273B8BF49428B4255
:107F9000B8BF0B4607EE903A4FF47E43C4F2FF633E
:107FA000F8EEE77A06EE903A87EEA67AF7EE007AD8
:107FB000B4EEE77AF1EE10FA06DD4CF27073C1F61A
:107FC000FF731A6801321A6072B64CF26023C2F273
:107FD00000031A7F02F0FF010AB100221A7762B68D
:107FE00079B372B647F6FF754FF40040B3F91E102F
:107FF000B3F92020DD83188462B6002982EAE27397
:10800000A3EBE273B8BF49428B42B8BF0B4607EE01
:10801000903A4FF47E43C4F2FF63F8EEE77A06EE3F
:10802000903A87EEA67AF7EE007AB4EEE77AF1EEB0
:1080300010FA06DD4CF27073C1F6FF731A68013254
:108040001A604CF62C30C1F6FF7007F025FB4CF699
:108050006C10C1F6FF7007F01FFB9BE695F86830C7
:1080600043B195F865309E423FF4C8AE002E3FF410
:10807000C5AEC9E6802385F86630F2E74BF21C23D3
:10808000C2F20003186804F021FC00287FF4D2AE8D
:10809000FEF7B4FBCEE6FEF74FFD23680293029B8A
:1080A0002B601DE741F24430C0F20200F8F716FBE6
:1080B00020E741F26C30C0F20200F8F70FFB23E733
:1080C0002DE9F04F4CF260448FB0C2F2000444F24C
:1080D000C016C2F200060DF075FC022320461022E5
:1080E0002721002509F0C2FA4FF060496FF060487F
:1080F0003046022203214EF28057FBF7B3FCC2F256
:108100000007C6F81490C6F81880357706F12000ED
:108110001D221C21FBF7A6FCC6F83490C6F8388057
:1081200086F83C503846142204210AF057FA07F129
:10813000100014221E210AF051FA4FF23463C2F2E9
:1081400000034DF698221B680A93C1F6FF720A9944
:1081500011604FF698734DF264302A46C0F2010365
:108160000121C1F6FF70FEF761FE01224FF6A473F4
:108170004DF220401146C0F20103C1F6FF70FEF738
:1081800055FE012241F210534DF2DC401146C0F27F
:108190000203C1F6FF70FEF749FE01224FF6B073ED
:1081A0004DF298501146C0F20103C1F6FF70FEF780
:1081B0003DFE01224FF6BC734DF254601146C0F2F1
:1081C0000103C1F6FF70FEF731FE01224FF6C473C2
:1081D0004DF21070C0F201031146C1F6FF70FEF7B8
:1081E00025FE4EF26870C2F200000AF0AFF84BF6BE
:1081F000FC2021460122C2F2000009F095FF41F265
:10820000AC634BF684102A46C0F202030121C2F28D
:10821000000049F24037FEF709FEC1F6FF77012260
:108220004CF2B0403B461146C2F20000FEF74EFD54
:108230004DF6D800C2F200000AF088F84AF6DC20B9
:1082400021460122C2F2000009F06EFF41F20853FC
:108250004AF2AC402A46C0F202030121C2F20000F9
:10826000FEF7E4FD012241F214734AF26850114610
:10827000C0F20203C2F20000FEF7D8FD012241F273
:108280001C734BF2C0001146C0F20203C2F20000A0
:10829000FEF7CCFD012241F264634AF2746011469C
:1082A000C0F20203C2F20000FEF7C0FD012241F25B
:1082B00028734AF230701146C0F20203C2F2000085
:1082C000FEF7B4FD012241F238734AF2EC70114618
:1082D000C0F20203C2F20000FEF7A8FD012241F243
:1082E00044734AF6A8001146C0F20203C2F200002D
:1082F000FEF79CFD012241F24C734AF664101146D0
:10830000C0F20203C2F20000FEF790FD012241F22A
:1083100054734AF62020C0F202031146C2F2000054
:10832000FEF784FD4BF22C30C2F200000AF00EF88A
:108330004CF2A45021460122C1F6FF7009F0F4FE70
:1083400041F2A4634BF24C202A46C0F20203012101
:10835000C1F6FF7049F2F826C1F6FF76FEF766FD1A
:1083600001224BF20830331D1146C1F6FF70FEF7B3
:10837000ADFC4BF64420C1F6FF7009F0E7FF4BF669
:10838000F44021460122C2F2000009F0CDFE4FF672
:10839000CC734BF260402A46C0F201030121C2F2C5
:1083A0000000FEF743FD01224BF21C50731D1146E5
:1083B000C2F20000FEF78AFC4CF22C20C1F6FF70DE
:1083C00009F0C4FF4CF60C1021460122C1F6FF70E3
:1083D00009F0AAFE41F2C8634BF608502A46C0F2E3
:1083E00002030121C1F6FF70FEF720FD01224BF6CA
:1083F000C450B31D1146C1F6FF70FEF767FC4BF287
:10840000CC10C2F2000009F0A1FF4DF62460214615
:108410000122C1F6FF7009F087FE41F244534DF688
:108420000C002A46C0F202030121C1F6FF70FEF7DC
:10843000FDFC01224DF6C800F31D1146C1F6FF7088
:10844000FEF744FC4CF67010C2F2000009F07EFF0B
:108450004BF2CC3021460122C2F2000009F064FE4A
:1084600041F20C734DF22C102A46C0F20203012196
:10847000C2F20000FEF7DAFC01224DF2E81006F12C
:1084800008031146C2F20000FEF75AFC4DF6BC206C
:10849000C2F2000009F05AFF4CF2D030214601220E
:1084A000C2F2000009F040FE41F2FC434BF60C0022
:1084B0002A46C0F202030121C2F20000FEF7B6FC18
:1084C00001224BF6D42006F109031146C1F6FF70D4
:1084D000FEF736FC4CF25450C1F6FF7009F036FF3F
:1084E0004DF6600021460122C2F2000009F01CFE98
:1084F00041F2F4634CF2D8302A46C0F20203012163
:10850000C1F6FF70FEF792FC012240F2FD534CF2DF
:108510009440C0F200031146C1F6FF70FEF74CFC18
:108520004CF6CC30C1F6FF7009F010FF4BF23C4026
:1085300021460122C1F6FF7009F0F6FD41F26C639D
:108540004CF248002A46C0F202030121C2F20000A8
:10855000FEF76CFC01224CF2041006F10B031146ED
:10856000C2F20000FEF7B2FB4BF67800C1F6FF70D6
:1085700009F0ECFE4DF2CC7021460122C1F6FF70ED
:1085800009F0D2FD41F2A8534DF2D8402A46C0F27C
:1085900002030121C2F20000FEF748FC01224DF661
:1085A000E05006F10C031146C2F20000FEF78EFB0C
:1085B0004CF2C010C2F2000009F0C8FE4DF62810BF
:1085C00021460122C2F2000009F0AEFD41F6180377
:1085D0004BF680602A46C0F202030121C1F6FF700B
:1085E000FEF724FC012241F628034BF63C701146AD
:1085F000C0F20203C1F6FF70FEF718FC012241F23F
:10860000C4534BF6F8701146C0F20203C1F6FF7076
:10861000FEF70CFC012241F2F0434CF2B40011468B
:10862000C0F20203C1F6FF70FEF700FC012241F226
:10863000D0534CF270101146C0F20203C1F6FF7025
:10864000FEF7F4FB01224FF63C734AF61450114634
:10865000C0F20103C2F20000FEF7E8FB01224FF670
:1086600048734AF68C601146C0F20103C2F2000062
:10867000FEF7DCFB012241F2F0534AF64870114646
:10868000C0F20203C2F20000FEF7D0FB012241F269
:1086900000634BF204001146C0F20203C2F2000074
:1086A000FEF7C4FB012241F2E8734CF6A0601146CC
:1086B000C0F20203C1F6FF70FEF7B8FB012241F2DF
:1086C000F8734CF65C701146C0F20203C1F6FF70FD
:1086D000FEF7ACFB012241F274634CF26C50114680
:1086E000C0F20203C2F20000FEF7A0FB012241F635
:1086F00008034CF268601146C0F20203C2F20000A7
:10870000FEF794FB012241F20C634DF22400114666
:10871000C0F20203C1F6FF70FEF788FB012241F2AE
:1087200080634DF2E0001146C0F20203C1F6FF7013
:10873000FEF77CFB012241F2C8734DF29C101146FA
:10874000C0F20203C1F6FF70FEF770FB012241F296
:1087500054634DF258201146C0F20203C1F6FF7077
:10876000FEF764FB012241F290634CF6B000114623
:10877000C0F20203C2F20000FEF758FB012241F2F0
:1087800098634BF29460C0F202031146C2F20000FB
:10879000FEF74CFB4BF24010C1F6FF7009F0D6FD1E
:1087A0004EF2B87021460122C2F2000009F0BCFC72
:1087B00041F2E4634AF658402A46C0F2020301211E
:1087C000C2F20000FEF732FB01224BF2901006F1DC
:1087D0000D031146C1F6FF70FEF778FA4EF2A05075
:1087E000C2F2000009F0B2FD4BF220402146012206
:1087F000C2F2000009F098FC41F278534DF6A01047
:108800002A46C0F202030121C2F20000FEF70EFB6D
:1088100001224DF6646006F10E031146C1F6FF70A9
:10882000FEF754FA4BF27C30C2F2000009F08EFDE4
:108830004DF25C0021460122C2F2000009F074FCF6
:108840004FF67C734DF294502A46C0F20103012189
:10885000C2F20000FEF7EAFA01224DF2506006F182
:108860000F031146C2F20000FEF730FA4CF60C205E
:10887000C1F6FF7009F06AFD4CF228602146012222
:10888000C2F2000009F050FC4FF658734BF2F4505E
:108890002A46C0F201030121C1F6FF70FEF7C6FAB5
:1088A000012240F26D434BF2B060C0F2000311466A
:1088B000C1F6FF70FEF780FA4BF63450C2F20000AA
:1088C00009F044FD4CF2704021460122C2F2000042
:1088D00009F02AFC41F26C734BF6D0602A46C0F2D4
:1088E00002030121C2F20000FEF7A0FA012240F2C9
:1088F0008D434BF68C70C0F200031146C2F20000AB
:10890000FEF75AFA4CF64C30C2F2000009F01EFD98
:108910004DF69C2021460122C1F6FF7009F004FCAF
:108920004FF670734DF6DC102A46C0F201030121A8
:10893000C1F6FF70FEF77AFA012240F2AD434CF225
:10894000CC20C0F200031146C1F6FF70FEF734FAE6
:108950004BF27C10C2F2000009F0F8FC4BF69420B8
:1089600021460122C1F6FF7009F0DEFB41F2A87337
:108970004BF220202A46C0F202030121C2F200007D
:10898000FEF754FA012240F229534CF65000C0F28F
:1089900000031146C1F6FF70FEF70EFA4DF20C709F
:1089A000C2F2000009F0D2FC4DF6881021460122E7
:1089B000C1F6FF7009F0B8FB41F2B8734DF61840EC
:1089C0002A46C0F202030121C2F20000FEF72EFA8D
:1089D000012240F275534DF6D440C0F20003114617
:1089E000C2F20000FEF7E8F94DF2DC00C2F200002E
:1089F00009F0ACFC4AF6184021460122C2F2000000
:108A000009F092FB4FF664734CF6D4102A46C0F27C
:108A100001030121C2F20000FEF708FA012240F230
:108A2000B9534CF69020C0F200031146C2F2000088
:108A3000FEF7C2F94EF6F800C2F2000009F086FC1B
:108A40004BF2001021460122C1F6FF7009F06CFBC9
:108A500041F2E0434CF61C402A46C0F202030121D9
:108A6000C1F6FF70FEF7E2F901224CF6204006F154
:108A700016031146C2F20000FEF728F94CF660001A
:108A8000C2F2000009F062FC4DF67C202146012272
:108A9000C2F2000009F048FB41F2B8634BF2BC702F
:108AA0002A46C0F202030121C1F6FF70FEF7BEF9AB
:108AB00001224BF6C80006F117031146C1F6FF70FC
:108AC000FEF704F94CF28830C1F6FF7009F03EFC65
:108AD0004DF29C0021460122C2F2000009F024FB65
:108AE0004FF688734BF27C402A46C0F20103012105
:108AF000C1F6FF70FEF79AF901224BF2385006F1E9
:108B000018031146C1F6FF70FEF7E0F84BF640601F
:108B1000C2F2000009F01AFC4CF264302146012236
:108B2000C2F2000009F000FB41F2FC634CF6DC40AD
:108B30002A46C0F202030121C2F20000FEF776F9D4
:108B400001224CF6985006F119031146C2F20000BA
:108B5000FEF7BCF84DF26030C2F2000009F0F6FBFF
:108B60004CF6E03021460122C2F2000009F0DCFAA6
:108B700041F228634BF688102A46C0F20203012115
:108B8000C1F6FF70FEF752F901224AF6D05006F105
:108B90001A031146C2F20000FEF798F84BF21C00CF
:108BA000C1F6FF7009F0D2FB4DF6E83021460122F4
:108BB000C1F6FF7009F0B8FA41F218534CF2F850C0
:108BC0002A46C0F202030121C1F6FF70FEF72EF91A
:108BD00001224CF2B46006F11B031146C1F6FF708E
:108BE000FEF774F84CF65060C1F6FF7009F0AEFB6A
:108BF0004CF6200021460122C2F2000009F094FA4E
:108C000041F234534CF6E4602A46C0F202030121DB
:108C1000C2F20000FEF70AF901224DF62C3006F1EF
:108C20001C031146C1F6FF70FEF750F84BF26C7052
:108C3000C1F6FF7009F08AFB4EF6B400214601220E
:108C4000C2F2000009F070FA41F298734AF61C3043
:108C50002A46C0F202030121C2F20000FEF7E6F844
:108C600001224BF2D85006F11D031146C2F200005A
:108C7000FEF72CF84DF60C30C2F2000009F066FB4E
:108C80004CF6A46021460122C2F2000009F04CFA21
:108C900041F264734EF2F8702A46C0F202030121D9
:108CA000C2F20000FEF7C2F801224DF2A42006F144
:108CB0001E031146C2F20000FEF742F84CF21040CB
:108CC000C2F2000009F042FB4DF6D05021460122CD
:108CD000C1F6FF7009F028FA41F28C734CF65C2063
:108CE0002A46C0F202030121C1F6FF70FEF79EF88A
:108CF00001224CF6A07006F11F031146C2F20000DB
:108D0000FEF71EF84DF69050C2F2000009F01EFB6F
:108D10004AF6D83021460122C2F2000009F004FAD6
:108D200041F228534EF2F0502A46C0F202030121CC
:108D3000C2F20000FEF77AF801224EF2AC603B4628
:108D40001146C2F20000FDF7C1FF4CF21020C2F242
:108D5000000009F0FBFA4BF63C3021460122C2F23A
:108D6000000009F0E1F941F2B8534BF250702A4685
:108D7000C0F202030121C2F20000FEF757F80122FF
:108D800041F288534BF6C8001146C0F20203C2F20A
:108D90000000FEF74BF8012241F298534DF62840AF
:108DA0001146C0F20203C1F6FF70FEF73FF8012240
:108DB00041F27C734BF64020C0F202031146C2F22E
:108DC0000000FEF733F84BF2DC20C2F2000009F09D
:108DD000BDFA4BF6906021460122C2F2000009F074
:108DE000A3F941F21C634BF64C402A46C0F2020341
:108DF0000121C1F6FF70FEF719F801224BF6903001
:108E000006F120031146C1F6FF70FDF75FFF4DF23A
:108E10001430C1F6FF7009F099FA4DF25C702146EA
:108E20000122C2F2000009F07FF941F2E0534BF653
:108E30008450C0F2020300220121C2F20000FDF7BB
:108E4000F5FF012240F231634CF22470C0F20003BE
:108E50001146C2F20000FDF7AFFF4DF6DC20C1F66F
:108E6000FF7009F073FA4DF2B03021460122C2F2D0
:108E7000000009F059F941F2D4634CF6D840C0F231
:108E8000020300220121C1F6FF70FDF7CFFF01228E
:108E900040F2D1434CF69450C0F200031146C1F6A3
:108EA000FF70FDF789FF4BF26C00C1F6FF7009F00F
:108EB0004DFA4BF2C00021460122C1F6FF7009F0C5
:108EC00033F941F2D8734BF67C30C0F20203002232
:108ED0000121C2F20000FDF7A9FF01224BF6384044
:108EE00006F123031146C2F20000FDF7EFFE4AF23D
:108EF0002460C2F2000009F029FA4DF2F030214658
:108F00000122C2F2000009F00FF9002241F2386399
:108F10004CF284201146C0F20203C2F20000FDF7B9
:108F200085FF41F248634CF29470C0F202030122C3
:108F30000021C1F6FF70FDF779FF4CF65460C2F2D4
:108F4000000009F003FA4CF2E07021460122C2F25F
:108F5000000009F0E9F841F258534DF2A470C0F254
:108F6000020300220121C2F20000FDF75FFF01228F
:108F700049F2EF234DF65C30C1F6FF731146C2F2A1
:108F80000000FDF7A3FE4CF27C20C1F6FF7009F053
:108F9000DDF94CF69C3021460122C2F200004DF66C
:108FA000E449C1F6FF7909F0BFF84DF230400121E4
:108FB000C2F2000009F098FA99F86430012243F0F7
:108FC000010362F3470349F2A025002489F86430C5
:108FD00049F214562B464FF6FF7E214689F865402C
:108FE00089F8664089F8674089F8684089F8E9405F
:108FF000C1F6FF73C1F6FF7609F1690080221D46B4
:10900000C9F85CE0C9F860E0C9F8486089F84C40EC
:1090100089F84D4089F84E40C9F85440C9F8584085
:109020004DF6A06613F048FB40F225514CF62C3368
:10903000C2F200062A46C1F6FF734846C0F200019C
:109040004FF6387A0195C9F800401D46C9F804402A
:10905000C9F80840C9F80C40C9F81040C9F81440D4
:10906000C9F81840C9F81C40C9F82040C9F8244084
:10907000C9F82840C9F82C40C9F83040C9F8344034
:10908000C9F83840C9F83C40C9F84040C9F84440E4
:10909000C0F20E0A12F09CFF06F5A36C06F5AB6E4B
:1090A00006F5B361502306F59B694022C6F818C047
:1090B000C6F81CE0B38574603046B460C6F800A002
:1090C000C6F81490716272850BF0D4F84CF24032FD
:1090D00002924FF6E862C0F2010232602146224657
:1090E0002846F9F7D1FD029A85F89C404CF66C1B96
:1090F000C1F6FF7BC2F200024FF6D4584CF2602357
:10910000C2F20003C0F20E080292214622465846DF
:109110000393C5F8984085F89D400695C5F80080F2
:10912000F9F7B2FD02998BF89C4044F20C200A46F4
:1091300089460546183208460121CBF80080CBF855
:1091400098408BF89D40F9F79FFD0399CDF8089062
:10915000C2F200054DF6207307950A464DF62075BC
:109160004FF678478A461832C0F20E0747F6FF7668
:109170004FF40048059508461D460121C9F80070C6
:10918000A9F81E60A9F82080C1F6FF75F9F77CFDEB
:109190004DF668190798CAF80070C2F20009AAF8DB
:1091A0001E60CDF80CA0AAF8208005F04FFD4DF60A
:1091B000A00A2846C2F2000A05954CF64C1705F0A5
:1091C00045FD4FF6BC5609F12802484604214CF2F1
:1091D0007475F9F759FD4FF48033C1F6FF77C0F28B
:1091E0000E060AF1280250460421C1F6FF75C9F89F
:1091F0000060C9F81830C9F81C30C9F82030C9F827
:10920000243008930495F9F73FFD089BCAF80060E5
:1092100007F11C02384601213D46CAF81830CAF849
:109220001C30CAF82030CAF82430F9F72DFD049F0D
:10923000089BAB6107F11C02089538462F464FF694
:10924000B055C0F20E05012109933D604DF6C818D6
:10925000F9F71AFD0499099B029A0D60C1F6FF788F
:1092600040F22566C0F20006069D8B6140464BF237
:10927000C437C1F6FF77C8F80420C8F8005088F852
:10928000084088F80940C8F80C4088F810400BF0F6
:1092900059FD019A314640464BF2D83812F098FEFB
:1092A000C1F6FF78039979603846C7F800B03C7280
:1092B0007C72FC603C740BF045FD019A31463846E7
:1092C00012F086FE4BF2EC3740460695C8F8005087
:1092D000079DC8F80450C1F6FF7788F8084088F861
:1092E0000940C8F80C4088F810400BF02BFD3146BF
:1092F000019A404612F06CFE059AC7F800B0384655
:109300007A603C727C72FC603C744BF200480BF05B
:1093100019FD019A3146384612F05AFEC1F6FF781F
:10932000069B88F8084040464BF2144788E808023C
:10933000C1F6FF7788F80940C8F80C4088F810405B
:109340000BF000FD019A3146404612F041FE3846CE
:10935000C7F800B0C7F804A03C727C72FC603C7493
:109360000BF0F0FCDDF804B04BF22848C1F6FF78B2
:109370005A463146384612F02BFE294640464FF0F9
:10938000010588E8020288F8084088F80950C8F802
:109390000C4088F810404DF610670BF0D3FC5A468D
:1093A0003146404612F014FEC1F6FF77059B3C7231
:1093B00038464CF2E458C1F6FF7887E808047D721D
:1093C000FC603C740BF0BEFC5A463146384612F045
:1093D000FFFD4BF20C47089BC8F804304046C2F230
:1093E0000007C8F8009088F8084088F80940C8F8D5
:1093F0000C4088F810400BF0A5FC5A463146404618
:1094000012F0E6FD4DF65C28049DC7F800A0384632
:10941000C2F200087D603C727C72FC603C740BF010
:1094200091FC5A463146384612F0D2FD08F1180236
:1094300002214046F9F728FC4FF6C853C0F20E034C
:1094400040464CF61839C1F6FF79C8F8003005F0EF
:1094500081FF089B89F8084048464CF6C017C2F2C5
:10946000000789E8080189F80940C9F80C4089F823
:1094700010400BF067FC31465A46484612F0A8FDF2
:109480002A464FF00103384687E804017B723C729C
:10949000FC603C740BF056FC31465A46384612F0DC
:1094A00097FD44F20023C2F200034FF68442C0F25B
:1094B0000E021A600A221A720DF09EF84FF23463FF
:1094C000C2F200034DF684151A680B92DDF82CC029
:1094D0001A680C92DDF830E01B680D934DF2200401
:1094E0004EF6F4014DF2A0724BF2BC03C1F6FF75CB
:1094F000C1F6FF74C2F20001C2F200020D9F2860A3
:10950000C1F6FF734DF66266C3F64E76C4F800C02E
:10951000C1F800E017601E600FB0BDE8F08F00BF1B
:109520002DE9F04F4CF26044C2F2000493B02046A3
:1095300008F066FC204608F00BFA204608F000FA16
:10954000204608F0A3F8204608F0E6FA204600225C
:10955000012108F0D1F941F294312046C0F2020114
:109560000E220BF0B9FF20460122002108F0C4F9B9
:1095700041F2A4311022C0F2020120464DF2643AB9
:109580004EF268740BF0A8FFC2F20004C1F6FF7A35
:109590004FF47A704DF220490DF056F8C1F6FF797C
:1095A000514620464DF2DC4808F0D8FEC1F6FF785F
:1095B000494620464DF2985708F0D0FEC1F6FF7795
:1095C000414620464DF2546608F0C8FEC1F6FF76CB
:1095D000394620464DF2107508F0C0FEC1F6FF7501
:1095E0003146204608F0BAFE4BF6FC2329462046B9
:1095F000019308F0B3FE019B2046C2F20003022152
:10960000019308F0E1FE2146019808F099FD41F62A
:109610006D725046C0F20002012108F005FC42F6CE
:109620004D324846C0F20002022108F0FDFB40F630
:1096300009424046C0F20002032108F0F5FB40F663
:10964000A5723846C0F20002042108F0EDFB42F694
:1096500091223046C0F20002052108F0E5FB40F2FD
:10966000BD72C0F20002284606214DF6D80408F06B
:10967000DBFBC2F200044BF684112046C2F200016B
:1096800008F06CFE4AF6DC224CF2B041154620464A
:10969000C2F2000108F062FE2A46C2F2000216463B
:1096A0004AF2AC4220461746022108F08DFE3A46A7
:1096B000C2F200024BF22C35C2F2000517462146D9
:1096C00030464AF2685B0F96C2F2000B08F038FD94
:1096D0004BF2C00A394628460497C2F2000A08F045
:1096E0003DFE4AF274695946284608F037FEC2F238
:1096F0000009514628464AF2307808F02FFEC2F29F
:1097000000084946284608F029FE4AF2EC7741460F
:10971000284608F023FEC2F200074AF664123946D2
:10972000144628464AF6A80608F018FEC2F20006BB
:109730002246C2F20002314628464AF6202403920D
:10974000C2F2000408F00AFE0399284608F006FE5B
:109750004CF2A45321462846029308F0FFFD029BD9
:109760002846C1F6FF730221029308F02DFE294618
:10977000029808F0E5FC41F6ED620498C0F20002A0
:10978000072108F051FB41F6ED425846C0F20002B5
:10979000082108F049FB41F6ED525046C0F20002A4
:1097A000092108F041FB41F66D324846C0F2000243
:1097B0000A2108F039FB41F2E1724046C0F2000292
:1097C0000B2108F031FB41F665023846C0F2000279
:1097D0000C2108F029FB41F2D5623046C0F20002AC
:1097E0000D2108F021FB41F66D520398C0F20002F2
:1097F0000E2108F019FB41F2D552C0F200022046BA
:109800000F214BF6442508F00FFBC1F6FF754BF214
:109810004C212846C1F6FF7108F0A0FD4BF6F4423A
:109820004BF2083114462846C1F6FF7108F096FD48
:109830002246C2F2000217462846022108F0C4FD63
:109840004CF22C2429463846C1F6FF74109708F0D4
:1098500077FC4BF260412046C2F2000108F07EFD29
:109860004BF21C512046C2F2000108F077FD204661
:10987000022108F0A9FD4CF60C102146C1F6FF703C
:109880004BF2CC1408F05CFCC2F200044BF6085119
:109890002046C1F6FF7108F061FD4BF6C451204629
:1098A000C1F6FF7108F05AFD2046022108F08CFD38
:1098B0004DF624602146C1F6FF704CF6701408F096
:1098C0003FFCC2F200044DF60C012046C1F6FF71C8
:1098D00008F044FD4DF6C8012046C1F6FF7108F0BE
:1098E0003DFD2046022108F06FFD4BF2CC302146B1
:1098F000C2F200004DF6BC2408F022FCC2F20004C3
:109900004DF22C112046C2F2000108F027FD4DF265
:10991000E8112046C2F2000108F020FD2046022195
:1099200008F052FD4CF2D0302146C2F200004CF259
:10993000545408F005FCC1F6FF744BF60C012046A8
:10994000C2F2000108F00AFD4BF6D4212046C1F610
:10995000FF7108F003FD2046022108F035FD4DF6A9
:1099600060002146C2F200004CF6CC3408F0E8FB5F
:10997000C1F6FF744CF2D8312046C1F6FF7108F0F1
:10998000EDFC4CF294412046C1F6FF7108F0E6FC74
:109990002046022108F018FD4BF23C402146C1F65A
:1099A000FF704BF6780408F0CBFBC1F6FF744CF265
:1099B00048012046C2F2000108F0D0FC4CF204112C
:1099C0002046C2F2000108F0C9FC2046022108F03E
:1099D000FBFC4DF2CC702146C1F6FF704CF2C01476
:1099E00008F0AEFBC2F200044DF2D8412046C2F2AC
:1099F000000108F0B3FC4DF6E0512046C2F2000130
:109A000008F0ACFC2046022108F0DEFC4DF62810E0
:109A10004BF680632146C1F6FF73C2F20000039348
:109A20004BF2401408F08CFB039B1193C1F6FF74BA
:109A30004BF63C7B1946C1F6FF7B20464BF6F87A85
:109A400008F08CFCC1F6FF7A594620464CF2B40966
:109A500008F084FCC1F6FF79514620464CF270189C
:109A600008F07CFCC1F6FF78494620464AF61457B8
:109A700008F074FCC2F20007414620464AF68C66A4
:109A800008F06CFCC2F200063946204608F066FC7D
:109A900031464BF20402204603924AF6487508F01C
:109AA0005DFC039AC2F200054CF6A06EC2F2000201
:109AB00029462046CDF810E0039208F04FFC0498A8
:109AC0000399C1F6FF7004904CF65C722046059233
:109AD00008F044FC059A0499C1F6FF724CF26C5EE2
:109AE00020460592CDF818E008F038FC069B059951
:109AF000C2F200034CF2686E20460693CDF81CE0DB
:109B000008F02CFC079A0699C2F200024DF2240ECE
:109B100020460792CDF820E008F020FC089B07992A
:109B2000C1F6FF734DF2E00E20460893CDF824E015
:109B300008F014FC099A0899C1F6FF724DF29C1EB8
:109B400020460992CDF828E008F008FC0A9B099904
:109B50009E46C1F6FF7ECDF828E020464DF2582EF5
:109B6000CDF82CE008F0FAFB0B9A0A999646C1F65C
:109B7000FF7ECDF82CE020464CF6B00ECDF830E05C
:109B800008F0ECFB0C9B0B999E46C2F2000ECDF840
:109B900030E020464BF2946ECDF834E008F0DEFB66
:109BA0000D9A0C999646C2F2000E2046CDF834E08C
:109BB00008F0D4FB0D994EF2B87E2046CDF838E07F
:109BC00008F0CCFB0E9A9646C2F2000E2046022107
:109BD000CDF838E008F0F8FB21460E9808F0B0FA0E
:109BE000119B41F6ED321846C0F20002102108F038
:109BF0001BF941F2D1325846C0F20002112108F09F
:109C000013F941F66D625046C0F20002122108F0CD
:109C10000BF941F6F1024846C0F20002132108F0A8
:109C200003F941F66D424046C0F20002142108F0EB
:109C3000FBF841F2DD423846C0F20002152108F07F
:109C4000F3F841F2D1223046C0F20002162108F0AA
:109C5000EBF841F245122846C0F20002172108F045
:109C6000E3F841F671220398C0F20002182108F0CF
:109C7000DBF841F6F1120498C0F20002192108F055
:109C8000D3F841F671120598C0F200021A2108F0CB
:109C9000CBF841F251220698C0F200021B2108F0D5
:109CA000C3F840F201720798C0F200021C2108F0CC
:109CB000BBF841F255520898C0F200021D2108F08D
:109CC000B3F841F251320998C0F200021E2108F0A7
:109CD000ABF841F255620A98C0F200021F2108F069
:109CE000A3F841F261720B98C0F20002202108F043
:109CF0009BF841F251420C98C0F20002212108F079
:109D000093F841F2C512C0F200020D9822214EF2E2
:109D1000A05408F089F8C2F200044AF658412046DF
:109D2000C2F2000108F01AFB4BF290112046C1F676
:109D3000FF7108F013FB2046022108F045FB4BF2AF
:109D400020402146C2F200004BF27C3408F0F8F9C2
:109D5000C2F200044DF6A0112046C2F2000108F044
:109D6000FDFA4DF664612046C1F6FF7108F0F6FA7F
:109D70002046022108F028FB4DF25C002146C2F289
:109D800000004CF60C2408F0DBF9C1F6FF744DF22C
:109D900094512046C2F2000108F0E0FA4DF2506101
:109DA0002046C2F2000108F0D9FA2046022108F04C
:109DB0000BFB4CF228602146C2F200004BF63454F3
:109DC00008F0BEF9C2F200044BF2F4512046C1F68D
:109DD000FF7108F0C3FA4BF2B0612046C1F6FF7183
:109DE00008F0BCFA2046022108F0EEFA4CF270406E
:109DF0002146C2F200004CF64C3408F0A1F9C2F240
:109E000000044BF6D0612046C2F2000108F0A6FA29
:109E10004BF68C712046C2F2000108F09FFA2046F2
:109E2000022108F0D1FA4DF69C202146C1F6FF70C0
:109E30004BF27C1408F084F9C2F200044DF6DC11F8
:109E40002046C1F6FF7108F089FA4CF2CC21204679
:109E5000C1F6FF7108F082FA2046022108F0B4FA38
:109E60004BF694202146C1F6FF704DF20C7408F0B9
:109E700067F9C2F200044BF220212046C2F2000131
:109E800008F06CFA4CF650012046C1F6FF7108F05C
:109E900065FA2046022108F097FA4DF6881021460F
:109EA000C1F6FF704DF2DC0408F04AF9C2F200047A
:109EB0004DF618412046C2F2000108F04FFA4DF667
:109EC000D4412046C2F2000108F048FA204602219F
:109ED00008F07AFA4AF618402146C2F200004EF61F
:109EE000F80408F02DF9C2F200044CF6D411204613
:109EF000C2F2000108F032FA4CF690212046C2F27C
:109F0000000108F02BFA2046022108F05DFA4BF21E
:109F100000102146C1F6FF704CF6600408F010F9FD
:109F2000C2F200044CF61C412046C1F6FF7108F055
:109F300015FA4CF620412046C2F2000108F00EFA54
:109F40002046022108F040FA4DF67C202146C2F25C
:109F500000004CF2883408F0F3F8C1F6FF744BF2BD
:109F6000BC712046C1F6FF7108F0F8F94BF6C80144
:109F70002046C1F6FF7108F0F1F92046022108F0F1
:109F800023FA4DF29C002146C2F200004BF64064D9
:109F900008F0D6F8C2F200044BF27C412046C1F62C
:109FA000FF7108F0DBF94BF238512046C1F6FF7122
:109FB00008F0D4F92046022108F006FA4CF2643089
:109FC0002146C2F200004DF2603408F0B9F8C2F246
:109FD00000044CF6DC412046C2F2000108F0BEF954
:109FE0004CF698512046C2F2000108F0B7F920461D
:109FF000022108F0E9F94CF6E0302146C2F20000F7
:10A000004BF21C0408F09CF8C1F6FF744BF6881163
:10A010002046C1F6FF7108F0A1F94AF6D05120465A
:10A02000C2F2000108F09AF92046022108F0CCF9AA
:10A030004DF6E8302146C1F6FF704CF6506408F04A
:10A040007FF8C1F6FF744CF2F8512046C1F6FF715B
:10A0500008F084F94CF2B4612046C1F6FF7108F0B3
:10A060007DF92046022108F0AFF94CF62000214688
:10A07000C2F200004BF26C7408F062F8C1F6FF7493
:10A080004CF6E4612046C2F2000108F067F94DF693
:10A090002C312046C1F6FF7108F060F920460221FC
:10A0A00008F092F94EF6B4002146C2F200004DF6D7
:10A0B0000C3408F045F8C2F200044AF61C31204680
:10A0C000C2F2000108F04AF94BF2D8512046C2F220
:10A0D000000108F043F92046022108F075F94CF61A
:10A0E000A4602146C2F200004CF2104408F028F8A7
:10A0F000C2F200044EF2F8712046C2F2000108F0EC
:10A100002DF94DF2A4212046C2F2000108F026F9F3
:10A110002046022108F058F94DF6D0502146C1F6EC
:10A12000FF704DF6905408F00BF8C2F200044CF6A4
:10A130005C212046C1F6FF7108F010F94CF6A071C1
:10A140002046C2F2000108F009F92046022108F079
:10A150003BF94AF6D8302146C2F200004CF21025F5
:10A1600007F0EEFFC2F200054EF2F0512846C2F2AF
:10A17000000108F0F3F84BF63C344EF2AC6128468F
:10A18000C2F20001C2F2000408F0E8F826462846B0
:10A1900002214BF250784BF2DC2408F015F9C2F2A0
:10A1A0000004C2F20008294630464BF6C807049660
:10A1B000C2F2000707F0C4FF4DF62846414620468C
:10A1C00008F0CCF8C1F6FF763946204608F0C6F80C
:10A1D0004BF640253146204608F0C0F8C2F2000593
:10A1E0004BF6906003902946204608F0B7F8039894
:10A1F000C2F2000003900221204608F0E5F8214653
:10A20000039807F09DFF40F625724046C0F2000219
:10A21000232107F009FE41F2C5023846C0F20002D0
:10A22000242107F001FE41F6F1223046C0F200027F
:10A23000252107F0F9FD41F23502C0F2000228465F
:10A2400026214DF2143407F0EFFDC1F6FF744BF6F2
:10A250004C412046C1F6FF7108F080F84BF6903172
:10A260002046C1F6FF714DF25C7B08F077F8C2F230
:10A27000000B2046022108F0A7F84DF6DC25214608
:10A28000584607F05DFFC1F6FF754BF6845128462E
:10A29000C2F2000108F062F84CF224712846C2F2C2
:10A2A00000014DF2B03A08F059F8C2F2000A28460F
:10A2B000022108F089F84BF26C042946504607F059
:10A2C0003FFFC1F6FF744CF6D8412046C1F6FF713E
:10A2D00008F044F84CF694512046C1F6FF714BF259
:10A2E000C00908F03BF8C1F6FF792046022108F0CA
:10A2F0006BF84AF224652146484607F021FFC2F276
:10A3000000054BF67C312846C2F2000108F026F821
:10A310004BF638412846C2F200014DF2F03808F001
:10A320001DF8C2F200082846022108F04DF84CF64C
:10A3300054642946404607F003FFC2F200044CF281
:10A3400084212046C2F2000108F008F84CF2947112
:10A350002046C1F6FF714CF2E07707F0FFFFC2F232
:10A3600000072046022108F02FF84CF27C252146F8
:10A37000384607F0E5FEC1F6FF754DF2A471284698
:10A38000C2F2000107F0EAFF4DF65C312846C2F246
:10A3900000014CF69C3607F0E1FFC2F200062846A9
:10A3A00002214DF23044C2F2000408F00DF82946B3
:10A3B000304607F0C5FE0199204608F09DF80F9938
:10A3C000204608F099F80299204608F095F80E9971
:10A3D000204608F091F81099204608F08DF84CF6C8
:10A3E0000C112046C1F6FF7108F086F84DF6246185
:10A3F0002046C1F6FF7108F07FF84BF2CC312046C1
:10A40000C2F2000108F078F84CF2D0312046C2F2D6
:10A41000000108F071F84DF660012046C2F200011B
:10A4200008F06AF84BF23C412046C1F6FF7108F093
:10A4300063F84DF2CC712046C1F6FF7108F05CF86C
:10A440004DF628112046C2F2000108F055F84EF2F0
:10A45000B8712046C2F2000108F04EF84BF22041DC
:10A460002046C2F2000108F047F84DF25C01204698
:10A47000C2F2000108F040F84CF228612046C2F216
:10A48000000108F039F84CF270412046C2F2000198
:10A4900008F032F84DF69C212046C1F6FF7108F015
:10A4A0002BF84BF694212046C1F6FF7108F024F8F2
:10A4B0004DF688112046C1F6FF7108F01DF84AF6E6
:10A4C00018412046C2F2000108F016F84BF20011C4
:10A4D0002046C1F6FF7108F00FF84DF67C212046AA
:10A4E000C2F2000108F008F84DF29C012046C2F2C9
:10A4F000000108F001F84CF264312046C2F200017C
:10A5000007F0FAFF4CF6E0312046C2F2000107F0F6
:10A51000F3FF4DF6E8312046C1F6FF7107F0ECFF7E
:10A520004CF620012046C2F2000107F0E5FF4EF68E
:10A53000B4012046C2F2000107F0DEFF4CF6A46130
:10A540002046C2F2000107F0D7FF4DF6D051204659
:10A55000C1F6FF7107F0D0FF4AF6D8312046C2F2AB
:10A56000000107F0C9FF0499204607F0C5FF0399D1
:10A57000204607F0C1FF5946204607F0BDFF51466F
:10A58000204607F0B9FF4946204607F0B5FF41468F
:10A59000204607F0B1FF3946204607F0ADFF3146AF
:10A5A000204607F0A9FF2046022107F0DFFF4CF20A
:10A5B000A4362046012107F0D3FFC2F20006204650
:10A5C0004EF2805507F0F6FFC2F200052922FF2166
:10A5D000304612F071F800242846347008F016F85E
:10A5E00005F1100008F012F820460BF03DFA49F290
:10A5F000EF2144F2C013C2F20003C1F6FF716322DF
:10A6000008701C775C619A6172B69042A8BF1046D0
:10A610008000D86062B64DF21802C1F6FF72087869
:10A6200083F83C4005215C631060996372B6DC627C
:10A6300062B6546013B0BDE8F08F00BF70B5022160
:10A6400082B004200BF09CFF02211E200BF098FF2B
:10A65000FEF766FF41F2B830C0F20200F6F73EF8AE
:10A6600041F2FC30C0F20200F6F738F841F22C401B
:10A67000C0F20200F6F732F841F25C40C0F202008C
:10A6800049F2E465F6F720F8C1F6FF754EF2244171
:10A690000A22C0F20C01002328460AF0A3FF41F26F
:10A6A0007040C0F20200F6F719F828460AF088FF59
:10A6B00041F27840C0F20200F6F710F840F6E440AC
:10A6C0000BF0B2FC044600F02FFC4BF21C23C2F24C
:10A6D000000301261C60FCF755F9FAF7FDFAFAF7BA
:10A6E000B7FC4EF28813CEF2000340F2002044F291
:10A6F00000241E60C2F200048021C1F6FF700AF03F
:10A70000C3F9204603F0B8FC204602F071FDB7EE15
:10A71000000A204603F08AF9E288242122F0100280
:10A72000204602F0BDFBF6EE000AB0EE600A2046BD
:10A7300002F058FEE288204622F48072242102F0C2
:10A74000AFFB1D21204602F0C9FD204603F0EAFAC6
:10A750000221204602F0D6FC204602F051FC2046A1
:10A7600002F0CCFB41F28840C0F20200F5F7B6FFE0
:10A7700049F2EF23C1F6FF734FF20E641878FAF72F
:10A7800007FE4FF20C61C2F200044FF20862C2F2FF
:10A7900000014FF28C53C2F20002C2F2000341F2F8
:10A7A000A440248809881480C0F202001980F5F7BB
:10A7B0008BFF802128460AF0A5FE41F2BC40C0F282
:10A7C0000200F5F781FF40F65A3128460AF09AFE5A
:10A7D00041F2D040C0F20200F5F780FF4EF20813BC
:10A7E000CEF2000341F2D4401E60C0F20200F5F741
:10A7F00075FF28460AF0E4FEFCF79EF94FF234623A
:10A80000C2F200024DF2A07312680192C2F200037C
:10A81000019A1A6002B070BD2DE9F04F2DED068B44
:10A820004BF2BC03844683B0C1F6FF7300F6A84424
:10A8300093ED000AD4ED008ADCF87CEC9FEDA35A7E
:10A84000DFEDA30A0CF6944300F6C44500F6AC49CC
:10A8500000F54B681C4600F6A44001930CF69C439F
:10A860000CF5496B90ED008A93ED00AAD5ED004AF6
:10A8700099ED003AD8ED003ADBED002A94ED004A5C
:10A880000CF54A630CF69840D3ED009A90ED001A4F
:10A8900002F1FE030239A2F1020A0093F6EE001A59
:10A8A000B7EE002ABFEE009ABEF1000F9FED896A55
:10A8B00040F30881DCF8806CF0EE465A0CF53C70F1
:10A8C000002550F8307C50F8343C50F82C2C50F8CF
:10A8D000284C3B4402EB234201359BB2A2422DB2ED
:10A8E00040F82C2C40F8303C04DD50F8244C121B6E
:10A8F00040F82C2C06EB420436F91220B4F9027011
:10A9000010ED087A50ED076ABF1A03FB07F302EB5C
:10A91000234307EE903AF8EEE77A67EE266A67EE91
:10A92000877A40ED086A67EE857AF5EEC07AF1EE37
:10A9300010FA0EDD24EEA77AE7EEC77AB0EE677A5A
:10A94000F1EE667AB4EEE77AF1EE10FA58BFF0EE67
:10A95000477A50ED036A10ED027A7545E7EEA65A84
:10A9600000F13400A7EE876AABDB36EE637A75EE52
:10A97000C37AE7EE283A019BA7EEA83AE1EE042A53
:10A9800036EE637AA2EEC14AA7EE086A75EEC37A84
:10A9900026EE297AE7EE885AA4EE076A65EE8A7AEF
:10A9A00026EE216AE4EE275AB4EEC26AF1EE10FAFE
:10A9B00089ED003A65EEA15AC8ED003ACBED002AC8
:10A9C00083ED004A76DDB7EE006AF4EEC25AF1EE8E
:10A9D00010FA67DDF7EE005A65EE805A26EE006A3F
:10A9E00065EEA05A26EE206AFDEEE57A17EE902A73
:10A9F000FDEEC67A2AF8022F17EE903A21F8023FB0
:10AA0000009B9A457FF450AFDFED337AB0EEC33A46
:10AA1000B4EEE73ADFED307AF1EE10FAF0EEE33A19
:10AA200048BF0023F4EEE73A48BFC9F80030F1EE22
:10AA300010FA44BF0023C8F80030BEF1000F2CDD2F
:10AA400000239FED267A1E46342706E0DCF87CECD6
:10AA5000013636B2764533461FDA07FB03C3D3ED22
:10AA6000B47A0EF1FF3EF4EEC77A07FB0EC4F1EEA6
:10AA700010FA04F52F7403F52F75E7D50FCCCCF839
:10AA80007CEC0FC50FCC0FC50FCC0FC5013636B20D
:10AA900023682B6076453346DFDB03B0BDEC068BC5
:10AAA000BDE8F08FF4EE495AF1EE10FA48BFF0EE2F
:10AAB000495A91E7B4EE496AF1EE10FA48BFB0EE98
:10AAC000496A82E7F0EE465A4FE700BF00000038BF
:10AAD00000FEFF4600000000FFE6DB2E17B7D1386E
:10AAE00041689FED157AD1ED056ADFED147AE6EE47
:10AAF000877A4FF4884243F2C673C4F22C72C3F2D1
:10AB0000BE7310B58260C360044617EE900A10F061
:10AB10004FFD41EC100B0FF097F851EC100B11F0BA
:10AB200093F8DFED077A07EE100A67EE277A04F64E
:10AB30009844C4ED007A10BD3D0AC7403D0A27C0C5
:10AB4000716415392DE9F84307292DED028B46680C
:10AB50005DD00FD9402901D0422936D102F04004FE
:10AB6000E4B2C0F88C4C002C64D0BDEC028B012008
:10AB7000BDE8F883012928D107EE902ADFED506A5D
:10AB80009FED507AF8EE677A00F6DC4367EEA67A1E
:10AB9000F4EEC77AF1EE10FAC3ED007AE5DD00F6C7
:10ABA0009C4300F54A60C3ED007AC0ED007AD6ED13
:10ABB000046AB6EE007AF4EEC76AF1EE10FAD4D564
:10ABC000F1EE677AC0ED007ACFE77A29CDD9037C20
:10ABD0007BB103EB430203EB820247F2A401C3F60D
:10ABE0007D7100EB82020346C3F8D41234339A42DB
:10ABF000FAD1BDEC028B00F6C8430022C4F2203229
:10AC00000021C0F88C1C01201A60BDE8F88312FBFB
:10AC100002F207EE902ABDEC028BF8EEE77A9FED88
:10AC20002A7A67EE877A00F6D840C0ED007A0120D4
:10AC3000BDE8F883027C002A97D007460546B1EEAE
:10AC4000048A03E0A24205F134058EDDD5F8EC322A
:10AC5000802B04F10104F5D1D7F88C3C002BF1D105
:10AC6000F86880F0004010F0A3FCD6ED017A67EEA2
:10AC7000887A804617EE900A894610F099FC0B46B8
:10AC800041F6B8610246C4F21D014FF0A04010F039
:10AC90002FFB41EC100B0EF0D7FF404653EC102B6E
:10ACA000494610F0D9FC41EC100B0EF0CDFF51ECF1
:10ACB000100B10F0C9FFC5F8D4023A7CC2E700BF00
:10ACC0002497FF3BCDCC4C3DACC5A73770B545684C
:10ACD000D0ED035A95ED024A95ED036A9FED697A2E
:10ACE0009FED695AF2EE084AF9EE087AE4EE247A0A
:10ACF00000F6A44300F6A846F1EE006A2DED028BA3
:10AD000066EE266ABFEE008AF0EE484AE6EE264A74
:10AD10000446FDEEE77AF6EE008A17EE902AC0F8B8
:10AD2000882CC3ED004AD5ED037AF4EEE87AF1EE13
:10AD300010FAD4BFF0EE457AF0EE477AC6ED007A0D
:10AD400065EEE77A17EE900A10F032FC41EC100B3A
:10AD50000EF07AFF51EC100B10F076FF07EE100AA0
:10AD6000F7EE007A77EEC77AB0EE007AC6ED007A99
:10AD7000D5ED047AA7EE878A04F69C4204F54A636F
:10AD800082ED008A83ED008A95ED047AB4EEE87ACC
:10AD9000F1EE10FA03D5F1EE487AC3ED007ADFED5B
:10ADA0003B6A95ED056A9FED3A7AD4ED037A9FED03
:10ADB000398AA6EE267A04F6984627EE888A17EE98
:10ADC000100A10F0F5FB41EC100B0EF03DFF51ECBA
:10ADD000100B10F039FF07EE900A27EE888AF7EE85
:10ADE000007A86ED008A95ED067A77EE277A04F6EA
:10ADF000D44377EE877AF5EE006AC3ED007A95EDDD
:10AE0000067AB4EEE67AF1EE10FA09D5B0EE086AE9
:10AE1000F6EE086AE7EE466A77EEE67AC3ED007A68
:10AE200095ED077A9FED1C6ADFED1C7ADFED1C6A59
:10AE300027EE067A04F6844383ED007A95ED097ACD
:10AE4000B6EE006A37EE467A04F6B84383ED007A30
:10AE500095ED0A7A67EE277A04F54C6367EE877AF8
:10AE600004F6BC410022C1ED007ABDEC028B1A60F1
:10AE7000D5ED0B7A67EEA67A04F6C444C4ED007AE9
:10AE800070BD00BF00C05A4600409C453D0AC74007
:10AE90003D0A27C0560EC9408FC2F53C2DB29D3DDC
:10AEA0006666E63FF0B547F2A4040025C3F67D745C
:10AEB000034600F51C61C3F8D052C3F8D4423433C2
:10AEC0008B424FF00002F6D100F6D8454CF6CD4744
:10AED000C3F64C6700F6C84400262F600023C4F276
:10AEE000203600F69845266000F5496EC0F87C3C97
:10AEF000C0F88C3C00F54B6700F6AC4600F6944475
:10AF00004CF6CD4100F54E632A60C3F64C714FF00C
:10AF10007E55CEF800203A60326025601960BDE8A9
:10AF2000F040FFF7D3BE00BFF8B54FF4884243F2BC
:10AF3000C67341F64001C0F20201C4F22C72C3F2A2
:10AF4000BE73044601608260C36030200BF06EF86F
:10AF500003464FF07C571F6060602046FFF7B6FE47
:10AF6000636820465F60FFF7B1FE636820469F601C
:10AF7000FFF7ACFE63682046DF60FFF7A7FE63685B
:10AF800020461F61FFF7A2FE636846F26662C3F6C1
:10AF900026725A612046FFF799FE63684FF07A5295
:10AFA0009A612046FFF792FE63682046DF61FFF753
:10AFB0008DFE63680126267420465F62FFF786FED9
:10AFC000636848F20612C3F615629A622046FFF7DC
:10AFD0007DFE63680025DD622046FFF777FE41F6BF
:10AFE0004C03C0F20203C4F8803C2423636127238E
:10AFF000A3612B2323652D2363653023C4F88C3094
:10B000003323C4F890303723C4F8C8303923C4F848
:10B01000CC303C23C4F804313F23C4F80831432327
:10B02000C4F840314523C4F844314823C4F87C3186
:10B030004B23C4F880314F23C4F8B8315123C4F8EE
:10B04000BC315423C4F8F4315723C4F8F8315B23DE
:10B05000C4F830325D23C4F834326023C4F86C3253
:10B0600040F2E733C4F870320023E36142F21C136C
:10B07000236241F23013636242F21D13236343F6ED
:10B080007873636341F22733A36343F67973636490
:10B0900048F20573A36441F6FE03E36448F20673C5
:10B0A000A3654AF2A813E36540F6627323664AF289
:10B0B000A913E3664BF2C023236740F26163636721
:10B0C0004BF2C123C4F880304FF6BB63C4F8843020
:10B0D00041F27D43C4F888304FF6BC63C4F8943025
:10B0E0004CF2496366F31F43294648F6230040F6B5
:10B0F0009B0566F31F40C4F8B050C4F8D43041F645
:10B10000C14242F6D40343F2223E4FF2AD2566F32C
:10B110001F4266F31F4E66F31F45C4F8C000C4F813
:10B12000D8304FF4C75043F2233745F21F5366F32C
:10B130001F47C4F89820C4F8ACE0C4F8C400C0F2BB
:10B140000203C4F8E85048F624024CF24A6E43F277
:10B15000F1204AF2334566F31F4266F31F4EC4F8EE
:10B16000BC70C0F20200C0F20205C4F8103141F612
:10B17000C24C41F2BC034FF2AE2766F31F4766F3A1
:10B180001F4CC4F8D020C4F8E4E0C4F8FC00C4F8B4
:10B19000143140F61B40C4F8245143F2F22240F629
:10B1A0004C7545F220564AF2344E41F63673C0F2E1
:10B1B0000202C0F20206C4F8F870C0F2020E41F2B8
:10B1C0006147C4F80001C0F20303C4F828514FF2EC
:10B1D000DE0040F67935C4F8EC70C0F20200C4F825
:10B1E0000C21C4F82061C4F89C50C4F8A8C045F2F2
:10B1F0007376C4F834E1C4F84C3141F27C23C0F2D8
:10B200000306C4F83801C4F8503149F249104CF62D
:10B21000CB03C0F20300C0F20303C4F8606141F243
:10B220007D26C4F86461C4F87401C4F8883140F61E
:10B23000ED0041F202034FF2DF0241F6377740F6AC
:10B240004746C0F20202C0F20307C4F83C51C0F204
:10B250000406C4F87801C4F88C3145F2747544F6DC
:10B260008F6047F69033C0F20305C4F84821C4F854
:10B270005C71C0F20400C0F20403C4F89C6149F29E
:10B280004A1241F203064CF6CC07C0F20302C0F2A8
:10B290000307C4F87051C4F8A061C4F8B001C4F841
:10B2A000C43140F6196040F68E1340F648454CF222
:10B2B000F646C0F20405C4F88421C4F89871C0F2BF
:10B2C0000406C4F8B401C4F8C83144F6906247F6E5
:10B2D000913740F6D81045F2D923C0F20402C0F2EB
:10B2E0000407C4F8AC51C0F20500C0F20503C4F86D
:10B2F000D8614CF2F74541F68606C0F20405C4F861
:10B30000C021C4F8D471C4F8DC61C4F8EC01C4F8FD
:10B31000003240F6EB0040F6812340F6D91245F2A8
:10B32000DA2749F26B46C0F20502C0F20507C0F207
:10B330000506C4F8E851C4F8F001C4F8043249F233
:10B340006C454DF6AD2043F21D23C0F20505C0F259
:10B350000500C4F8FC21C0F20603C4F810729D2257
:10B36000C4F8146241F21216C0F2060245F2173711
:10B37000C4F81862C4F8245247F208264DF6AE25E8
:10B38000C4F82802C4F8643241F2694041F2AA13B9
:10B39000C0F20505C0F20607C0F20606C4F82C028A
:10B3A000C4F860229C2043F21E22C4F8683245F2A1
:10B3B0001633C0F20600C0F20603C0F20602C4F85B
:10B3C0009C7240F6790E40F6FB27C4F8A062C4F8E0
:10B3D000385240F60216C4F84C5247F2A405C4F89D
:10B3E0003C02C4F85002C4F87832C4F88C32C4F875
:10B3F000A4E2C3F67D75C4F84072C4F85472C4F870
:10B400007422C4F88822C4F87C62C4F8906223468F
:10B4100004F51C60C3F8D012C3F8D452343383420D
:10B420004FF00002F6D104F6D8464CF6CD4704F6AC
:10B43000C840C3F64C6700253760002304F69846E1
:10B44000C4F22035056004F5496EC4F87C3CC4F8AC
:10B450008C3C04F6AC4004F54E6304F54B6704F6EF
:10B4600094454CF6CD413260C3F64C714FF07E5698
:10B47000CEF800203A60026020462E601960FFF787
:10B4800025FC2046F8BD00BF70B545689FED6C7A7D
:10B4900095ED025A95ED036AF2EE085AF9EE087A34
:10B4A000E5EE257A00F6A44300F6A846F1EE006A20
:10B4B0002DED028B66EE266ABFEE008AF0EE485A4A
:10B4C000E6EE265A0446FDEEE77A85ED000A17EE11
:10B4D000902AC0F8882CC3ED005A95ED036ADFED81
:10B4E000597AD0ED036AF6EE008AB4EEE86AF1EE1E
:10B4F00010FAC8BFF0EE477AC6ED007A66EEE77A3A
:10B5000017EE900A10F054F841EC100B0EF09CFB73
:10B5100051EC100B10F098FB07EE100AF7EE007AD2
:10B5200077EEC77AB0EE007AC6ED007AD5ED047AF0
:10B53000A7EE878A04F69C4204F54A6382ED008AEE
:10B5400083ED008A95ED047AB4EEE87AF1EE10FA14
:10B5500003D5F1EE487AC3ED007ADFED3B6A95ED55
:10B56000056A9FED3A7AD4ED037A9FED398AA6EE0B
:10B57000267A04F6984627EE888A17EE100A10F00D
:10B5800017F841EC100B0EF05FFB51EC100B10F0B4
:10B590005BFB07EE900A27EE888AF7EE007A86EDCD
:10B5A000008A95ED067A77EE277A04F6D44377EE93
:10B5B000877AF5EE006AC3ED007A95ED067AB4EE6F
:10B5C000E67AF1EE10FA09D5B0EE086AF6EE086AEE
:10B5D000E7EE466A77EEE67AC3ED007A95ED077AF4
:10B5E0009FED1C6ADFED1C7ADFED1C6A27EE067A00
:10B5F00004F6844383ED007A95ED097AB6EE006A8D
:10B6000037EE467A04F6B84383ED007A95ED0A7A70
:10B6100067EE277A04F54C6367EE877A04F6BC413F
:10B620000022C1ED007ABDEC028B1A60D5ED0B7AD9
:10B6300067EEA67A04F6C444C4ED007A70BD00BF7C
:10B6400000C05A4600409C453D0AC7403D0A27C0FD
:10B65000560EC9408FC2F53C2DB29D3D6666E63F51
:10B6600070B545689FED6C7A95ED025A95ED036AC9
:10B67000F2EE085AF9EE087AE5EE257A00F6A443D0
:10B6800000F6A846F1EE006A2DED028B66EE266A02
:10B69000BFEE008AF0EE485AE6EE265A0446FDEE6A
:10B6A000E77A85ED010A17EE902AC0F8882CC3EDE1
:10B6B000005A95ED036ADFED597AD0ED036AF6EE94
:10B6C000008AB4EEE86AF1EE10FAC8BFF0EE477AED
:10B6D000C6ED007A66EEE77A17EE900A0FF068FF83
:10B6E00041EC100B0EF0B0FA51EC100B10F0ACFA6C
:10B6F00007EE100AF7EE007A77EEC77AB0EE007A1E
:10B70000C6ED007AD5ED047AA7EE878A04F69C424E
:10B7100004F54A6382ED008A83ED008A95ED047A90
:10B72000B4EEE87AF1EE10FA03D5F1EE487AC3ED03
:10B73000007ADFED3B6A95ED056A9FED3A7AD4ED2C
:10B74000037A9FED398AA6EE267A04F6984627EE0C
:10B75000888A17EE100A0FF02BFF41EC100B0EF049
:10B7600073FA51EC100B10F06FFA07EE900A27EE07
:10B77000888AF7EE007A86ED008A95ED067A77EEF4
:10B78000277A04F6D44377EE877AF5EE006AC3EDA4
:10B79000007A95ED067AB4EEE67AF1EE10FA09D564
:10B7A000B0EE086AF6EE086AE7EE466A77EEE67AE9
:10B7B000C3ED007A95ED077A9FED1C6ADFED1C7AE8
:10B7C000DFED1C6A27EE067A04F6844383ED007AE7
:10B7D00095ED097AB6EE006A37EE467A04F6B8437C
:10B7E00083ED007A95ED0A7A67EE277A04F54C63CB
:10B7F00067EE877A04F6BC410022C1ED007ABDEC09
:10B80000028B1A60D5ED0B7A67EEA67A04F6C44473
:10B81000C4ED007A70BD00BF00C05A4600409C4590
:10B820003D0AC7403D0A27C0560EC9408FC2F53CAD
:10B830002DB29D3D6666E63F70B545689FED6B7A1B
:10B8400095ED036AF2EE085AF9EE087AE0EE257AF1
:10B8500000F6A44300F6A846F1EE006A2DED028B37
:10B8600066EE266ABFEE008AF0EE485AE6EE265AE9
:10B870000446FDEEE77A85ED020A17EE902AC0F83D
:10B88000882CC3ED005A95ED036ADFED597AD0EDAF
:10B89000036AF6EE008AB4EEE86AF1EE10FAC8BF69
:10B8A000F0EE477AC6ED007A66EEE77A17EE900A78
:10B8B0000FF07EFE41EC100B0EF0C6F951EC100BB0
:10B8C00010F0C2F907EE100AF7EE007A77EEC77AA9
:10B8D000B0EE007AC6ED007AD5ED047AA7EE878A3D
:10B8E00004F69C4204F54A6382ED008A83ED008AE7
:10B8F00095ED047AB4EEE87AF1EE10FA03D5F1EEA4
:10B90000487AC3ED007ADFED3B6A95ED056A9FED5D
:10B910003A7AD4ED037A9FED398AA6EE267A04F6B8
:10B92000984627EE888A17EE100A0FF041FE41EC88
:10B93000100B0EF089F951EC100B10F085F907EEA1
:10B94000900A27EE888AF7EE007A86ED008A95ED58
:10B95000067A77EE277A04F6D44377EE877AF5EE07
:10B96000006AC3ED007A95ED067AB4EEE67AF1EE60
:10B9700010FA09D5B0EE086AF6EE086AE7EE466AF4
:10B9800077EEE67AC3ED007A95ED077A9FED1C6AB3
:10B99000DFED1C7ADFED1C6A27EE067A04F684439D
:10B9A00083ED007A95ED097AB6EE006A37EE467AB5
:10B9B00004F6B84383ED007A95ED0A7A67EE277AAC
:10B9C00004F54C6367EE877A04F6BC410022C1EDB2
:10B9D000007ABDEC028B1A60D5ED0B7A67EEA67A81
:10B9E00004F6C444C4ED007A70BD00BF00C05A46DE
:10B9F00000409C453D0AC7403D0A27C0560EC9403D
:10BA00008FC2F53C2DB29D3D6666E63F70B5456838
:10BA10009FED6B7AD5ED025AB2EE086AF9EE087A1C
:10BA2000E5EE867A00F6A44300F6A846F1EE006A39
:10BA30002DED028B60EE266ABFEE008AB0EE486AFA
:10BA4000A0EE266A0446FDEEE77A85ED030A17EEBE
:10BA5000902AC0F8882C83ED006A95ED036ADFED2B
:10BA6000597AD0ED036AF6EE008AB4EEE86AF1EE98
:10BA700010FAC8BFF0EE477AC6ED007A66EEE77AB4
:10BA800017EE900A0FF094FD41EC100B0EF0DCF86D
:10BA900051EC100B10F0D8F807EE100AF7EE007A10
:10BAA00077EEC77AB0EE007AC6ED007AD5ED047A6B
:10BAB000A7EE878A04F69C4204F54A6382ED008A69
:10BAC00083ED008A95ED047AB4EEE87AF1EE10FA8F
:10BAD00003D5F1EE487AC3ED007ADFED3B6A95EDD0
:10BAE000056A9FED3A7AD4ED037A9FED398AA6EE86
:10BAF000267A04F6984627EE888A17EE100A0FF089
:10BB000057FD41EC100B0EF09FF851EC100B10F0AC
:10BB10009BF807EE900A27EE888AF7EE007A86ED0A
:10BB2000008A95ED067A77EE277A04F6D44377EE0D
:10BB3000877AF5EE006AC3ED007A95ED067AB4EEE9
:10BB4000E67AF1EE10FA09D5B0EE086AF6EE086A68
:10BB5000E7EE466A77EEE67AC3ED007A95ED077A6E
:10BB60009FED1C6ADFED1C7ADFED1C6A27EE067A7A
:10BB700004F6844383ED007A95ED097AB6EE006A07
:10BB800037EE467A04F6B84383ED007A95ED0A7AEB
:10BB900067EE277A04F54C6367EE877A04F6BC41BA
:10BBA0000022C1ED007ABDEC028B1A60D5ED0B7A54
:10BBB00067EEA67A04F6C444C4ED007A70BD00BFF7
:10BBC00000C05A4600409C453D0AC7403D0A27C078
:10BBD000560EC9408FC2F53C2DB29D3D6666E63FCC
:10BBE00070B545689FED6C7A95ED025A95ED036A44
:10BBF000F2EE085AF9EE087AE5EE257A00F6A4434B
:10BC000000F6A846F1EE006A2DED028B66EE266A7C
:10BC1000BFEE008AF0EE485AE6EE265A0446FDEEE4
:10BC2000E77A85ED040A17EE902AC0F8882CC3ED58
:10BC3000005A95ED036ADFED597AD0ED036AF6EE0E
:10BC4000008AB4EEE86AF1EE10FAC8BFF0EE477A67
:10BC5000C6ED007A66EEE77A17EE900A0FF0A8FCC0
:10BC600041EC100B0DF0F0FF51EC100B0FF0ECFF5E
:10BC700007EE100AF7EE007A77EEC77AB0EE007A98
:10BC8000C6ED007AD5ED047AA7EE878A04F69C42C9
:10BC900004F54A6382ED008A83ED008A95ED047A0B
:10BCA000B4EEE87AF1EE10FA03D5F1EE487AC3ED7E
:10BCB000007ADFED3B6A95ED056A9FED3A7AD4EDA7
:10BCC000037A9FED398AA6EE267A04F6984627EE87
:10BCD000888A17EE100A0FF06BFC41EC100B0DF088
:10BCE000B3FF51EC100B0FF0AFFF07EE900A27EEF9
:10BCF000888AF7EE007A86ED008A95ED067A77EE6F
:10BD0000277A04F6D44377EE877AF5EE006AC3ED1E
:10BD1000007A95ED067AB4EEE67AF1EE10FA09D5DE
:10BD2000B0EE086AF6EE086AE7EE466A77EEE67A63
:10BD3000C3ED007A95ED077A9FED1C6ADFED1C7A62
:10BD4000DFED1C6A27EE067A04F6844383ED007A61
:10BD500095ED097AB6EE006A37EE467A04F6B843F6
:10BD600083ED007A95ED0A7A67EE277A04F54C6345
:10BD700067EE877A04F6BC410022C1ED007ABDEC83
:10BD8000028B1A60D5ED0B7A67EEA67A04F6C444EE
:10BD9000C4ED007A70BD00BF00C05A4600409C450B
:10BDA0003D0AC7403D0A27C0560EC9408FC2F53C28
:10BDB0002DB29D3D6666E63F70B545689FED6C7A95
:10BDC00095ED025A95ED036AF2EE085AF9EE087AFB
:10BDD000E5EE257A00F6A44300F6A846F1EE006AE7
:10BDE0002DED028B66EE266ABFEE008AF0EE485A11
:10BDF000E6EE265A0446FDEEE77A85ED050A17EED3
:10BE0000902AC0F8882CC3ED005A95ED036ADFED47
:10BE1000597AD0ED036AF6EE008AB4EEE86AF1EEE4
:10BE200010FAC8BFF0EE477AC6ED007A66EEE77A00
:10BE300017EE900A0FF0BCFB41EC100B0DF004FF65
:10BE400051EC100B0FF000FF07EE100AF7EE007A2E
:10BE500077EEC77AB0EE007AC6ED007AD5ED047AB7
:10BE6000A7EE878A04F69C4204F54A6382ED008AB5
:10BE700083ED008A95ED047AB4EEE87AF1EE10FADB
:10BE800003D5F1EE487AC3ED007ADFED3B6A95ED1C
:10BE9000056A9FED3A7AD4ED037A9FED398AA6EED2
:10BEA000267A04F6984627EE888A17EE100A0FF0D5
:10BEB0007FFB41EC100B0DF0C7FE51EC100B0FF0A7
:10BEC000C3FE07EE900A27EE888AF7EE007A86ED29
:10BED000008A95ED067A77EE277A04F6D44377EE5A
:10BEE000877AF5EE006AC3ED007A95ED067AB4EE36
:10BEF000E67AF1EE10FA09D5B0EE086AF6EE086AB5
:10BF0000E7EE466A77EEE67AC3ED007A95ED077ABA
:10BF10009FED1C6ADFED1C7ADFED1C6A27EE067AC6
:10BF200004F6844383ED007A95ED097AB6EE006A53
:10BF300037EE467A04F6B84383ED007A95ED0A7A37
:10BF400067EE277A04F54C6367EE877A04F6BC4106
:10BF50000022C1ED007ABDEC028B1A60D5ED0B7AA0
:10BF600067EEA67A04F6C444C4ED007A70BD00BF43
:10BF700000C05A4600409C453D0AC7403D0A27C0C4
:10BF8000560EC9408FC2F53C2DB29D3D6666E63F18
:10BF900070B545689FED6C7A95ED025A95ED036A90
:10BFA000F2EE085AF9EE087AE5EE257A00F6A44397
:10BFB00000F6A846F1EE006A2DED028B66EE266AC9
:10BFC000BFEE008AF0EE485AE6EE265A0446FDEE31
:10BFD000E77A85ED060A17EE902AC0F8882CC3EDA3
:10BFE000005A95ED036ADFED597AD0ED036AF6EE5B
:10BFF000008AB4EEE86AF1EE10FAC8BFF0EE477AB4
:10C00000C6ED007A66EEE77A17EE900A0FF0D0FAE6
:10C0100041EC100B0DF018FE51EC100B0FF014FE5C
:10C0200007EE100AF7EE007A77EEC77AB0EE007AE4
:10C03000C6ED007AD5ED047AA7EE878A04F69C4215
:10C0400004F54A6382ED008A83ED008A95ED047A57
:10C05000B4EEE87AF1EE10FA03D5F1EE487AC3EDCA
:10C06000007ADFED3B6A95ED056A9FED3A7AD4EDF3
:10C07000037A9FED398AA6EE267A04F6984627EED3
:10C08000888A17EE100A0FF093FA41EC100B0DF0AE
:10C09000DBFD51EC100B0FF0D7FD07EE900A27EEF9
:10C0A000888AF7EE007A86ED008A95ED067A77EEBB
:10C0B000277A04F6D44377EE877AF5EE006AC3ED6B
:10C0C000007A95ED067AB4EEE67AF1EE10FA09D52B
:10C0D000B0EE086AF6EE086AE7EE466A77EEE67AB0
:10C0E000C3ED007A95ED077A9FED1C6ADFED1C7AAF
:10C0F000DFED1C6A27EE067A04F6844383ED007AAE
:10C1000095ED097AB6EE006A37EE467A04F6B84342
:10C1100083ED007A95ED0A7A67EE277A04F54C6391
:10C1200067EE877A04F6BC410022C1ED007ABDECCF
:10C13000028B1A60D5ED0B7A67EEA67A04F6C4443A
:10C14000C4ED007A70BD00BF00C05A4600409C4557
:10C150003D0AC7403D0A27C0560EC9408FC2F53C74
:10C160002DB29D3D6666E63F70B545689FED6C7AE1
:10C1700095ED025A95ED036AF2EE085AF9EE087A47
:10C18000E5EE257A00F6A44300F6A846F1EE006A33
:10C190002DED028B66EE266ABFEE008AF0EE485A5D
:10C1A000E6EE265A0446FDEEE77A85ED070A17EE1D
:10C1B000902AC0F8882CC3ED005A95ED036ADFED94
:10C1C000597AD0ED036AF6EE008AB4EEE86AF1EE31
:10C1D00010FAC8BFF0EE477AC6ED007A66EEE77A4D
:10C1E00017EE900A0FF0E4F941EC100B0DF02CFD66
:10C1F00051EC100B0FF028FD07EE100AF7EE007A55
:10C2000077EEC77AB0EE007AC6ED007AD5ED047A03
:10C21000A7EE878A04F69C4204F54A6382ED008A01
:10C2200083ED008A95ED047AB4EEE87AF1EE10FA27
:10C2300003D5F1EE487AC3ED007ADFED3B6A95ED68
:10C24000056A9FED3A7AD4ED037A9FED398AA6EE1E
:10C25000267A04F6984627EE888A17EE100A0FF021
:10C26000A7F941EC100B0DF0EFFC51EC100B0FF0A7
:10C27000EBFC07EE900A27EE888AF7EE007A86ED4F
:10C28000008A95ED067A77EE277A04F6D44377EEA6
:10C29000877AF5EE006AC3ED007A95ED067AB4EE82
:10C2A000E67AF1EE10FA09D5B0EE086AF6EE086A01
:10C2B000E7EE466A77EEE67AC3ED007A95ED077A07
:10C2C0009FED1C6ADFED1C7ADFED1C6A27EE067A13
:10C2D00004F6844383ED007A95ED097AB6EE006AA0
:10C2E00037EE467A04F6B84383ED007A95ED0A7A84
:10C2F00067EE277A04F54C6367EE877A04F6BC4153
:10C300000022C1ED007ABDEC028B1A60D5ED0B7AEC
:10C3100067EEA67A04F6C444C4ED007A70BD00BF8F
:10C3200000C05A4600409C453D0AC7403D0A27C010
:10C33000560EC9408FC2F53C2DB29D3D6666E63F64
:10C340000174704770B545689FED6C7A95ED025A9F
:10C3500095ED036AF2EE085AF9EE087AE5EE257AD1
:10C3600000F6A44300F6A846F1EE006A2DED028B1C
:10C3700066EE266ABFEE008AF0EE485AE6EE265ACE
:10C380000446FDEEE77A85ED090A17EE902AC0F81B
:10C39000882CC3ED005A95ED036ADFED597AD0ED94
:10C3A000036AF6EE008AB4EEE86AF1EE10FAC8BF4E
:10C3B000F0EE477AC6ED007A66EEE77A17EE900A5D
:10C3C0000FF0F6F841EC100B0DF03EFC51EC100BA9
:10C3D0000FF03AFC07EE100AF7EE007A77EEC77A14
:10C3E000B0EE007AC6ED007AD5ED047AA7EE878A22
:10C3F00004F69C4204F54A6382ED008A83ED008ACC
:10C4000095ED047AB4EEE87AF1EE10FA03D5F1EE88
:10C41000487AC3ED007ADFED3B6A95ED056A9FED42
:10C420003A7AD4ED037A9FED398AA6EE267A04F69D
:10C43000984627EE888A17EE100A0FF0B9F841ECFB
:10C44000100B0DF001FC51EC100B0FF0FDFB07EE93
:10C45000900A27EE888AF7EE007A86ED008A95ED3D
:10C46000067A77EE277A04F6D44377EE877AF5EEEC
:10C47000006AC3ED007A95ED067AB4EEE67AF1EE45
:10C4800010FA09D5B0EE086AF6EE086AE7EE466AD9
:10C4900077EEE67AC3ED007A95ED077A9FED1C6A98
:10C4A000DFED1C7ADFED1C6A27EE067A04F6844382
:10C4B00083ED007A95ED097AB6EE006A37EE467A9A
:10C4C00004F6B84383ED007A95ED0A7A67EE277A91
:10C4D00004F54C6367EE877A04F6BC410022C1ED97
:10C4E000007ABDEC028B1A60D5ED0B7A67EEA67A66
:10C4F00004F6C444C4ED007A70BD00BF00C05A46C3
:10C5000000409C453D0AC7403D0A27C0560EC94021
:10C510008FC2F53C2DB29D3D6666E63F70B545681D
:10C520009FED6C7A95ED025A95ED036AF2EE085A8A
:10C53000F9EE087AE5EE257A00F6A44300F6A8465F
:10C54000F1EE006A2DED028B66EE266ABFEE008AE0
:10C55000F0EE485AE6EE265A0446FDEEE77A85EDFF
:10C560000A0A17EE902AC0F8882CC3ED005A95ED00
:10C57000036ADFED597AD0ED036AF6EE008AB4EE75
:10C58000E86AF1EE10FAC8BFF0EE477AC6ED007A1D
:10C5900066EEE77A17EE900A0FF00AF841EC100BFE
:10C5A0000DF052FB51EC100B0FF04EFB07EE100A92
:10C5B000F7EE007A77EEC77AB0EE007AC6ED007A31
:10C5C000D5ED047AA7EE878A04F69C4204F54A6307
:10C5D00082ED008A83ED008A95ED047AB4EEE87A64
:10C5E000F1EE10FA03D5F1EE487AC3ED007ADFEDF3
:10C5F0003B6A95ED056A9FED3A7AD4ED037A9FED9B
:10C60000398AA6EE267A04F6984627EE888A17EE2F
:10C61000100A0EF0CDFF41EC100B0DF015FB51ECA4
:10C62000100B0FF011FB07EE900A27EE888AF7EE49
:10C63000007A86ED008A95ED067A77EE277A04F681
:10C64000D44377EE877AF5EE006AC3ED007A95ED74
:10C65000067AB4EEE67AF1EE10FA09D5B0EE086A81
:10C66000F6EE086AE7EE466A77EEE67AC3ED007A00
:10C6700095ED077A9FED1C6ADFED1C7ADFED1C6AF1
:10C6800027EE067A04F6844383ED007A95ED097A65
:10C69000B6EE006A37EE467A04F6B84383ED007AC8
:10C6A00095ED0A7A67EE277A04F54C6367EE877A90
:10C6B00004F6BC410022C1ED007ABDEC028B1A6089
:10C6C000D5ED0B7A67EEA67A04F6C444C4ED007A81
:10C6D00070BD00BF00C05A4600409C453D0AC7409F
:10C6E0003D0A27C0560EC9408FC2F53C2DB29D3D74
:10C6F0006666E63F70B545689FED6C7A95ED025A27
:10C7000095ED036AF2EE085AF9EE087AE5EE257A1D
:10C7100000F6A44300F6A846F1EE006A2DED028B68
:10C7200066EE266ABFEE008AF0EE485AE6EE265A1A
:10C730000446FDEEE77A85ED0B0A17EE902AC0F865
:10C74000882CC3ED005A95ED036ADFED597AD0EDE0
:10C75000036AF6EE008AB4EEE86AF1EE10FAC8BF9A
:10C76000F0EE477AC6ED007A66EEE77A17EE900AA9
:10C770000EF01EFF41EC100B0DF066FA51EC100BA1
:10C780000FF062FA07EE100AF7EE007A77EEC77A3A
:10C79000B0EE007AC6ED007AD5ED047AA7EE878A6E
:10C7A00004F69C4204F54A6382ED008A83ED008A18
:10C7B00095ED047AB4EEE87AF1EE10FA03D5F1EED5
:10C7C000487AC3ED007ADFED3B6A95ED056A9FED8F
:10C7D0003A7AD4ED037A9FED398AA6EE267A04F6EA
:10C7E000984627EE888A17EE100A0EF0E1FE41EC1B
:10C7F000100B0DF029FA51EC100B0FF025FA07EE93
:10C80000900A27EE888AF7EE007A86ED008A95ED89
:10C81000067A77EE277A04F6D44377EE877AF5EE38
:10C82000006AC3ED007A95ED067AB4EEE67AF1EE91
:10C8300010FA09D5B0EE086AF6EE086AE7EE466A25
:10C8400077EEE67AC3ED007A95ED077A9FED1C6AE4
:10C85000DFED1C7ADFED1C6A27EE067A04F68443CE
:10C8600083ED007A95ED097AB6EE006A37EE467AE6
:10C8700004F6B84383ED007A95ED0A7A67EE277ADD
:10C8800004F54C6367EE877A04F6BC410022C1EDE3
:10C89000007ABDEC028B1A60D5ED0B7A67EEA67AB2
:10C8A00004F6C444C4ED007A70BD00BF00C05A460F
:10C8B00000409C453D0AC7403D0A27C0560EC9406E
:10C8C0008FC2F53C2DB29D3D6666E63FD0F87C0CEC
:10C8D000704700BF2DE9F04F2DED028B151E83B080
:10C8E00006460F46D0F804A040F3D181D0F87C4C26
:10C8F000017C8C4280F29A81342303FB04030022E2
:10C90000611CC0F87C1CC3F8DC22C3F8D822A7F154
:10C910003C094EF64F4309FB09F2C4F6C46383FB9E
:10C920000231D317C3EBA10303EB430103EB8103F4
:10C93000D31A07EE903AF8EEE77AB1EE0A7A06F6E5
:10C94000BC4106F6B84377EEC77AD3ED006A91EDA5
:10C95000007A3C2FE7EE276A09DD07EE102A06F57C
:10C960004C63D3ED007AB8EEC77AE7EE876AD6F863
:10C97000883CB2691A44974240F30082726D1A44AF
:10C98000974240F32F82D6F890201A44974240F302
:10C990002682D6F8CC201A44974240F31D82D6F85E
:10C9A00008211A44974240F3FB81D6F844211A44E7
:10C9B000974240F3F281D6F880211A44974240F31F
:10C9C000E981D6F8BC211A44974240F3E081D6F8B9
:10C9D000F8211A44974240F3D781D6F834221A44FA
:10C9E000974240F3CE81D6F8702213449F42CCBFC9
:10C9F0004FF021084FF01E084FEA880B0BEB08039D
:10CA000006EB8303D6ED037A5B699FEDE78A9FED22
:10CA1000E76AFB1A07EE103AB8EEC77A27EE888A63
:10CA200077EE267A67EE867A17EE900A0EF0C0FD52
:10CA300041EC100B0DF008F9342303FB046351ECB7
:10CA4000100B00930FF000F907EE900A27EE888A8A
:10CA5000009BBEEEC88A0022302DC3F8C02283EDB1
:10CA6000AF8A07DD502DD4BF08F1010808F1020894
:10CA70004FEA880BD84406EB88084FF0340E06F6D0
:10CA8000D442D8F82030D2ED008AD8F81C00D8F86B
:10CA900024100EFB0468013BC8F8C832C8F8C40271
:10CAA000C8F8CC1218EE900A0EF082FD07EE905AEC
:10CAB0009FEDBF7AF8EEE77ACDE9000167EE877A5D
:10CAC000B0EE088A17EE900A0EF072FD9DED001B85
:10CAD00041EC100B0DF03CF9F0EE007A51EC100B2C
:10CAE000A8EEA78A0FF0B0F807EE900A28EE278A82
:10CAF0003C2F88EDB48A00F32281DAED046A9FEDC1
:10CB0000AD7ADFEDAD5ADFEDAD7A9FEDAD6A96ED12
:10CB1000038A06F6C84393ED005A66EEA66A403DC6
:10CB2000A6EE857A06F6CC4306F6D84105EE107AD5
:10CB3000F0EE476A07EE105AD3ED004AB8EEC77A16
:10CB4000B8EEC55AE4EE876A342303FB0463E5EECE
:10CB5000257AC3F8EC7206F68442F4EEE76AF1EE49
:10CB600010FA58BFF0EE667AF4EEC67AF1EE10FADB
:10CB7000D4BF67EEA77ADFED937A68EE277A0B2FA2
:10CB8000C3EDB87A6CDD6C2F40F33181D1ED007AC2
:10CB900092ED007A9FED8C6A27EE877AF0EE675A65
:10CBA000E7EE065A4EF685394FF0A858F0EE006AC7
:10CBB000B0EE657AC4F20109B0EE476A97EEA66A54
:10CBC00083EDBA7A83EDB96ADAED007A77EEA77A67
:10CBD00017EE900A0EF0ECFC02460B464046494622
:10CBE0000EF086FB41EC100B0DF02EF8F1EE487ABA
:10CBF00053EC102B17EE900ACDE900230EF0D8FC71
:10CC0000DDE900230EF028FD41EC100B0DF01CF8BF
:10CC1000342351EC100B03FB04660FF015F8C6F833
:10CC2000D40203B0BDEC028BBDE8F08F002900F008
:10CC3000DC800024DFED657A2346024692EDB47A6B
:10CC4000B4EEE77AF1EE10FA48BF1C4603F1010397
:10CC500048BFF0EE477A994202F13402EED156E62F
:10CC6000D1ED007A92ED007A9FED596A27EE877A2E
:10CC7000F0EE675AE7EE065A47F6E1294FF02058E2
:10CC8000F0EE006AB0EE657AC3F6D47994E7027CE0
:10CC9000002AC6D0044600254FF0800B04E0013581
:10CCA000AA4204F13404BCDDD4F8EC329F42F6D140
:10CCB000D6F88C3C1BB1C4F8ECB2327CEFE7F068DC
:10CCC00080F000400EF074FCCDE9000138460EF013
:10CCD0005DFC47F6E1234FF08042C3F684730EF00B
:10CCE000BBFC00230022C4F218030EF003FB9AEDF4
:10CCF000017AF1EE047A67EE277A804617EE900A01
:10CD000089460EF055FC02460B46404649460EF059
:10CD1000EFFA41EC100B0CF097FFDDE9000153EC4A
:10CD2000102B0EF099FC41EC100B0CF08DFF51EC28
:10CD3000100B0EF089FFC4F8D402327CAFE7C7F1C4
:10CD40003C0307EE903A9FED237AF8EEE77A67EE20
:10CD5000877A17EE900A0EF02BFC41EC100B0CF0CA
:10CD600073FF51EC100B0EF06FFFD8EDB47A07EEA5
:10CD7000100A67EE877AC8EDB47ABEE64FF0000875
:10CD80003AE64FF01B0837E64FF0180834E64FF04C
:10CD9000150831E64FF012082EE64FF00F082BE68B
:10CDA0004FF00C0828E600BF0000FA4620986C3DC2
:10CDB0002497FF3B00004842CDCCCC3E00005C42B3
:10CDC0000000524300442C47000040420000C6428D
:10CDD000000040C20AD7233C4FF009080CE64FF090
:10CDE000060809E64FF0030806E60C468FE591EDCC
:10CDF000007AD2ED006A07EE909A67EE266AF8EEA6
:10CE0000E77AF0EE475AE6EEA75A2B2FB0EE006A0B
:10CE1000F0EE656AD7EE066AC3EDBA5AC3EDB96A99
:10CE200006DC47F6E1294FF02058C3F6D479CBE66B
:10CE300038460EF0ABFB4BF651034FF06042C3F6A1
:10CE40009E730EF009FC00230022C3F6F0730EF06F
:10CE50004FFA80468946B7E670B50021064607F0CE
:10CE6000EDFEC0B1B6F91E40B6F92010031D00F565
:10CE7000827533F9022B9442A8BF14469142B8BF81
:10CE800011469D42F5D80123F48331843377BDE800
:10CE9000704007F08BBE70BD0020704700207047C7
:10CEA000F8B549F22044037AC1F6FF74242908BF7B
:10CEB000C2805B0001250E462046C1F307211746BC
:10CEC00084F83B3084F85E5084F85D5003F05CFFDA
:10CED000F1B2204603F058FFC7F30721204603F0C4
:10CEE00053FFF9B2204603F04FFF2946204604F0D5
:10CEF00023F8B0FA80F04009F8BD00BF2DE9F843EF
:10CF000049F22044037AC1F6FF740125AB4029465B
:10CF10000746204684F83B3084F85E5084F85D5024
:10CF200003F032FF0421204603F02EFF20460021AB
:10CF300004F002F8B8B34FF0010846464FF000097C
:10CF40003B7A012549F22040AB402946C1F6FF70EB
:10CF500084F83B3084F85E5084F85D5003F014FF91
:10CF600049F220400421C1F6FF7003F00DFF49F2A1
:10CF700020404946C1F6FF7003F006FF49F2204009
:10CF80004146C1F6FF7003F0FFFE49F220402946FA
:10CF9000C1F6FF7003F0D0FF10B10020BDE8F883A8
:10CFA000B0B2BDE8F8832B460222397A204604F05D
:10CFB0004FF80128BFD994F8381094F83950A94295
:10CFC00018D263184A1CD2B2187E84F838209542D1
:10CFD0004FEA00230ED922440231107E84F8381023
:10CFE000184320F0010040F001064FEA16295FFACD
:10CFF00086F8A5E74FF0FF08C1464FF0FF369FE7E0
:10D000002DE9F84349F22044037AC1F6FF74012563
:10D01000AB4029460746204684F83B3084F85E50F2
:10D0200084F85D5003F0B0FE2421204603F0ACFEEE
:10D030002046002103F080FFB8B34FF001084646B8
:10D040004FF000093B7A012549F22040AB402946C8
:10D05000C1F6FF7084F83B3084F85E5084F85D5070
:10D0600003F092FE49F220402421C1F6FF7003F044
:10D070008BFE49F220404946C1F6FF7003F084FE62
:10D0800049F220404146C1F6FF7003F07DFE49F2AF
:10D0900020402946C1F6FF7003F04EFF10B100207A
:10D0A000BDE8F883B0B2BDE8F8832B460222397A96
:10D0B000204603F0CDFF0128BFD994F8381094F82A
:10D0C0003950A94218D263184A1CD2B2187E84F88B
:10D0D000382095424FEA00230ED922440231107EB7
:10D0E00084F83810184320F0010040F001064FEAA0
:10D0F00016295FFA86F8A5E74FF0FF08C1464FF002
:10D10000FF369FE7F8B549F22044037AC1F6FF7471
:10D110000126B340074601F003052046314684F856
:10D120003B3084F85E6084F85D6003F02DFE0821DA
:10D13000204603F029FE2046002103F0FDFE98B3AF
:10D1400000233A7A012649F22040B2403146C1F626
:10D15000FF701D4384F83B2084F85E6084F85D60B6
:10D1600003F012FE49F220400821C1F6FF7003F0DF
:10D170000BFE49F22040C5F30721C1F6FF7003F012
:10D1800003FE49F22040E9B2C1F6FF7003F0FCFD56
:10D1900049F220403146C1F6FF7003F0CDFE08B1E0
:10D1A0000020F8BDA8B2F8BD33460222397A2046E5
:10D1B00003F04EFF0128C3D994F8381094F83900D1
:10D1C000814212D263184A1CD2B21B7E84F83820E6
:10D1D00090424FEA032308D922440231127E84F898
:10D1E0003810134323F00303ABE76FF00303A8E702
:10D1F000F8B549F22044027AC1F6FF7452000126C4
:10D2000000210546204684F83B2084F85E6084F8BF
:10D210005D6003F0B9FD0E21204603F0B5FD204608
:10D22000002103F089FE88B3002603272B7A49F2F8
:10D2300020405B0001250021C1F6FF7084F83B30DF
:10D2400084F85E5084F85D5003F09EFD49F2204062
:10D250000E21C1F6FF7003F097FD49F220403946D8
:10D26000C1F6FF7003F090FD49F220403146C1F64F
:10D27000FF7003F089FD49F220402946C1F6FF7096
:10D2800003F05AFEB0FA80F04009F8BD334602229E
:10D29000297A204603F0DCFE0128C5D994F838101D
:10D2A00094F83900814216D263184A1CD2B21E7E0D
:10D2B00084F8382090424FEA06230CD922440231E8
:10D2C000167E84F838101E4326F4407646F44076E5
:10D2D000370AF6B2AAE7FF263746A7E71F29F8B5AF
:10D2E000064652D80C294DD840F60D55327A49F2EF
:10D2F0002044C1F6FF74520001270021204684F823
:10D300003B2084F85E7084F85D7003F03DFD2E21B3
:10D31000204603F039FD2046002103F00DFEC8B37E
:10D320000023327A49F22040520001260021C1F642
:10D33000FF701D4384F83B2084F85E6084F85D60D4
:10D3400003F022FD49F220402E21C1F6FF7003F0C8
:10D350001BFD49F22040C5F30721C1F6FF7003F021
:10D3600013FD49F22040E9B2C1F6FF7003F00CFD55
:10D3700049F220403146C1F6FF7003F0DDFD38B1BF
:10D380000020F8BD41EA0125B0E741F61F75ADE781
:10D39000A8B2F8BD3B460222317A204603F058FE7F
:10D3A0000128BDD994F8381094F83900814214D27C
:10D3B00063184A1CD2B21B7E84F8382090424FEA90
:10D3C00003230AD922440231127E84F83810134311
:10D3D00023F4F85323F01F03A3E74EF2E003CFF644
:10D3E000FF739EE70023C4F2FE2307EE103A47F6D0
:10D3F000EE43C3F6FF6307EE903A70B5E0EE877A2E
:10D400000023C4F2FE2307EE103AFCEEE77A47F65B
:10D41000EE4382B0C3F6FF63CDED017A07EE903A9A
:10D42000E0EE077A9DF80450027AFCEEE77A7F2D51
:10D43000CDED017A9DF804309CBFC5F17F052D022A
:10D4400049F22044C1F6FF7494BF2DB200257F2B12
:10D4500094BFC3F17F030023520001262046002120
:10D460001D4384F83B2084F85E6084F85D6003F01F
:10D470008BFC2046222103F087FCC5F307212046C0
:10D4800003F082FCE9B2204603F07EFC31462046E0
:10D4900003F052FDB0FA80F0400902B070BD00BF49
:10D4A0000023C4F27C2307EE103A47F6EE43C3F69E
:10D4B000FF6307EE903AF0B5E0EE077A0023C4F27E
:10D4C000FE2307EE103AFCEEE77A47F6EE4383B010
:10D4D000C3F6FF63CDED017A07EE903AE0EE877A6E
:10D4E0009DF804500646FCEEE77A3F2DCDED017A1B
:10D4F0009DF80400337A98BFC5F13F0549F22044F6
:10D50000C1F6FF744FF0010794BF2D0200257F285C
:10D5100094BFC0F17F020022BB403946204615432C
:10D5200084F83B3084F85E7084F85D7003F02CFC66
:10D530000621204603F028FC2046002103F0FCFCD5
:10D54000A8B30023327A49F220400126B240314686
:10D55000C1F6FF701D4384F83B2084F85E6084F8B8
:10D560005D6003F011FC49F220400621C1F6FF7016
:10D5700003F00AFC49F22040C5F30721C1F6FF7011
:10D5800003F002FC49F22040E9B2C1F6FF7003F05B
:10D59000FBFB49F220403146C1F6FF7003F0CCFCA2
:10D5A00010B1002003B0F0BDA8B203B0F0BD3B46FF
:10D5B0000222317A204603F04BFD0128C1D994F8AC
:10D5C000381094F83900814214D263184A1CD2B240
:10D5D0001B7E84F8382090424FEA03230AD9224464
:10D5E0000231127E84F83810134323F47D5323F064
:10D5F0003F03A7E74CF28003CFF6FF73A2E700BF1B
:10D600002DE9F84F49F2204490F808E0C1F6FF7484
:10D610000E46C1F307294FEA4E0E4FF0010A494664
:10D6200007465FFA86F8204693461D4684F83BE09D
:10D6300084F85EA084F85DA003F0A6FB4146204676
:10D6400003F0A2FB2046002103F076FCC0B30025C6
:10D650003B7A242E4BEA050549F2204008BFFD80A5
:10D660005B0001264946C1F6FF7084F83B3084F820
:10D670005E6084F85D6003F087FB49F2204041461C
:10D68000C1F6FF7003F080FB49F22040C5F307218B
:10D69000C1F6FF7003F078FB49F22040E9B2C1F611
:10D6A000FF7003F071FB49F220403146C1F6FF7074
:10D6B00003F042FC00280CBF28460020BDE8F88F8C
:10D6C00053460222397A204603F0C2FC0128BED913
:10D6D00094F8381094F83900814204D34FF0FF33A6
:10D6E00023EA0505B4E763184A1CD2B21B7E84F80E
:10D6F000382090424FEA0323F0D922440231127EAF
:10D7000084F838101343EBE72DE9F041437A2DED0F
:10D71000028B0646B0EE408AF0EE608A49F2204461
:10D72000002B40F0E580C1F6FF740023C4F24023D3
:10D7300007EE103A47F6EE43C3F6FF6307EE903A62
:10D740000023E8EE077ACCF23C2306EE903AF4EEA2
:10D75000E67AF1EE10FA00F1C780F4EEC77AF1EE46
:10D7600010FAC8BF5F2740F35681337A49F220454B
:10D770004FF00108C1F6FF7503FA08F34146284649
:10D7800084F83B3084F85E8084F85D8003F0FCFA16
:10D790001621284603F0F8FA2846002103F0CCFBB6
:10D7A000002800F0E8800023327A4FF0010849F2A7
:10D7B000204002FA08F24146C1F6FF7047EA03052D
:10D7C00084F83B2084F85E8084F85D8003F0DCFA06
:10D7D00049F220401621C1F6FF7003F0D5FA49F254
:10D7E0002040C5F30721C1F6FF7003F0CDFA49F2DE
:10D7F0002040E9B2C1F6FF7003F0C6FA49F22040BA
:10D800004146C1F6FF7003F097FB0023C4F24023AA
:10D8100007EE103A47F6EE43C3F6FF6307EE903A81
:10D820000023E8EE877ACCF23C2306EE903AF4EE41
:10D83000E67AF1EE10FA59D4F4EEC77AF1EE10FA66
:10D84000C8BF5F2740F3DE80337A49F220454FF0AE
:10D850000108C1F6FF7503FA08F34146284684F82B
:10D860003B3084F85E8084F85D8003F08DFA1E21E1
:10D87000284603F089FA2846002103F05DFB0028C2
:10D8800057D00025337A49F220400126B340314673
:10D89000C1F6FF7084F83B3084F85E6084F85D6008
:10D8A00003F072FA49F220401E21C1F6FF7003F026
:10D8B0006BFA3D4349F22040C5F30721C1F6FF70E2
:10D8C00003F062FA49F22040E9B2C1F6FF7003F0BA
:10D8D0005BFABDEC028B49F220403146C1F6FF7085
:10D8E000BDE8F04103F028BB00273EE70027ABE787
:10D8F000037AC1F6FF740125AB402946204684F81F
:10D900003B3084F85E5084F85D5003F03DFA082106
:10D91000204603F039FA2046002103F00DFB0028D1
:10D9200051D0032302224FF484713046FFF768FE82
:10D93000FBE643460222317A284603F089FB0128A0
:10D940009FD995F8381095F83900814238D26B1874
:10D950004A1CD2B21B7E85F8382090424FEA03233E
:10D960002ED92A440231127E85F8381042EA030586
:10D9700025F07F0586E743460222317A284603F0E8
:10D9800067FB01287FF60FAF95F8381095F839003E
:10D99000814212D26B184A1CD2B21B7E85F8382005
:10D9A00090424FEA032308D92A440231127E85F8B7
:10D9B0003810134323F07F03F6E66FF07F03F3E69E
:10D9C0006FF07F055EE72B460222317A204603F096
:10D9D0003FFBA842A5D994F8383094F839108B420F
:10D9E0009FD25A19D2B2914284F8382099D9224450
:10D9F0000233127E84F8383002F00303022B3FF426
:10DA000094AE8EE79FED087A77EE877AFCEEE77AA0
:10DA100017EE907A18E79FED047A77EE877AFCEE9E
:10DA2000E77A17EE907AA0E600003C422DE9F04F2D
:10DA30002DED028B49F22044027AC1F6FF7483B0C7
:10DA400052000125002180462046B0EE408A84F82D
:10DA50003B2084F85E5084F85D5003F095F90E2168
:10DA6000204603F091F92046002103F065FA0028D2
:10DA700000F0D580B5EEC08AF1EE10FA56DCB5EEB6
:10DA8000C08AF1EE10FA00F344810C26B1464FF043
:10DA9000FF0A98F8082049F22045C1F6FF755200A8
:10DAA0004FF0010B0021284684F83B2084F85EB03B
:10DAB00084F85DB003F068F90E21284603F064F99C
:10DAC0002846002103F038FA0746002800F0F180CC
:10DAD000002798F8083049F220405B00012500211A
:10DAE000C1F6FF7084F83B3084F85E5084F85D50D6
:10DAF00003F04AF949F220400E21C1F6FF7003F00D
:10DB000043F949F220403946C1F6FF7003F03CF971
:10DB100049F220403146C1F6FF7003F035F949F271
:10DB200020402946C1F6FF7003F006FA0023C4F234
:10DB3000403307EE103A47F6EE43C3F6FF6307EEB5
:10DB4000903AE8EE077A98F8082049F22047FCEE70
:10DB5000E77AC1F6FF77CDED017A9DF80450C02D2C
:10DB600098BFC5F1FC054FEA42024FF001094FF0A2
:10DB70000001384694BF45EA052543F63C4584F844
:10DB80003B2084F85E9084F85D9003F0FDF810214E
:10DB9000384603F0F9F83846002103F0CDF906467F
:10DBA00000285BD0002698F8083049F220405B003E
:10DBB00001270021C1F6FF7084F83B3084F85E70C5
:10DBC00084F85D7003F0E0F849F220401021C1F6BE
:10DBD000FF7003F0D9F8354349F22040C5F307211F
:10DBE000C1F6FF7003F0D0F849F22040E9B2C1F667
:10DBF000FF7003F0C9F849F220403946C1F6FF70C2
:10DC000003F09AF928B1002003B0BDEC028BBDE807
:10DC1000F08FA8B203B0BDEC028BBDE8F08F0646D2
:10DC20002B46022298F80810204603F011FA01282A
:10DC30007FF620AF94F8383094F839108B422AD30D
:10DC40000C23B5EEC08AF1EE10FA67DD002B3FF42D
:10DC50006DAF4FF0F30A4FF000091AE74B4602226E
:10DC600098F80810384603F0F3F901289AD997F884
:10DC7000383097F83920934209D2591CC9B28A42E8
:10DC800087F8381003D9023387F838308BE700263D
:10DC9000CFF6FF7687E75A1CD2B2914284F838203B
:10DCA000CED922440233127E84F8383002F00C03BD
:10DCB000C7E75B46022298F80810284603F0C8F927
:10DCC00058457FF606AF95F8382095F8390082421E
:10DCD0001CD2A91802EB0B03DBB2097E85F83830A1
:10DCE00098424FEA012111D92B44023293F818A02F
:10DCF00085F838204AEA010A2AF00C0A4AEA09099A
:10DD00005FFA89FA4FEA19275646E2E6FF27564698
:10DD1000DFE60026B1464FF0F30ABAE60C2B3FF4DB
:10DD200005AFACE6F8B549F22044037AC1F6FF74BA
:10DD30000125AB4029460746204684F83B3084F84D
:10DD40005E5084F85D5003F01FF80021204603F078
:10DD50001BF80021204603F017F82946204603F05F
:10DD600013F82946204603F0E7F808B10020F8BD73
:10DD70003B7A84F85E505B0006460146204684F8F4
:10DD80003B3084F85D5002F0FFFF0A21204602F08C
:10DD9000FBFF3146204602F0F7FF7021204602F0DB
:10DDA000F3FF2946204603F0C7F8B0FA80F0400997
:10DDB000F8BD00BFFFFFFFFFF3EE047A80EE277A85
:10DDC0002DE9F04F98464FF4AA43C4F6571307467F
:10DDD00091460E4649F22044C1F6FF742DED068BA4
:10DDE00017EE100A83B008EE103AB0EE60AAF0EE1B
:10DDF000418A0DF0DDFB9FED9E0B41EC110B0BF00A
:10DE0000A7FFCAEE087AB0EE409AF0EE609A0125BC
:10DE100008EA0508F1EE677A17EE900A0DF0C8FBE4
:10DE20009FED930B41EC110B0BF092FFC8EE887A3B
:10DE30005BEC10ABF1EE677A17EE900A0DF0B8FBD1
:10DE40009FED8B0B41EC110B0BF082FF3B7A84F8BA
:10DE50005E50AB40294620468DED000B84F83B30E8
:10DE600084F85D5002F090FF2621204602F08CFFDE
:10DE70000021204602F088FF45F61C234FF0204287
:10DE8000C3F6E47351EC190B0DF0E6FB00230022FE
:10DE9000C4F2E0030DF0E0FB0DF0B6FEC1B2204687
:10DEA00002F072FF2946204603F046F83B7A84F8D8
:10DEB0005E50AB402946204684F83B3084F85D50E4
:10DEC00002F062FF2821204602F05EFF002120467A
:10DED00002F05AFF002152465B460020C3F6F07163
:10DEE0000DF006FA00230022C4F220130DF0B4FB5B
:10DEF0000DF08AFEC1B2204602F046FF29462046B8
:10DF000003F01AF83B7A84F85E50AB40294620466D
:10DF100084F83B3084F85D5002F036FF2A21204619
:10DF200002F032FF0021204602F02EFF9DED000B93
:10DF3000002153EC102B0020C3F6F0710DF0D8F93E
:10DF400000230022C4F260130DF086FB0DF05CFE8E
:10DF5000C1B2204602F018FF2946204602F0ECFF2D
:10DF60003A7A84F85E504FEA481309F00308022E0B
:10DF700043EA0828294602FA05F3204628BF02266C
:10DF800084F83B3084F85D5002F0FEFE24212046E8
:10DF900002F0FAFE2046002148EA063602F0CCFFE5
:10DFA00000283BD000233A7A012549F22040AA40BC
:10DFB0002946C1F6FF701E4384F83B2084F85E506A
:10DFC00084F85D5002F0E0FE49F220402421C1F6C1
:10DFD000FF7002F0D9FE49F22040C6F30721C1F6D6
:10DFE000FF7002F0D1FE49F22040F1B2C1F6FF709D
:10DFF00002F0CAFE49F220402946C1F6FF7002F045
:10E000009BFF28B1002003B0BDEC068BBDE8F08F6C
:10E01000B0B203B0BDEC068BBDE8F08F2B460222F8
:10E02000397A204603F014F80128BBD994F8381047
:10E0300094F83900814214D263184A1CD2B21B7E74
:10E0400084F8382090424FEA03230AD9224402314F
:10E05000127E84F83810134323F44C5323F020032A
:10E06000A1E74CF6DF43CFF6FF739CE7AFF30080E8
:10E0700000000000000024402DE9F041074649F26D
:10E080002044C1F6FF74012520463D7102F090FE48
:10E09000052008F0D9FA3B7A84F85E50AB400021A5
:10E0A000204684F83B3084F85D5002F06DFE30214C
:10E0B000204602F069FE4021204602F065FE602104
:10E0C000204602F061FE2946204602F035FF10B1DD
:10E0D0000020BDE8F0813B7A84F85E5006465B0084
:10E0E0000146204684F83B3084F85D5002F04CFE37
:10E0F0002621204602F048FE3146204602F044FE2A
:10E100006C21204602F040FE2946204602F014FF12
:10E110003B7A84F85E505B003146204684F83B3001
:10E1200084F85D5002F030FE2821204602F02CFEDB
:10E130002946204602F028FEF221204602F024FE65
:10E140002946204602F0F8FE3B7A84F85E505B00D8
:10E150003146204684F83B3084F85D5002F014FECE
:10E160002C21204602F010FE0F21204602F00CFE6A
:10E170002221204602F008FE2946204602F0DCFE5D
:10E180003B7A84F85E505B003146204684F83B3091
:10E1900084F85D5002F0F8FD3C21204602F0F4FDC9
:10E1A0004421204602F0F0FD4621204602F0ECFD1D
:10E1B0002946204602F0C0FE3B7A40F23712FA8030
:10E1C0005B003146204684F83B3084F85E5084F88A
:10E1D0005D5002F0D9FD2421204602F0D5FD2946EC
:10E1E000204602F0D1FD3721204602F0CDFD294620
:10E1F000204602F0A1FE3B7A84F85E505B00314677
:10E20000204684F83B3084F85D5002F0BDFD30219B
:10E21000204602F0B9FD4021204602F0B5FDFF2165
:10E22000204602F0B1FD2946204602F085FE3B7AE9
:10E2300084F85E505B003146204684F83B3084F819
:10E240005D5002F0A1FD0221204602F09DFD314605
:10E25000204602F099FD7321204602F095FD2946E3
:10E26000204602F069FE4FF4C87008F0EDF93B7AE1
:10E2700084F85E505B003146204684F83B3084F8D9
:10E280005D5002F081FD2E21204602F07DFD1D2112
:10E29000204602F079FD1D21204602F075FD294639
:10E2A000204602F049FE3B7A84F85E505B0031461E
:10E2B000204684F83B3084F85D5002F065FD04216F
:10E2C000204602F061FD3146204602F05DFD04214A
:10E2D000204602F059FD2946204602F02DFE3B7AE9
:10E2E00084F85E505B003146204684F83B3084F869
:10E2F0005D5002F049FD0621204602F045FD294609
:10E30000204602F041FD3021204602F03DFD294625
:10E31000204602F011FE3B7A84F85E505B003146E5
:10E32000204684F83B3084F85D5002F02DFD0A2130
:10E33000204602F029FD3146204602F025FD10213D
:10E34000204602F021FD2946204602F0F5FD3B7AE9
:10E3500084F85E505B003146204684F83B3084F8F8
:10E360005D5002F011FD0E21204602F00DFD3146F8
:10E37000204602F009FD3146204602F005FD2946FF
:10E38000204602F0D9FD3B7A84F85E505B003146AE
:10E39000204684F83B3084F85D5002F0F5FC1021F3
:10E3A000204602F0F1FC3C21204602F0EDFC3C212D
:10E3B000204602F0E9FC2946204602F0BDFD3B7AEA
:10E3C00084F85E505B003146204684F83B3084F888
:10E3D0005D5002F0D9FC2221204602F0D5FC7F21BD
:10E3E000204602F0D1FC7F21204602F0CDFC2946D8
:10E3F000204602F0A1FD3B7A4FF036085B00A7F8FB
:10E4000006803146204684F83B3084F85E5084F81C
:10E410005D5002F0B9FC2421204602F0B5FC3146E3
:10E42000204602F0B1FC4146204602F0ADFC2946F0
:10E43000204602F081FD7D722846BDE8F08100BFD4
:10E440002DE9F8430023C4F2013307EE103A47F6F2
:10E45000EE43C3F6FF6307EE903AE0EE077A064616
:10E46000FCEEE77A17EE904A002C71D0802C39D957
:10E47000337900242746002B3ED149F22045C1F6CE
:10E48000FF75337A49F220405B0001260021C1F676
:10E49000FF7085F83B3085F85E6085F85D6002F0BE
:10E4A00073FC49F220402221C1F6FF7002F06CFC9F
:10E4B00049F220403946C1F6FF7002F065FC49F28E
:10E4C00020402146C1F6FF7002F05EFC49F2204078
:10E4D0003146C1F6FF7002F02FFDB0FA80F040091E
:10E4E000BDE8F883C4F18004337944EA0424C4F31A
:10E4F0000727E4B2002BC0D0B6F80680337A49F281
:10E500002045C1F6FF7528F0100800215B0031712D
:10E51000A6F806804FF00109284685F83B3085F8BB
:10E520005E9085F85D9002F02FFC2846242102F0D1
:10E530002BFC4FEA1821284602F026FC08F0EF01D8
:10E54000284602F021FC4946284602F0F5FC98E7EF
:10E55000037A49F22045C1F6FF75012717EE901A9C
:10E56000BB400771284685F83B3085F85E7085F81A
:10E570005D7002F009FC2846222102F005FC2846C5
:10E580007F2102F001FC28467F2102F0FDFB394685
:10E59000284602F0D1FCB6F80680337A48F010081D
:10E5A0001FFA88F8BB40A6F806802146284685F861
:10E5B0003B3085F85E7085F85D7002F0E5FB28461B
:10E5C000242102F0E1FB4FEA1821284602F0DCFB8F
:10E5D0005FFA88F1284602F0D7FB3946284602F058
:10E5E000ABFCB0FA80F04009BDE8F883F8B5064608
:10E5F0000D4619B1012948D00020F8BD037A49F22F
:10E600002044C1F6FF745B000127204684F83B30AC
:10E6100084F85E7084F85D7002F0B6FB202120461D
:10E6200002F0B2FB2946204602F0AEFB55212046FF
:10E6300002F0AAFB3946204602F07EFC0028DBD11E
:10E64000F588337A45F00405ADB25B00F5800146EC
:10E65000204684F83B3084F85E7084F85D7002F0E8
:10E6600093FB2421204602F08FFB290A204602F06A
:10E670008BFBE9B2204602F087FB3946204602F0C8
:10E680005BFCB0FA80F04009F8BD037A49F22044FF
:10E69000C1F6FF745B000021204684F83B3084F80B
:10E6A0005E5084F85D5002F06FFB2A21204602F094
:10E6B0006BFB2946204602F067FB7321204602F0DF
:10E6C00063FB2946204602F037FC0746002893D119
:10E6D000337A84F85E505B000146204684F83B3074
:10E6E00084F85D5002F050FB2021204602F04CFBE4
:10E6F0003946204602F048FB8821204602F044FBC0
:10E700002946204602F018FC00287FF475AFF788F0
:10E71000337A27F004075B00F7800146204684F82F
:10E720003B3084F85E5084F85D5002F02DFB2421CC
:10E73000204602F029FB390A204602F025FB07F0AB
:10E74000FB01204602F020FB2946204602F0F4FBA4
:10E75000B0FA80F04009F8BD2DE9F04F9BB00446B7
:10E7600006F0CCF91690002800F05F8200212046C8
:10E7700006F064FA1790002800F060824FF6984384
:10E78000C0F20E03199345F24C6945F24E6734F915
:10E790000930049345F25266E35F099345F25460F1
:10E7A000A35F089345F25661235E189345F25862C1
:10E7B000635E059345F25A6AA35E079334F90A3003
:10E7C000069304F5AC431A4604F5C5491E46CDF838
:10E7D000449002F13C093E320B9206F140020C9249
:10E7E00006F142020D9206F144020E9206F1460233
:10E7F0000F9206F14802119B109232464A32039260
:10E800001A46183211921A461A3245F2506512927F
:10E8100045F25E681A4645F25C6C45F2606E1C3249
:10E820001E3334F905B0139234F9088034F90CC062
:10E8300034F90EE0CDF808901493179B18989A1CA1
:10E840000192169A03F5817302321593019B0A9285
:10E850004FF0000A5D4633F9022F019302EB0212DA
:10E8600002EB0222520022F34F42029B04991E88BF
:10E8700004EB460701FB0CF9B7F91C3003FB0899C0
:10E8800029F3CF390FFA89F1049112B201FB0EF985
:10E8900029F3CF39914409F30F090136A7F81C90E9
:10E8A0000299B6B240F25B47BE4294BF0E80A1F817
:10E8B00000A00B99099F0E8804EB460907FB0CFB8F
:10E8C000B9F9D4783B4407FB08BB2BF3CF3B0FFAD5
:10E8D0008BF7099707FB0EF727F3CF37174407F39A
:10E8E0000F070136A9F8D4780B99B6B240F2A347C6
:10E8F000BE4294BF0E80A1F800A00C990E8804EBD4
:10E90000460707F590571C37B7F9009005FB0CF543
:10E910004B4409FB085525F3CF352DB205FB0EF905
:10E9200029F3CF39914409F30F090136A7F8009074
:10E93000B6B240F2FC47BE4294BF0E80A1F800A0E0
:10E940000D990E88089904EB460707F5E05716372E
:10E95000B7F9009001FB0CFB4B4409FB08BB2BF300
:10E96000CF3B0FFA8BF9CDF8209009FB0EF929F374
:10E97000CF39914409F30F090136A7F800900D999A
:10E98000B6B240F24B57BE4294BF0E80A1F800A031
:10E990000E990E8804EB460707F51A572E37B7F97C
:10E9A000009000FB0CF04B4409FB080020F3CF3033
:10E9B00000B200FB0EF929F3CF39914409F30F0996
:10E9C0000136A7F80090B6B240F28D57BE4294BF10
:10E9D0000E80A1F800A00F990E88059904EB460758
:10E9E00007F547570A37B7F9009001FB0CFB4B447A
:10E9F00009FB08BB2BF3CF3B0FFA8BF9CDF8149032
:10EA000009FB0EF929F3CF39914409F30F090136B7
:10EA1000A7F800900F99B6B240F2D257BE4294BF09
:10EA20000E80A1F800A010990E88079904EB460704
:10EA300007F575573037B7F9009001FB0CFB4B44D5
:10EA400009FB08BB2BF3CF3B0FFA8BF9CDF81C90D9
:10EA500009FB0EF929F3CF39914409F30F09013667
:10EA6000A7F800901099B6B240F21467BE4294BF66
:10EA70000E80A1F800A003990E88069904EB4607C2
:10EA800007F593471A37B7F9009001FB0CF14B4497
:10EA900009FB081121F3CF3109B2069101FB0EF9F0
:10EAA00029F3CF394A4402F30F020136B6B2B6F564
:10EAB000CA6F3A808ABF039A0399A2F800A047F66A
:10EAC000E12298BF0E8002FB03F323F34F43119919
:10EAD0000E8804EB460707F5AC470FFA83F9B7F940
:10EAE000622003EB6203A7F86230C9EB020222F353
:10EAF0004F020136B6B2B6F50B7F34BF0E80A1F8D7
:10EB000000A012990E8804EB460707F5B5470FFAE7
:10EB100082F9B7F93A3002EB63027A87C9EB030353
:10EB200023F34F030136B6B2B6F5DC7F94BF0E80F7
:10EB3000A1F800A013990E8804EB460707F5BC471F
:10EB40000FFA83F9B7F92C2003EB6203BB85C9EBFD
:10EB5000020222F34F020136B6B2B6F5AA7F94BF85
:10EB60000E80A1F800A014990E8804EB460707F563
:10EB7000C1470FFA82F9B7F9563002EB6302A7F8E2
:10EB80005620C9EB030323F34F030136B6B21BB281
:10EB9000E02EC3EB031394BF0E80A1F800A05B002E
:10EBA00003F30F030A9A22F8023F019B0A92159A77
:10EBB00093427FF450AE0499002213461E4661F33F
:10EBC0000F02079965F30F03354661F30F050999A5
:10EBD00061F31F42089961F31F43059960F30F0623
:10EBE00061F31F46069945F2546E45F2586C45F2A2
:10EBF000506045F24C6761F31F45E251235044F8E1
:10EC00000E60204644F80C50169C0022214605F068
:10EC1000FBFF204605F0CAFF1798199A90420AD0C8
:10EC20001BB0BDE8F04F05F0C1BF0146204606F01D
:10EC300005F80028F4D11BB0BDE8F08F4FF69843DB
:10EC4000C0F20E03199317939DE500BFF8B54FF678
:10EC5000DC630446C0F2010303600021012004F1DB
:10EC600018020B46607222612172E16000E02269A5
:10EC700042F82310627A01339A42F8DC4FF288534B
:10EC8000C2F200031A680AB9B9E01A465369002BA8
:10EC9000FBD1546120464FF6A4530025C0F20E0369
:10ECA0006561A580E580A572294640F81C3B40F6C9
:10ECB000B8020DF001FD294640F6481204F6D400D2
:10ECC0000DF0FAFC04F59050294640F6FA121C307B
:10ECD0000DF0F2FC04F5E050294640F6982216307B
:10ECE0000DF0EAFC04F51A50294640F61C322E308D
:10ECF0000DF0E2FC04F54750294640F6A6320A30F2
:10ED00000DF0DAFC04F57550294640F62A42303001
:10ED10000DF0D2FC04F59340294640F6A2421A3089
:10ED20000DF0CAFC45F23C6345F23E6045F2406797
:10ED300045F2426145F24462E55245F2466625528B
:10ED400045F2486345F24A60E553655245F24C6727
:10ED5000A55245F24E6145F25062A553E55245F287
:10ED60005266255245F2546345F25660E5536552AA
:10ED700045F25867A55245F25A6145F25C62A553C7
:10ED8000E55245F25E66255245F2606341F6991000
:10ED9000E553655246F26767A05246F6843204F5A1
:10EDA000AC402946A7536230E2524FF48B620DF01B
:10EDB00083FC04F5B540294640F272323A300DF03A
:10EDC0007BFC04F5BC40294640F2AA222C300DF011
:10EDD00073FC04F5C14029464FF4E17256300DF042
:10EDE0006BFC46F2982046F29A2146F29C2246F2AB
:10EDF0009E23255265522046A552E552F8BD1C605F
:10EE000048E700BF10B5044606F03EF9204610BDA5
:10EE100049F2A0224EF605614EF64810C1F6FF7287
:10EE2000C0F20001C2F200000DF0D2B838B549F2CC
:10EE3000A0254EF60564C1F6FF75C0F200044EF63B
:10EE400050102A462146C2F200000DF0C1F84EF6DD
:10EE500058102A462146C2F20000BDE838400DF0A5
:10EE6000B7B800BF49F2A0224EF605614EF6601019
:10EE7000C1F6FF72C0F20001C2F200000DF0A8B8A6
:10EE800049F2A0224EF605614EF66810C1F6FF72F7
:10EE9000C0F20001C2F200000DF09AB849F2A022BF
:10EEA0004EF605614EF67010C1F6FF72C0F2000119
:10EEB000C2F200000DF08CB849F2A0224EF60561B6
:10EEC0004EF67810C1F6FF72C0F20001C2F20000E7
:10EED0000DF07EB82DE9F04F00F5807EB1E8A00A74
:10EEE000B2E84015C5EA0643C6EA2544C7EA084524
:10EEF000C8EA2746C9EA0A47CAEA2948CBEA0C49C0
:10EF0000CCEA2B4AA0E8F8078645E7D1BDE8F04FE8
:10EF100070474FF000022DE9F00F00F5807C00BF34
:10EF2000B1E8A00AC5EA0203C2EA2544C7EA02051D
:10EF3000C2EA2746C9EA0207C2EA2948CBEA02091F
:10EF4000C2EA2B4AA0E8F8078445E9D1BDE8F00FF2
:10EF500070474FF000022DE9F00F00F5807C00BFF4
:10EF6000B1E8A00AC2EA0543C2EA0504C2EA0745BD
:10EF7000C2EA0706C2EA0947C2EA0908C2EA0B491F
:10EF8000C2EA0B0AA0E8F8078445E9D1BDE8F00F12
:10EF900070472DE9F00F089C00F5007B51F8045BE9
:10EFA00053F8046BC5EA0647C6EA254952F8045BE4
:10EFB00054F8046BC5EA0648C6EA254AA0E880076B
:10EFC0008345EBD1BDE8F00F704700BF2DE9F84352
:10EFD0004FF00008064600F1180547464146304606
:10EFE000002F4FD005F02AFEF0B12C68B4F5803F19
:10EFF00007F1040100F1040E07F5827C27D05EF8CA
:10F00000042B34FB02F334FB12F903F30F0209F370
:10F010000F03C2EA03430A6893FA12F341F8043B70
:10F020008C45ECD805F0C2FD08F10108B8F1040FD9
:10F0300005F10405D2D1002F40D0304639460022D8
:10F0400005F0E2FD3846BDE8F84305F0AFBD07F135
:10F050000C0100F10C0451F8083C54F8082C93FA08
:10F0600012F341F8083C54F8042C51F8043C93FA8C
:10F0700012F38C4541F8043C04F1080401F1080145
:10F08000E9D8CFE705F0E6FD07460028CCD0286890
:10F09000B0F5803FC8D0391D07F582740B6830FB8E
:10F0A00003F230FB13F302F30F0203F30F03C2EA80
:10F0B000034341F8043B8C42F0D8B5E7BDE8F88340
:10F0C00070B584692CB3B4F5803F06464FF000015B
:10F0D00025D005F0BFFD054600B3011D00F5827087
:10F0E0000B6834FB03F234FB13F302F30F0203F358
:10F0F0000F03C2EA034341F8043B8842F0D830468C
:10F100000022294605F080FD2846BDE8704005F044
:10F110004DBD214605F092FD0028F6D170BD05F0E9
:10F120008DFD04460028F9D030462146002205F026
:10F130006BFD2046BDE8704005F038BD49F2A022C5
:10F140004EF605614EF68010C1F6FF72C0F2000166
:10F15000C2F200000CF03CBF49F2A0224EF605615D
:10F160004EF68810C1F6FF72C0F20001C2F2000034
:10F170000CF02EBF49F2A0224EF605614EF690101B
:10F18000C1F6FF72C0F20001C2F200000CF020BF15
:10F190002DE9F84F4EF69C13C2F2000348F21F020D
:10F1A00019681B79096848F20050C1F6FF70C4F273
:10F1B00000028142137035D24EF6B413C2F200033E
:10F1C0001B7893BB4EF6AC19C2F200094EF6A41898
:10F1D0004EF698154EF6A816C2F20008C2F20005C7
:10F1E000C2F20006D9F800A0D8F800B02C88378801
:10F1F000BAF1000F45D0BBF1000F3AD00BF1040279
:10F200000AF1040102EB470201EB4401FFF762FE41
:10F21000403740347F2C1ED82C807F2F0CD837806D
:10F22000BDE8F88FA0F58070CCE74EF20823CEF24F
:10F23000000301221A60C5E700245846348005F017
:10F24000B5FC4EF6B013C2F200031A68C8F80020ED
:10F250001C60BDE8F88F002450462C8005F0A6FC09
:10F260004EF6B813C2F200031A68C9F800201C60F9
:10F27000D3E70AF1040101EB4401FFF74AFE4034F1
:10F28000C8E7BBF1000F07D00BF1040101EB470108
:10F29000FFF75FFE4037BDE74FF4807259460DF02F
:10F2A0000BFAB7E7F8B50021054605F0C7FCC8B171
:10F2B00072B64EF6AC13C2F200031968002938D0BA
:10F2C0004EF6B812C2F20002166866B34EF69814F3
:10F2D000C2F2000400271E601060278062B6084654
:10F2E00005F064FC2846012105F0A8FCD0B172B6F7
:10F2F0004EF6A413C2F200031C6814B34EF6B0120B
:10F30000C2F2000215688DB14EF6A811C2F20001DA
:10F3100000261D6010600E8062B62046BDE8F840F1
:10F3200005F044BCF8BD106062B6DBE7106062B661
:10F33000F8BD4EF69812C2F200021860118062B653
:10F34000D0E74EF6A812C2F200021860148062B62E
:10F35000F8BD00BF4EF69C10F8B5C2F200000121C6
:10F3600005F0ECFD48F23C03C4F204034EF6AC1485
:10F3700019684EF6A410C2F20004C2F2000048F26E
:10F3800040020025C4F2040241F4004125600560FA
:10F390001960116841F0020111601A684FF4704160
:10F3A00042F00202C4F202011A600B68AB427DDB3C
:10F3B0004FF28003C4F202031B68AB4276DB4FF4CA
:10F3C0007142C4F202024FF0804313601368002BB5
:10F3D000FCDB4FF20410C4F202004FF26003C4F2EF
:10F3E00002034FF2FE054FF2040E0560C4F2020E56
:10F3F00000251D604FF2080101234FF20C07CEF8E3
:10F400000030C4F20201C4F202079E46C0F2007E40
:10F410004FF4803C4FF21002C1F800E0C4F2020247
:10F42000C7F800C041F61B7763F31F474FF214067D
:10F430004FF2E0044FF284001760C4F20206C4F2F7
:10F440000204C4F202004FF288014FF4F852C4F2F1
:10F450000201C1F61F7241F61B77326063F31F474A
:10F4600025600360C4F200730B604FF28C0E4FF204
:10F4700090064FF294054BF208044BF20C004BF24D
:10F480001801C4F2020EC4F20206C4F20205C4F26C
:10F490000404C4F20400C4F204014FF4C063CEF8C3
:10F4A00000C037602A60236003600B604EF69C1436
:10F4B000C2F200044BF204002368C4F2040048F2D4
:10F4C000004202214FF4C065C1F6FF7205601A6068
:10F4D00099802279996002F180424FF2220102F56F
:10F4E0000432C4F2020140F201164FF47E45196164
:10F4F000DE8000214FF48070CFF6FF7506278D2641
:10F50000D882DD609982D88399619F8311701670CB
:10F5100005F0B0FC22794EF6B4115311C2F200018D
:10F5200048F21B06C4F200069B00087003F160431A
:10F5300002F01F004FF4704548F200640121327060
:10F54000C4F2020502F11007814003F56143C1F6E0
:10F55000FF7401204FF29112C9F200004FF0807643
:10F56000C0F200022E60286044F827201960F8BD20
:10F5700049F2A0224EF605614EF69C10C1F6FF72CC
:10F58000C0F20001C2F200000CF022BD49F2A0223C
:10F590004EF605614EF6BC10C1F6FF72C0F20001D6
:10F5A000C2F200000CF014BD49F2A0224EF6056133
:10F5B0004EF6C410C1F6FF72C0F20001C2F20000A4
:10F5C0000CF006BD49F2A0224EF605614EF6CC10B5
:10F5D000C1F6FF72C0F20001C2F200000CF0F8BCEC
:10F5E00049F2A0224EF605614EF6D410C1F6FF7224
:10F5F000C0F20001C2F200000CF0EABC49F2A02205
:10F600004EF605614EF6DC10C1F6FF72C0F2000145
:10F61000C2F200000CF0DCBC90F89D3090F89C2009
:10F62000DBB2934215D001331F2B84BF00210B4660
:10F6300010B598BFD9B20633002250F8234080F8A5
:10F640009D10214605F0E0FA2046BDE8104005F087
:10F65000ADBA7047D0F898300BB10120704710B5A3
:10F66000044605F04BFAC4F89800003018BF01209A
:10F6700010BD00BF10B50446D0F8980018B1043092
:10F6800010BD09F0C9FC05F039FAC4F8980000284B
:10F69000F7D0043010BD00BFD0F89810B1B190F889
:10F6A0009C2001321F2A10B4CABF0024D4B22246C3
:10F6B00090F89D309342FBD00632002340F8221090
:10F6C00080F89C405DF8044BC0F89830704700BF4C
:10F6D00010B4047F4160022CC26003D05DF8044B7B
:10F6E00005F0F0BC83685DF8044B1847F0B449F2AC
:10F6F0007033C1F6FF7348F21F02996BC4F2000227
:10F7000008791070586B48F21C02C4F200020479A8
:10F710001470097911701A6B002A4FD05968C968A2
:10F720008A4247D80168CC8B240402F1FF3073D49D
:10F73000C0F30E00C883C88B80B2C882996B096879
:10F74000C88B000460D4C2F30E00C883C88B0024A9
:10F7500080B212F1FF32C88218BF01221C63596BBC
:10F76000086849F270310568C1F6FF7101F12C0497
:10F77000A54241D00968CC6814F0804F0468056840
:10F7800015BF248824780235013544F00044056013
:10F790004C63996B48F21B03C4F20003097919709A
:10F7A00049F27031C1F6FF7112B14A6B12791A70C9
:10F7B000F0BC7047521A1A630122D0E71968D86B5F
:10F7C0000A630024CFF60F74CC620468CD68266803
:10F7D0004FF2D164C0F2000425F080450327A64211
:10F7E000CD6083F82D701FD1037F4260022BC26071
:10F7F0001ED0F0BC05F066BC086891F82C10C468F7
:10F8000041F000414163C4E7CC8BC2F3080004F42B
:10F810007E442043C88399E7CC8BC0F3080004F4EE
:10F820007E442043C88386E733461146F0BC184720
:10F830008368F0BC184700BF00207047704700BFC6
:10F840004EF6E413C2F2000302224FF67461C0F2D6
:10F850000E015A600022D9629A7083F8242083F83E
:10F86000302083F83220704741F23801C4F20B0196
:10F8700041F230020B6823F0805323F00A030B603F
:10F88000C4F20B0213689907FCD541F22C03C4F2B1
:10F890000B031A68920703D51A6822F002021A6055
:10F8A00041F22803C4F20B034EF63822196821F006
:10F8B000080119601968C2F2000241F00801012034
:10F8C00019601060704700BF830769D1F0B54EF62C
:10F8D0003C24C2F2000423780BB10320F0BD41F2B6
:10F8E0002402C4F20B0215461368DE07FCD42B6811
:10F8F0009B07F9D4637803B9490241F23003C4F29B
:10F900000B0341F234021C681C60C4F20B0241F28A
:10F910003804136823F4081323F0310343F08053B1
:10F9200041F22C05C4F20B0543F00A03C4F20B04A8
:10F93000136023682E684EF6382246F002064FF414
:10F94000805EC2F200022E60C4F20B0E002541F26E
:10F9500008071560C4F20B0741F2040641F20C05DA
:10F96000CEF8000043F08053C4F20B06C4F20B053E
:10F970001120396043F00A03C1F222104FF48131A3
:10F980003160236028601368002BFCD041F2300303
:10F99000C4F20B0300201A6802F003021A60F0BDE3
:10F9A0004FF0FF30704700BF830740F0AD802DE976
:10F9B000F0414EF63C25C2F200052B7813B103202E
:10F9C000BDE8F08141F22402C4F20B021446136830
:10F9D000DF07FCD423689E07F9D46B7803B949028A
:10F9E00041F23003C4F20B0341F234021C681C6084
:10F9F000C4F20B0241F23804136823F4081323F015
:10FA0000310343F0805341F22C06C4F20B0643F05D
:10FA10000A03C4F20B041360236837684EF63822D9
:10FA200047F002074FF4805E3760C2F20002C4F272
:10FA30000B0E41F20807C4F20B0700261660CEF841
:10FA4000000041F2040641F20C00396043F080539B
:10FA5000C4F20B06C4F20B00012143F00A034FF479
:10FA60008137C1F622013760236001601368002BE3
:10FA7000FCD041F23003C4F20B0341F224021968B6
:10FA800001F003011960C4F20B0213685907FCD49A
:10FA900041F2240141F23002C4F20B01C4F20B0224
:10FAA00041F2340741F2080841F20C0C41F2100611
:10FAB0008E461446C4F20B07C4F20B08C4F20B0CBA
:10FAC000C4F20B060B68DB07FCD4DEF800309807A5
:10FAD000F8D43B6843F001033B60136813600020D7
:10FAE0006B68C8F80030C0F60250CCF8000013680C
:10FAF000DB07FCD5236803F001032360306810F4B2
:10FB00000070DFD1BDE8F0814FF0FF30704700BFDB
:10FB1000F0B54FF23466C2F2000683B03368019349
:10FB20004FF44044C4F20204019F0546A4464FF03E
:10FB3000004EFF20236843F480632360C4F82CE068
:10FB40006063E36A002BFCDADCF83830DBB2FF2BB1
:10FB500006D033680093009BDB1BB3F5967FE9D397
:10FB60004FF44043C4F202034FF00046186841F0DE
:10FB7000400440F480601860DE6218465C63C36A2B
:10FB8000002BFCDA4FF44044C4F2020418204FF07A
:10FB90000047266822FA00F346F48066DBB226604E
:10FBA000E7626363E36A002BFCDA083810F1080FA0
:10FBB000EFD1002932D008290CBF8721FF214FF453
:10FBC0004043C4F202034FF000401A6842F48062DE
:10FBD0001A60D8621A465963D36A002BFCDA4FF4D4
:10FBE0004042C4F20202164600274FF00044FF21B3
:10FBF000136843F480631360D4625163D36A002BAB
:10FC0000FCDAB36BD8B21B06687001D403B0F0BD48
:10FC10000137B7F5807FEBD103B0F0BD9521CEE77A
:10FC20002DE9F0414EF650258378C2F20005032BF2
:10FC30002B780F4682B00446164618BF4F02002BA1
:10FC40006AD00021207806F067FC3A461121204650
:10FC5000FFF75EFF60BB4FF23460C2F200004FF46A
:10FC6000404103680093C4F20201DDF800808C4635
:10FC70004FF0004EFF270B6843F480630B60C1F820
:10FC80002CE04F63CA6A4FF44043002AC4F20203D7
:10FC9000F8DADCF83820D2B2FF2A627040F09180A6
:10FCA00003680193019BC8EB0303B3F5967FE2D988
:10FCB0002078012106F030FC2B784EF65022C2F25B
:10FCC00000022BB349F27033C1F6FF730020D97ADA
:10FCD00010700A46E1B1CC0706D54FF46142CEF26E
:10FCE0000002D86910600A46880706D54EF2041251
:10FCF000CEF20002196A1160DA7A510700F1EE8043
:10FD0000120705D54EF20C12CEF200029B6A136068
:10FD1000002002B0BDE8F08149F27033C1F6FF73F4
:10FD20004EF64C22C2F20002D97A126801202870E5
:10FD3000002933D072B6D97A11F0010F08460DD0E0
:10FD40004EF2801CCEF2000CD868DCF800E00EEA1F
:10FD5000000EC3F81CE00846CCF800E089070BD57C
:10FD60004EF2841ECEF2000E1869DEF8001001403B
:10FD70001962CEF80010D87A41070BD54EF2881ED2
:10FD8000CEF2000E5869DEF8001001405962CEF83C
:10FD90000010D87A010700F1A98062B61B68D96803
:10FDA00091423FF44EAF44F20100C0F23F00002107
:10FDB0001860C8F23F0142F08040DA6018611960B3
:10FDC0003FE7FE2A7FF474AF4FF480604FF6FF7177
:10FDD000C9F20001C8F21F0018608E4659631A4626
:10FDE00059631846596306F5FE77B11CD36A13F0C0
:10FDF000F00FFBD0C0F834E0836B01F8013C1B121C
:10FE000001F8023C02318F42F0D106F5FD7106F592
:10FE10000076B14210D24FF44042C4F202021746BB
:10FE2000D36A13F0F00FFBD0BB6B181201F8020B72
:10FE3000B14201F8013CF3D34FF44043C4F2020352
:10FE40004FF480614FF6FF72C8F21F01C9F2000241
:10FE5000196019465A63CA6A4FF4404312F0F00F12
:10FE6000C4F20203F7D020789B6B012106F054FB0B
:10FE70002B784EF65022C2F200025BB349F2703387
:10FE8000C1F6FF730020D97A10700A4611B3C80773
:10FE900006D54FF46142CEF20002D86910600A46DE
:10FEA0008F0706D54EF20412CEF20002196A1160D5
:10FEB000DA7A560706D54EF20812CEF20002596AD7
:10FEC0001160DA7A150705D54EF20C12CEF2000257
:10FED0009B6A1360012002B0BDE8F0814EF2081267
:10FEE000CEF20002596A1160DA7A09E74EF28C1EEE
:10FEF000CEF2000E9869DEF8001001409962CEF84B
:10FF000000104AE7F0B44FF44046C4F202064FF046
:10FF10000047336843F4806333603D46F7623446FC
:10FF200071633346511C02F20127E26A002AFCDAAF
:10FF30001A6811F8016C42F480621A60DD625E6337
:10FF4000E26A002AFCDA1A6811F8026B42F4806255
:10FF5000B9421A60DD625E63E7D14FF44041C4F2FA
:10FF60000201CA6A4FF44043002AC4F20203F8DADD
:10FF70001A684FF0004542F48062FF241A60194667
:10FF8000DD625C63CA6A4FF44043002AC4F2020394
:10FF9000F8DA1A684FF0004542F48062FF241A60D4
:10FFA0001946DD625C63CA6A4FF44043002AC4F21A
:10FFB0000203F8DA1A684FF0004542F48062FF2429
:10FFC0001A601946DD625C63CA6A4FF44043002A36
:10FFD000C4F20203F8DA9B6BDBB203F01F0243703A
:10FFE000A2F10500B0FA80F04009F0BC704700BFF4
:10FFF0002DE9F041064682B0002900F0AC804EF6B3
:020000021000EC
:1000000050258378C2F20005032B2B780C46174647
:1000100018BF4C02002B3FD00021307806F07CFA4C
:10002000224618213046FFF773FD002800F0988023
:100030003078012106F070FA2B784EF65022C2F289
:1000400000022BB349F27033C1F6FF730020D97A56
:1000500010700A46E1B1CC0706D54FF46142CEF2EA
:100060000002D86910600A46880706D54EF20412CD
:10007000CEF20002196A1160DA7A510700F1A48009
:10008000120705D54EF20C12CEF200029B6A1360E5
:10009000002002B0BDE8F08149F27033C1F6FF7371
:1000A0004EF64C22C2F20002D97A12680120287062
:1000B00000293DD072B6D87A10F0010F01460DD05C
:1000C0004EF2801CCEF2000CD968DCF800E00EEA9B
:1000D000010EC3F81CE00146CCF800E080070BD508
:1000E0004EF2841ECEF2000E1869DEF800100140B8
:1000F0001962CEF80010D97A48070BD54EF2881E47
:10010000CEF2000E5869DEF8001001405962CEF8B8
:100110000010D97A09070AD54EF28C1ECEF2000ED5
:100120009869DEF8001001409962CEF8001062B6BE
:100130001B68D96891423FF46FAF44F20100C0F2EE
:100140003F0000211860C8F23F0142F08040DA60B1
:100150001861196060E74EF65025C2F2000567E7A6
:100160003A46FE213046FFF7CDFE00283FF460AF4F
:100170004FF23461C2F200014FF440420B68019328
:10018000C4F20202DDF8048094464FF0004EFF20D6
:10019000136843F480631360C2F82CE05063D36AA1
:1001A0004FF44044002BC4F20204F8DADCF8387053
:1001B000FFB2FF2F10D00B680093009BC8EB030326
:1001C000B3F5167FE4D333E74EF20812CEF2000205
:1001D000596A1160DA7A53E700220D213046FFF7A1
:1001E00097FC00287FF424AF23684FF0004243F4CB
:1001F000806323602146E2626763CA6A4FF440432A
:10020000002AC4F20203F8DA9B6B13F0FF047FF4B8
:100210000FAF3078012106F07FF92B784EF650228F
:10022000C2F2000253B349F27033C1F6FF73147087
:10023000D97A0A4611B3C80706D54FF46142CEF207
:100240000002D86910600A468F0706D54EF20412E4
:10025000CEF20002196A1160DA7A560706D54EF21C
:100260000812CEF20002596A1160DA7A150705D534
:100270004EF20C12CEF200029B6A1360012008E7D6
:100280004EF64C23C2F2000342F20302C3F6000210
:100290001A6070472DE9F04F837987B0012B05462E
:1002A000029205D001232B71002007B0BDE8F08F2A
:1002B00042799007F6D553070E4626D5EB68AF690D
:1002C000BB4200F03781002F00F058812A6A147C6D
:1002D000591E09347A1EE14022FA04F4A14200F2C8
:1002E0005181002B00F04E81641A05F1080806E0E8
:1002F000A968286A00F062FC013C0028D2D042467E
:10030000002CF5D1EF603B4600E0EB68029A002A32
:1003100000F09C8049F2B0324EF660414EF6602B00
:10032000C1F6FF72C2F20001029F0192C2F2000BFD
:100330000391286A0279013A02EA532212F0FF0976
:10034000C3F3080840F08B80B8F1000F40F08780BD
:10035000A968002940F0BE80EB69002B00F0D08036
:10036000AB60C8F50074017C4269A4B2023B8B40CB
:100370004A44BC4203EB020973D9BCB2B8F1000F86
:1003800004D1A869EB68834280F086804846012149
:1003900000F030FA002885D008EB0B0318198342CF
:1003A0004ED008F10408321DD844934238BF464568
:1003B00043EA060E2CBF01220022591C1EF0030F37
:1003C00002F00102C1EB000E18BF00220EF101097C
:1003D0009C46002A6ED0B9F1090F6BD9AEF1030229
:1003E000920801324FEA820AA6F104084FF0000E8B
:1003F00000940EF1010E58F8044F4CF8044B96454A
:10040000F7D3CA45009C06EB0A0C03EB0A0E13D087
:1004100016F8228003F822800EF1010398420BD0D7
:100420009CF801308EF801300EF10203984203D09F
:100430009CF802308EF80230C1F1010108440644F4
:10044000EB683F1B2344EB607FF473AFAA699A42C9
:1004500075D26A79AB6142F080026A717BE0AB6869
:100460007FE7B4F5007F89D1019B1B6899452CD0AB
:100470004EF65C23C2F20003494618680378FE2B4F
:1004800051D03246FFF7B4FD00283FF40BAF06F51C
:1004900000764FF40074D3E700F05EF900283FF4D3
:1004A00001AF039A01991378C1F8009043F001035A
:1004B000137071E7013B721E00F1FF3C12F801EF6F
:1004C00003F801EF9C45F9D1B6E7019A4FF0FF33ED
:1004D0001360CDE705AA00F071FB00283FF4E5AEFC
:1004E000286A059B90F820404FF6F872C0F6FF721C
:1004F0004FF6F871102C08BF0A469342FFF430AF54
:1005000005F10802012100F0EDF900283FF4CAAE20
:10051000EB69002B30D16A79AB68EB6162F07F0246
:100520006A71286A1DE73046FFF73EFAB0FA80F09C
:100530004009A9E7029900297FF4ECAE0BE04EF6E2
:100540005423C2F200036A791B6823B1029B13B1E2
:1005500042F080026A7111070AD5AB79002B3FF493
:10056000A1AE120611D400F0F7F800283FF49AAEBD
:10057000029807B0BDE8F08FAB68D2E7AF60EF60DC
:100580003B46C3E6EB69AB60AFE60121286900F0AA
:1005900031F900283FF486AE4EF660232C7DC2F27E
:1005A000000313EB44143FF47DAEAB794EF65422B6
:1005B000012B9CBFAB69E361C2F20002EB691268D8
:1005C00063831B0CA38232B104F1160104F11800FD
:1005D0009047238B63826B7903F07F036B71C2E7D3
:1005E00000B583B002AB012203F8011D1946FFF7E5
:1005F00051FE03B05DF804FB2DE9F84F90F8203070
:10060000C66949F2B038102B05460F469146C1F62F
:10061000FF7822D006EBD116D8F800108E422FD1E9
:100620004EF66044C2F200044EF6602307F07F07E6
:10063000C2F2000343F8279023782A7E43F0010397
:10064000012A237054D9AA684EF65823C2F2000337
:10065000114419600120BDE8F88F06EB1126D8F887
:100660000010B1420CD14EF66044C2F200044EF6C6
:100670006023FFB2C2F20003314623F81790DBE794
:100680004EF66044C2F200044EF65C2A2378C2F2B1
:10069000000AA3B9DAF800000378FE2B2BD04EF63F
:1006A0006022C2F200023146FFF7BAFAE8B195F8CB
:1006B0002030C8F80060102BD9D03146B4E7DAF802
:1006C00000000378FE2B32D04EF66022C2F2000208
:1006D000FFF78EFC48B14EF6582BC2F2000BDBF848
:1006E000001099B900232370D4E70020BDE8F88FEB
:1006F0000120BDE8F88F4EF66020C2F200003146BE
:10070000FFF7E2F8B0FA80F04009CFE7DAF800002E
:100710000378FE2B15D04EF66022C2F20002FFF7DE
:1007200067FC0028E1D00023CBF80030DAE74EF672
:100730006020C2F20000FFF737F9B0FA80F04009FC
:10074000C8E74EF66020C2F20000FFF72DF9B0FABC
:1007500080F04009E5E700BF70B54EF66044C2F294
:10076000000423780BB9012070BD4EF65C25C2F25F
:10077000000549F2B03328680278C1F6FF73FE2AFB
:10078000196820D04EF66022C2F20002FFF730FC5A
:10079000B8B14EF65826C2F20006316819B90023E6
:1007A0002370012070BD28680378FE2B15D04EF60B
:1007B0006022C2F20002FFF71BFC10B1002333607D
:1007C000EDE7002070BD4EF66020C2F20000FFF79A
:1007D000EBF8B0FA80F04009DAE74EF66020C2F29A
:1007E0000000FFF7E1F8B0FA80F040090028E5D1F9
:1007F000E7E700BF2DE9F84349F2B035C1F6FF75D0
:1008000088462B68834218D04EF66044C2F200043A
:100810004EF65C2722780646C2F20007C2B9386855
:100820000378FE2B38D04EF66022C2F20002314629
:10083000FFF7F6F910B32E6003E04EF66044C2F203
:100840000004217848EA010121700120BDE8F88305
:1008500038680278FE2A14D04EF660221946C2F299
:100860000002FFF7C5FB48B14EF65829C2F2000955
:10087000D9F80010D9B900232370D0E70020BDE8D3
:10088000F8834EF660201946C2F20000FFF78CF89C
:10089000B0FA80F04009E6E74EF66020C2F20000B0
:1008A0003146FFF711F8B0FA80F04009C2E7386826
:1008B0000378FE2B0BD04EF66022C2F20002FFF747
:1008C00097FB0028DAD00023C9F80030D3E74EF6B2
:1008D0006020C2F20000FFF767F8B0FA80F040092C
:1008E000EFE700BF2DE9F04F136889B0002B00F04F
:1008F000AF8003F1010A00230693C3685E1CB04673
:10090000002B44D05446A04538BF022401910592E3
:100910004EF660234EF660424EF65C21C2F20003B2
:10092000C2F20002C2F2000138BFA246B44205463C
:10093000029203914FF00007994628D895F820308D
:10094000EE6949F2B03B102BC1F6FF7B2BD0DBF8F0
:10095000001006EBD416B1422BD104F07F034EF603
:10096000602659F82330C2F2000623F0704393B199
:100970000134A246EE680137BE4208D9A04538BF0F
:10098000022406F1010638BFA246B442D6D900209F
:1009900009B0BDE8F08F631C0199CAEB03029142D4
:1009A00073D01C46E6E7DBF8001006EB1426B142D4
:1009B00019D0029B1B78F3B94EF65C23C2F20003F8
:1009C00018680378FE2B38D04EF66022C2F200027F
:1009D0003146FFF725F90028D9D095F82030CBF81B
:1009E0000060102BB9D1E3B24EF6602639F813300F
:1009F000C2F20006BBE7039B186802784EF65C2340
:100A0000C2F20003FE2A049300F0A6804EF6602294
:100A1000C2F20002FFF7ECFA049B0028B7D04EF6B2
:100A20005822C2F2000204921168D1B902991868E2
:100A300000220A700378FE2BC6D14EF66020C2F267
:100A400000003146FEF740FFB0FA80F04009C2E7EF
:100A5000A1F10103B3FA83F35B09D0F800A0069378
:100A60004BE7039A079310680278FE2A00F09B80F8
:100A70004EF66022C2F20002FFF7BAFA079B002886
:100A800085D0049900220A60D0E7012C7FF67FAF61
:100A9000EB6801339C423FF67AAF6FF0704221461B
:100AA0002846FFF7A9FD00283FF471AFA2455ED2AA
:100AB00004F1FF38B8F1010F7FF669AFEB6801333D
:100AC0004345FFF464AF4EF658234EF66049C2F238
:100AD0000003C2F2000901932EE007EBD817BA42D7
:100AE0000AD000213846FFF785FE00283FF44FAFBB
:100AF00095F82020102A2AD008F07F0246F82240DC
:100B000099F80020297E42F00102012989F800208D
:100B100003D9AA68019B17441F60C24527D008F17A
:100B2000FF38B8F1010F3FF432AFEA680132904567
:100B300004F1FF343FF62BAF95F82020EF69102A1F
:100B4000DBF80020C9D107EB1827BA42C9D15FFAF8
:100B500088F226F81240D3E74EF66020C2F2000079
:100B6000FEF722FFB0FA80F04009049B55E7059B91
:100B7000196871B101297FF60AAFEB680133994218
:100B80003FF605AF52462846FFF736FD00283FF4F2
:100B9000FEAE059BC3F800A0069B13B10AF101034A
:100BA0002B600120F4E64EF66020C2F20000FEF752
:100BB000FBFEB0FA80F04009079B60E72DE9F84F93
:100BC000C36801338B423DD390F82030C46949F2A9
:100BD000B038102B17460E460546C1F6FF7813D0E5
:100BE00004EBD114D8F800108C4213D14EF66023D8
:100BF00006F07F01C2F20003012053F8213023F0F8
:100C000070433B60BDE8F88F04EB1124D8F8001066
:100C1000A14220D04EF6604AC2F2000A4EF65C298C
:100C20009AF80030C2F2000903BBD9F8000003783B
:100C3000FE2B3FD04EF66022C2F200022146FEF7A4
:100C4000EFFF10B90020BDE8F88F95F82030C8F804
:100C50000040102BCAD14EF66023F1B2C2F200035D
:100C6000012033F811303B60BDE8F88FD9F800005F
:100C70000378FE2B12D04EF66022C2F20002FFF77C
:100C8000B7F90028DED04EF6582BC2F2000BDBF885
:100C90000010E1B900238AF80030C6E74EF6602064
:100CA000C2F20000FEF780FEB0FA80F04009002892
:100CB000E9D1C7E74EF66020C2F200002146FEF7F8
:100CC00003FEB0FA80F040090028BED1BAE7D9F897
:100CD00000000378FE2B0BD04EF66022C2F2000219
:100CE000FFF786F90028ADD00023CBF80030D1E71C
:100CF0004EF66020C2F20000FEF756FEB0FA80F019
:100D00004009EFE790F8392090F83800101A704742
:100D100090F8383090F839209A4205D95A1C03448B
:100D200080F83820187E70474FF0FF30704700BFC2
:100D300090F8383090F839209A4286BF1B18187EF8
:100D40004FF0FF30704700BF704700BF38B5054611
:100D5000B0F85E0090B195F85D301446C3F1210201
:100D600094420CD805F13B001844224604F0CEFE14
:100D700095F85D30234485F85D30204638BD01206C
:100D800014462871EEE700BFB0F85E306BB190F802
:100D90005D30202B07D8C218013380F85D30012068
:100DA00082F83B107047012303710020704700BF99
:100DB0000023426980F8383080F8393080F85C30A0
:100DC00080F85D3080F85E3080F85F3006CA30B45D
:100DD0000D68046943662A4383660A60A37041690B
:100DE00090F861300C680B444FF6CC721D7A5B7B37
:100DF000C0F20E0202EBC5051B026D6803F4E0634E
:100E000043F064032B6090F862300B449D7CDB7DE3
:100E100002EBC5021B02526803F4E06343F0640373
:100E2000136022684B681A4205D003692C225A705D
:100E3000036904229A71036920225A71036980228E
:100E40009A7030BC704700BF2DE9F0474FF234670D
:100E5000C2F2000782B03B6800934FF6CC79DDF810
:100E6000008002690646C0F20E0900214FF4967513
:100E7000D3789B065BD53B680193019BC8EB0303CA
:100E80000F2BF5D949B1102BF2D0002090703369A7
:100E900080229A7002B0BDE8F087726996F86130DE
:100EA00013440521187A05F06BFB726996F86130DE
:100EB0001344012193F812A0504605F061FB092468
:100EC0000021504605F028FB2B46013BFDD10121B6
:100ED000504605F021FB2B46013BFDD1013CEFD1F3
:100EE000706996F8611001444FF416720C7A4B7BCE
:100EF00009EBC4011B02496803F4E06343F0640397
:100F00000B6096F862300344997CDB7D09EBC101EC
:100F10001B02496803F4E06343F064030B60013A89
:100F2000FDD13269D3789B064FF00101A3D4012093
:100F300002B0BDE8F08700BFF0B503691222DA7095
:100F40000269937803F0200385B004460D46002B18
:100F500061D0B42393704FF23461C2F20001226970
:100F60000B680093009E05E00B680193019B9B1B9F
:100F7000042B42D8D37803F0200303F0FF00002BAA
:100F8000F2D094F85D30002B31D04FF0000E4FF0CE
:100F9000020C04EB0E0393F83B3013710B680393C0
:100FA000039F206907E09B060DD50B680293029B07
:100FB000DB1B052B28D8C378DBB203F0020202F05A
:100FC000FF06002AEFD080F803C02669F378DBB271
:100FD000DF0632462DD49F062BD5DB0731D40EF128
:100FE000010E94F85D305FFA8EFE7345D1D8002073
:100FF0001DBB002384F85E3004E0907023698022DA
:101000009A70042005B0F0BD867023698022042008
:101010009A7005B0F0BD03F0FF06FFF715FF10B999
:10102000042005B0F0BD236984F85F60B0229A7097
:1010300091E78023B3700420DAE726698023B37038
:10104000D7E7BEF1000F0CBF02200320F6E700BF78
:101050002DE9F04306690024122780F8384080F813
:101060003940F770D0F810E09EF8024004F02004F8
:1010700089B00546884616461F46002C48D0B42342
:101080008EF802304FF23464C2F200042A692368F9
:101090000093009905E0236801930198401A042801
:1010A0002DD8D07800F0200000F0FF090028F2D001
:1010B0004FEA480343F00103DBB213712368029344
:1010C00002982A6905E0236803930399091A052900
:1010D00015D8D17801F0020101F0FF090029F2D002
:1010E0000220D0702B6993F8039019F011091BD1DD
:1010F000FEB9002F0CBFA02280229A7004E082F873
:1011000002902B6980229A70484609B0BDE8F083AE
:1011100004F0FF09FFF798FE0028F5D02B6985F849
:101120005F90B0229A70ADE780229A704FF000096C
:10113000EAE7012E76D0A0229A7029690B79CE4673
:101140004FF0A80C23680493049A05E023680593E4
:10115000059B9B1A052B4CD8CB7803F0020303F0B8
:10116000FF08002BF2D0C8702969CB78DBB213F0EE
:10117000100F0A465CD19B065AD5013EF6B2012EED
:101180004BD0BEF11F0F3DD90B79012EDAD1236868
:101190000693069805E023680793079B1B1A052B07
:1011A00055D8D37803F0020303F0FF01002BF2D0EF
:1011B0000223D3702A69D378DBB2D9063AD49B06CE
:1011C00036D5B0239370BEF11F0F2B6941D805EBC4
:1011D0000E02197911760EF1010E5FFA8EFE00BF34
:1011E00000BF00BF0FB180229A7085F839E0F14648
:1011F0008AE781F802802B6980229A70F14685F88F
:1012000039E081E705EB0E0391F8048083F818803C
:101210000EF1010E5FFA8EFEB7E781F802C0296970
:101220000A46AEE7A8229A702A69CE461379AEE73D
:10123000F14669E710214FF49673D170013BFDD15F
:101240002A69937803F0F703F14693705CE7917095
:10125000D1E71A79C3E700BF38B549F22044C1F697
:10126000FF742269D578EDB2E9062BD51023D3702F
:101270006B0626D505F0040505F0FF03002D6CD0A4
:101280004EF66143C2F20003616E002249F220452E
:101290001A7084F85D20C1F6FF75002974D0884764
:1012A00095F85D30002B6FD02369D0229A702369A6
:1012B00094F83B201A712369012284F85C200222F1
:1012C000DA7038BD05F0400303F0FF00002BD1D1E8
:1012D0009379DBB203F0600160295CD0937803F06E
:1012E000100303F0FF01D3B115F0010545D194F8C7
:1012F0005C1094F85D0049F220438842C1F6FF7308
:1013000055D95818013190F83B0083F85C101071E2
:101310002369D0229A7023690222DA70D1E784F817
:101320006010937943F020039371236994F8390096
:10133000197949F220421F28C9B2C1F6FF72BED8FE
:101340004EF66144C2F200042478002CB7D0141881
:101350000130217682F83900B1E7226984F839300A
:10136000C023937023694EF66142C2F200021979DC
:10137000012111700222DA70A3E7C0239370236960
:101380001A790222DA709CE70122002384F85D209A
:1013900084F83B3088E703F0DF039371A36E23B139
:1013A00084F8380094F839009847226996E7157157
:1013B000AEE700BF38B549F28C44C1F6FF7422692C
:1013C000D578EDB2E9062BD51023D3706B0626D560
:1013D00005F0040505F0FF03002D6CD04EF66143C7
:1013E000C2F20003616E002249F28C451A7084F843
:1013F0005D20C1F6FF75002974D0884795F85D30EF
:10140000002B6FD02369D0229A70236994F83B2077
:101410001A712369012284F85C200222DA7038BD37
:1014200005F0400303F0FF00002BD1D19379DBB22C
:1014300003F0600160295CD0937803F0100303F09F
:10144000FF01D3B115F0010545D194F85C1094F873
:101450005D0049F28C438842C1F6FF7355D9581894
:10146000013190F83B0083F85C1010712369D022A1
:101470009A7023690222DA70D1E784F860109379B8
:1014800043F020039371236994F83900197949F2E4
:101490008C421F28C9B2C1F6FF72BED84EF6614415
:1014A000C2F200042478002CB7D014180130217641
:1014B00082F83900B1E7226984F83930C02393708B
:1014C00023694EF66142C2F20002197901211170BE
:1014D0000222DA70A3E7C023937023691A790222EB
:1014E000DA709CE70122002384F85D2084F83B3009
:1014F00088E703F0DF039371A36E23B184F838000B
:1015000094F839009847226996E71571AEE700BF55
:1015100038B549F2B434C1F6FF742269D578EDB21A
:10152000E9062BD51023D3706B0626D505F00405EC
:1015300005F0FF03002D6CD04EF66143C2F20003AC
:10154000616E002249F2B4351A7084F85D20C1F64C
:10155000FF75002974D0884795F85D30002B6FD057
:101560002369D0229A70236994F83B201A71236969
:10157000012284F85C200222DA7038BD05F04003B5
:1015800003F0FF00002BD1D19379DBB203F06001AF
:1015900060295CD0937803F0100303F0FF01D3B10E
:1015A00015F0010545D194F85C1094F85D0049F2FE
:1015B000B4338842C1F6FF7355D95818013190F8F9
:1015C0003B0083F85C1010712369D0229A70236964
:1015D0000222DA70D1E784F86010937943F0200397
:1015E0009371236994F83900197949F2B4321F28AC
:1015F000C9B2C1F6FF72BED84EF66144C2F2000411
:101600002478002CB7D014180130217682F83900E4
:10161000B1E7226984F83930C023937023694EF60C
:101620006142C2F200021979012111700222DA70BE
:10163000A3E7C023937023691A790222DA709CE72A
:101640000122002384F85D2084F83B3088E703F012
:10165000DF039371A36E23B184F8380094F8390046
:101660009847226996E71571AEE700BF30B44FF690
:101670001075C0F20E05417100210560C27203733E
:1016800001718172417330BC704700BF38B549F2B7
:1016900020444379C1F6FF7401255B0008224273A0
:1016A00084F83B3084F85E5084F85D50417B2046DE
:1016B000FFF76AFB29462046BDE83840FFF73CBCEF
:1016C0002DE9F84349F220444379C1F6FF7401251E
:1016D0005B0084F83B3084F85E5084F85D50437BB7
:1016E00001F0F00949EA050806460F01204648EADC
:1016F0000301FFF749FB29462046FFF71DFC7379DC
:1017000084F85E50AB4084F83B3084F85D50717BC8
:1017100041F0050149EA01012046FFF735FB4FF092
:101720003C0929462046FFF707FCFFB24B46013B28
:10173000FDD1737984F85E50AB4084F83B3084F877
:101740005D50717B204648EA0101FFF71DFB40F622
:10175000B83829462046FFF7EFFB4346013BFDD151
:10176000737984F85E50AB4084F83B3084F85D5068
:10177000717B294339432046FFF706FB2946204663
:10178000FFF7DAFB737984F85E50AB4084F83B30A6
:1017900084F85D50717B41F0050139432046FFF725
:1017A000F3FA29462046FFF7C7FBB9F10109FCD13E
:1017B000737984F85E50AB4084F83B3084F85D5018
:1017C000717B294339432046FFF7DEFA294620463C
:1017D000FFF7B2FBB8F10108FCD12846BDE8F88359
:1017E0002DE9F84349F220444379C1F6FF740125FD
:1017F0005B0084F83B3084F85E5084F85D500F46FF
:10180000417B07F0F008064648EA01012046FFF751
:10181000BBFA29462046FFF78FFB737984F85E50A8
:10182000AB4084F83B3084F85D50717B41F004019B
:1018300048EA01012046FFF7A7FA4FF03C09294684
:1018400020463F01FFF778FBFFB24B46013BFDD13D
:10185000737984F85E50AB4084F83B3084F85D5077
:10186000717B204648EA0101FFF78EFA40F6B8384E
:1018700029462046FFF760FB4346013BFDD17379C3
:1018800084F85E50AB4084F83B3084F85D50717B47
:1018900020463943FFF778FA29462046FFF74CFBEC
:1018A000737984F85E50AB4084F83B3084F85D5027
:1018B000717B41F0040139432046FFF765FA294660
:1018C0002046FFF739FBB9F10109FCD1737984F89F
:1018D0005E50AB4084F83B3084F85D50717B20460D
:1018E0003943FFF751FA29462046FFF725FBB8F1A7
:1018F0000108FCD1BDE8F883F0B54FF62073C0F2C3
:101900000E03144606460F460FCB85B0757A0DF1CF
:10191000100E0EE90F00A5423CBF05F1FF34E4B202
:1019200004AB03EB8404304654F8101C394461F0D6
:101930007F01C9B205B0BDE8F040FFF751BF00BF5D
:10194000C17901F0FD01C17141F00801FFF748BF05
:10195000C17901F0FE01C17141F00801FFF740BFFC
:101960002DE9F04F01F00701C90083B041F04001BB
:1019700092460546FFF734FF41F2C16349F2204425
:101980000AF10702C0F201030AF1FF3B0092019342
:10199000C1F6FF7401264FF03C09ACE06A7984F887
:1019A0005E60520084F83B2084F85D6095F80DE09D
:1019B00001F0F00A4AF0010849F220400F01C1F697
:1019C000FF7048EA0E01FFF7DFF949F220400121DC
:1019D000C1F6FF70FFF7B0FA697984F85E604900DC
:1019E00084F83B1084F85D60697B49F2204041F047
:1019F00005014AEA0101C1F6FF70FFF7C5F949F296
:101A000020400121C1F6FF70FFF796FAFFB24A4667
:101A1000013AFDD16A7984F85E60520084F83B2077
:101A200084F85D60697B49F2204048EA0101C1F613
:101A3000FF70FFF7A9F949F22040012140F6B838BC
:101A4000C1F6FF70FFF778FA4246013AFDD16A7994
:101A500084F85E60520084F83B2084F85D60697B06
:101A600049F2204041F001013943C1F6FF70FFF710
:101A70008BF949F220400121C1F6FF70FFF75CFAB3
:101A80006A7984F85E60520084F83B2084F85D60D7
:101A9000697B49F2204041F005013943C1F6FF70EE
:101AA000FFF772F949F220400121C1F6FF70FFF7FC
:101AB00043FA4A46013AFDD16A7984F85E605200E1
:101AC00084F83B2084F85D60697B49F2204041F056
:101AD00001013943C1F6FF70FFF756F949F2204082
:101AE0000121C1F6FF70FFF727FAB8F10108FCD118
:101AF000009B5B450CD02A68019B12681BF8011FF4
:101B00009A423FF44BAF28469047009B5B45F2D189
:101B100003B0BDE8F08F00BF10B501210446FFF708
:101B20005FFE4DF2C043C0F20103013BFDD1A37A39
:101B300003B910BD20468021BDE81040FFF750BE1C
:101B4000012A2DE9F843064603D9817941F00801BD
:101B50008171727213B1012A00F04D81322004F0BC
:101B600073FD49F220447379717BC1F6FF7401253E
:101B70005B0084F83B3084F85E5084F85D50737BE2
:101B800020461943FFF700F929462046FFF7D4F90C
:101B90004FF47A7004F058FD737984F85E50AB40CE
:101BA00084F83B3084F85D50717B204641F0300171
:101BB000FFF7EAF829462046FFF7BEF9737984F863
:101BC0005E50AB4084F83B3084F85D50717B20461A
:101BD00041F03401FFF7D8F84FF03C082946204681
:101BE000FFF7AAF94346013BFDD1737984F85E50B3
:101BF000AB4084F83B3084F85D50717B204641F067
:101C00003001FFF7C1F840F6B83729462046FFF704
:101C100093F93B46013BFDD141F6B069C0F204099E
:101C20004B46013BFDD1737984F85E50AB4084F89C
:101C30003B3084F85D50717B204641F03001FFF766
:101C4000A3F829462046FFF777F9737984F85E50A8
:101C5000AB4084F83B3084F85D50717B204641F006
:101C60003401FFF791F829462046FFF765F943460E
:101C7000013BFDD1737984F85E50AB4084F83B3072
:101C800084F85D50717B204641F03001FFF77CF80D
:101C900029462046FFF750F93B46013BFDD1B9F1FB
:101CA0000109FCD1737984F85E50AB4084F83B3075
:101CB00084F85D50717B204641F03001FFF764F8F5
:101CC00029462046FFF738F9737984F85E50AB4017
:101CD00084F83B3084F85D50717B204641F034013C
:101CE000FFF752F829462046FFF726F94346013B05
:101CF000FDD1737984F85E50AB4084F83B3084F8B2
:101D00005D50717B204641F03001FFF73DF82946D8
:101D10002046FFF711F93B46013BFDD142F2283343
:101D2000013BFDD1737984F85E50AB4084F83B30C1
:101D300084F85D50717B204641F02001FFF724F8C4
:101D400029462046FFF7F8F8737984F85E50AB40D7
:101D500084F83B3084F85D50717B204641F02401CB
:101D6000FFF712F829462046FFF7E6F8B8F1010818
:101D7000FCD1737984F85E50AB4084F83B3084F832
:101D80005D50717B204641F02001FEF7FDFF2946A2
:101D90002046FFF7D1F8013FFDD1B179304641F03F
:101DA0002001FFF71DFD0423F37130460C21FFF7DE
:101DB00017FD29463046FFF713FD4DF2C04365F38A
:101DC0001F43013BFDD1B37A1BB180213046FFF7A1
:101DD00007FD0224304634720621FFF701FD21463B
:101DE0003046FFF7FDFC4DF2C043C0F20103013B5A
:101DF000FDD1BDE8F883B37943F00403B371ADE6D8
:101E000010B5044649F22040C1F6FF70FEF7D0FF3E
:101E10000023A371227BE17A2046BDE81040FFF742
:101E20008FBE00BF704700BF26290BD80346013183
